:100000000100000000000000000400000094511AEC
:100010001CF09FE51CF09FE51CF09FE51CF09FE5A0
:100020001CF09FE51CF09FE51CF09FE51CF09FE590
:100030000C440F0A182D0400B42C0400C42C040036
:10004000C82C0400D82C0400E82C0400F82C040070
:10005000042D0400000000EA0AEC00EA28008FE208
:10006000000C90E800A08AE000B08BE001704AE24A
:100070000B005AE103EC000A0F00BAE814E04FE26B
:10008000010013E303F0471013FF2FE13C3B040092
:100090008C3B04000030A0E30040A0E30050A0E34C
:1000A0000060A0E3102052E27800A128FCFFFF8A44
:1000B000822EB0E13000A128003081451EFF2FE1E3
:1000C00004309FE503308FE013FF2FE1E5B3030019
:1000D000002070470200144810B50068682109F339
:1000E0006AF910BD10B5104C206800280CD101F041
:1000F000CFFB20600D4A2021A06009F35CF90C4A77
:100100006068202109F357F910BD10B5064C20682E
:10011000002808D00022132109F34DF9206809F3C3
:100120002EF90020206010BD00000004B5B50300CA
:10013000F1B5030010B542F036EE05F33FF90020AB
:1001400010BD10B5EF480C00FFF7C4FFEE49486B37
:1001500002229043486321000A2042F096EE0120DB
:1001600010BD70B50D0003F0F5FE0400E548401C1D
:10017000FFF7B0FFE549E0074C6002D029000520F9
:1001800015E0A00702D52900062010E0600702D57F
:10019000290007200BE0200702D52900082006E0EF
:1001A000E00602D52900092001E02900002042F0E4
:1001B0006CEE012070BDF1B50020D5490E68D54F19
:1001C000340005000AE0E10706D0A9007A58002AA9
:1001D00002D000993000904764086D1C002CF2D1C9
:1001E000012807D0C7481938FFF774FF009900208D
:1001F00042F04AEEF8BDC54910B5886005F045FBF0
:1002000010BD202800D3FEE7C24A80001358002BFF
:1002100000D0FEE7115000207047BE4A0021800048
:1002200011500800704702688368C16810001847C1
:1002300070B5052804D2B84D84002B59002B01D08D
:10024000012070BD2C23B44E4343DC3E9B192B513F
:1002500035000401F03528516019C2608160002129
:100260004160AE4919615861002070BDFEB50E00B5
:100270001700052815D2A8490201143155186968DC
:10028000A54B840000290DD101220197009602920E
:1002900018594369026906F373FC002801D1012053
:1002A0006860FEBD18591D0006F3A6FC28593A00E7
:1002B000310006F353FC285906F340FCFEBD934978
:1002C00070B50878401C0006000E08700121490432
:1002D0004018FFF7FFFE8C4D6C6AE00705D003F372
:1002E0006CE909F3BBF8A81768628D4EA00709D521
:1002F0002020F0600221C9436962B1680143B16006
:1003000009F3A4F8600705D5A86A04218843A86208
:1003100009F3C5FB20070AD5A86A08218843A8620B
:100320008020F060C9436962B1680143B160012077
:1003300070BD70B501247A4D8440EC6000203CF023
:10034000E4FCA8682043A860012070BD0121744A24
:10035000814010B5D1600D3800D5FEE7022800DBE2
:10036000FEE7704C00238000041923606D4C40347C
:1003700000190362906808439060012010BD70B5B9
:100380000125674E8540F56003F0BCFD0400400583
:1003900032D509F030FA402802D103201CF024F9AC
:1003A00002F0C7FD002815D002F07BFC002809D020
:1003B00029201CF019F9012120008902084003F0CE
:1003C000ACFD19E002F0F2FC002815D032201CF040
:1003D0000BF911E00AF010FB00280DD011F0EAF83B
:1003E000002809D01AF0A1F9002805D019F033FF30
:1003F000002801D111F022F9600708D504F032FD80
:1004000020000421084003F088FD04F08DC200495B
:1004100001000000FC030000000400005AEF5E131E
:1004200070FD200003F088FDB0682843B060012013
:1004300070BDF8B5414DEC68E00702D0A817E86040
:100440000440200606D58020C043E8608020844315
:1004500003F081FD200407D50126F603300003F0E8
:100460007AFDF043E860B4436003400F06D00720F4
:10047000000421000140C943E96084430B262000A9
:1004800036053040070005D0380002F053FBF84332
:10049000E860B443E000400F09D00727BF062600FC
:1004A0003E40300002F0D8FAF043E860BC43E0067A
:1004B0000FD51020C043E8601020844303F07AFE7B
:1004C000002806D010F0E4F9002802D0102002F035
:1004D000C1F9002C06DA0120C00702F0D8FA18484A
:1004E000E860044081200003044205D0200002F0AF
:1004F0006FF9200005F06EFE0E4988680122120592
:1005000010438860F8BD0B4B0122120510B5DA606C
:10051000FFF78FFF012010BD5A000100003400805A
:100520001400000400310080A4C40004642C000402
:10053000170200000030008040E800808022008028
:10054000FFFFFF7F30B5040020202081656920185F
:10055000AD7905706469E47944700171090A4171EB
:10056000110A8271C171190A8370C17030BDFFB563
:1005700081B0002206000D000398417800780F0238
:1005800007432037380034300104FD48090C1BF3C1
:1005900031F8040037D038001430A0802020666184
:1005A00020812018142100901AF362EB3B04049A76
:1005B0001B0C14212000FFF7C5FF002D12D0288945
:1005C0002E0028811C360B20072130567156401A08
:1005D0003EF0F1F800990873072030563EF0DEF83F
:1005E0000099487334202081039920183A001AF3A7
:1005F0007AEA002120003BF0B6F8207B202805D1C4
:1006000020003BF08DF8002005B0F0BD20202081B7
:100610003FF07BF8002802D005201BF0EFFF3BF0F5
:1006200043F8D94B0500D74821001C680022006818
:100630000523A04728003BF03BF80120E4E7FFB585
:100640000120904004060E0083B003991120240E6F
:1006500040010F18F879150020422FD1FF22913266
:10066000462301A902A811F002FD002826D0F8793E
:1006700017212043F871019C103420001AF3F8EA86
:100680000698002801D1052000E00D206072257237
:100690002000627A0C990A301AF324EA310006220B
:1006A0000C31A01C1AF31EEA607A01990A30887294
:1006B000000AC8720299039811F0A4FC07B0F0BDBB
:1006C000F3B5FF30401C0500006A81B0002803D05C
:1006D00009F38DFA00202862686A401C01D10120CC
:1006E000FEBDA84F00241FE0A8481AF3ECFF060047
:1006F00002D03868002801D10020FEBD02980028F1
:100700000ED13FF002F8002802D005201BF076FF42
:100710009D4B31001E68002238680523B04702E077
:1007200030003AF0FDFF641C686AA042DCD800206B
:100730006862D4E795490020086048608860C86016
:1007400008612C3948627047F8B504000E00904DDE
:100750003AF0AAFF070021002800FFF7B1FF8B4CF9
:100760000C3C012E06D1FF21213128001AF356EA54
:100770000020A0720020C043208138003AF098FF8A
:10078000FFF7D8FFF8BD81482C38406A002801D017
:10079000401C01D10020704701207047F3B583B0A1
:1007A00000210500049EFF30B61D2130009101910B
:1007B000029049E06A7801202C1D0021012A0FD007
:1007C000022A12D0032A13D13388724A93420FD1DE
:1007D000738893420CD1B388934209D1012107E079
:1007E0003178C907C917491C02E03178C907C90F18
:1007F000002900D10020002717E060880499627862
:100800000818211D3AF07BFB01002078802803D1D5
:100810000120002907D005E0812803D1D7D9D51CB4
:1008200001000000F80700000004000009358D7F7A
:10083000002901D0012000E0002008347F1C01289D
:1008400004D12878B842E2DC0120009001982435D8
:10085000401C01900098002804D102980199807AE8
:100860008842B1DC0098D9E60800FF310022491C1B
:100870000A6211002EE770B501253BF0D2FF002877
:100880000CD0474C2C3C606A401C07D045480121E5
:10089000FFF720FF05000020C0436062280070BD04
:1008A00010B53BF0BEFF002805D13D482C38416A09
:1008B000491C00D1416210BDF8B505000C000027AD
:1008C0003AF0FCFE0090E168A06800232E00594039
:1008D000584008433BD0A088A779344BC119403910
:1008E0002A1A8C460100D21840315B009A4205D981
:1008F0009A1CA84201D2AE1A00E0AE18664524DD6B
:100900008E4222DAB0420FDD801B0604360CE1680D
:10091000A068320019F3BAEEE160B919A1710121A2
:100920000843A580A06018E0301A0204120C974218
:1009300000D2A2710021012019F3A8EEA268E36899
:1009400010431943E160A06007E011F08EFC002025
:10095000A5800121A071A160E06000983AF0B2FE8C
:10096000F8BDFFB59FB00600080037680021179159
:1009700021997C6900291ED060301E901AF3FEE98F
:10098000229905004118C0782031400610D4B8885B
:1009900023B0F0BD901900040400000434030004E7
:1009A00050C6000424C50004FFFF0000FF0700003C
:1009B0002888882801D80020EAE719AA189100920F
:1009C000219918981AAA17AB0DF3F4F828000DF323
:1009D00018F9002853D0002104AAFF4801AB07C32F
:1009E00018ABFE4A00921D7910AB1A7F38002B001D
:1009F0001AA90CF332F905002DD11120400120185D
:100A0000C179090624D5002C0CD00D21890161186B
:100A1000896B002906D018AB1A79920068328B587E
:100A20005B1C8B50C1794906490EC1711E981AF39F
:100A3000A6E918AB1D7921992A01521B52180E32D2
:100A40000092010010AB1B7F2A002000FFF701FE7F
:100A500000203060AFE7356028891E9940191AF3ED
:100A60009EE90088A88011204001201818AB1B794E
:100A700001263200C1799A409143C1711DE010AB4B
:100A8000197F009101952A8818991898843A091DB0
:100A90001AAB10F368F806001CD0112018AB1A79B5
:100AA000400120180123C17993409943C1712888DE
:100AB00008382880B8880838B880002C08D00D2065
:100AC00080012018806B002802D0416E491C4166CD
:100AD00030005DE7002C14D00D2080012018816BC0
:100AE00000290ED018AB1A79920068328B585B1C23
:100AF0008B50816B0A69521C0A61806BC168491C6A
:100B0000C1601E981AF33AE9010018AB1879219ACE
:100B100003011B1A9A180E320092020010AB1B7FC1
:100B20002000FFF796FDD3E700280CD00D218901A6
:100B30004118886B002806D00269521C0261886B3C
:100B4000C16C491CC1647047F0B58446059D1468AA
:100B50002E68A64203D11F880888874203D9601CEB
:100B600003D0A64201D2012013E76046002803D03B
:100B7000188808802868106000200AE7FFB585B053
:100B8000002405001E000E9F20F046FF002847D0DD
:100B90003000603004901AF3F2E88078403604099F
:100BA000307E46070698760F808B03900698006A81
:100BB000029028003FF078FC00282BD068790228AA
:100BC00028D0082C26D3082E02D3012009B0E0E655
:100BD00030001BF3CDF9810002AA00921D224919B1
:100BE00052018A1840003B21401909014118079819
:100BF00003ABFFF7A9FF040004981AF3C0E8784A92
:100C00000C3031001AF3E0FE76490968884207D2B9
:100C10000020DBE702AA00923A002C32111DE6E721
:100C20002000D3E7F0B5012A069D059C9055D1C858
:100C300001000000F40B000000040000FD5AF8CB96
:100C400013D0022A15D0042A2DD14A780E78120228
:100C500092194E790F793602F619CF7812043602BE
:100C6000120CF6198978360212E00A788E78120290
:100C700002E04A780E7812029219CE798F79360204
:100C8000F6194F79120436020979120CF619360258
:100C9000711826688E4202D11F88974203D2771CB2
:100CA00003D08E4201D901207DE6002801D01A80B0
:100CB00021602A8007980160002074E6FFB583B0A8
:100CC00004001E000C9F0E9D3FF0F8FB002820D072
:100CD000607902281DD0082E1BD3082F01D30120D4
:100CE00000E538001BF34EF9030080001D250019B4
:100CF0006D01119A109940196D4607C558003B21A6
:100D00000019090143180D9A05990498FFF794FFFB
:100D1000E8E40FA807C86C462B0007C4F3E7F7B553
:100D200092B014000F00129800680D9000200A90F5
:100D30000D9845690800603011901AF32AE8060002
:100D400020300990280020F071FE21002C311091F4
:100D5000091D403700280F9122D0109807AA08A932
:100D600003AB07C36B46E0790F9A0107387E090F82
:100D70004007400F07C30021B078099A03092800F3
:100D8000FFF79CFF00280BD0002D08D00D2080011C
:100D90002818806B0028F8D0016D491C016593E08C
:100DA00030888828FBD922004C3288380304111F70
:100DB000081F0692021F0591049003920C393838DF
:100DC0001C3A029101900092387E1B0C47077F0F5E
:100DD0001A00099930003B000FF3E7FD07003000CF
:100DE0000CF319FF002847D0002007E060FD02C087
:100DF0002CB901C0DCCB000498F800040AA90091CA
:100E00000BAA01920A900D9B099A310038000CF34D
:100E1000E2FD002858D0614A0092614A614B0D986A
:100E200031001AF3FDFC002802D1129908604BE052
:100E300012990600086001890818119919F3B8EF92
:100E40000E900A9800284AD00BAA009209990E9891
:100E5000230032000CF3EEFD070040D1002D08D036
:100E60000D2080012818806B002802D00168491CE1
:100E700001600E98807922E0002F28D03807800F7B
:100E80000FD0002D20D00D2080012918886B00285C
:100E90001AD0C26C521CC264886B0169491C016182
:100EA00012E0B80710D5002D08D00D2080012818B9
:100EB000806B002802D00168491C0160B079C1072D
:100EC000C90F280042F04AE8002015B06BE53088D1
:100ED000143830800D980D99808814388880079CCC
:100EE0006B461A8C10990F9823000CF3BEFD002F4F
:100EF0000AD1002D08D00D2080012818806B002811
:100F000002D0416E491C41660120DEE7F7B582B090
:100F1000140000250298076803980197603019F3C0
:100F200038EF0600C0787F69400605D42037B87DC9
:100F3000400731D401252FE0002C01D100209CE492
:100F4000A07AC00721D0E0790007000F012805D161
:100F50000399220001A8FFF7E2FE05E003992200B1
:100F6000002301A8FFF707FD02990500019808601A
:100F7000B079C00710D1002D0ED0A07980070BD515
:100F8000210038003BF08BFC06E00D208001381872
:100F9000806B8168491C816028006EE420B901C023
:100FA00028B901C060FD02C070B505000089441970
:100FB0003EF0BFFB00280AD0607B217B0002084383
:100FC0000B2804D00A2802D005201BF02BFBFD4B78
:100FD000FB481C680022290000680223A04770BD5E
:100FE000F948010008394860F848012141700021A2
:100FF00001707047F449002008394860F34948708F
:101000000870704710B5F14C6078002807D00120B7
:101010002070A06D002802D00EF394F8606510BD1A
:1010200070B53AF055FB0500E9481AF360FB04007F
:1010300028003AF051FB02250DE020002685094DDD
:1010400001000000F00F000000040000AE802BA79C
:101050002573FFF7B3FF3AF045FB0600E1481AF3AA
:1010600050FB040030003AF041FB002CEFD170BD82
:1010700070B53AF037FBDA4C05006078002809D0EB
:10108000D64904200856411C04D0811C02D00121FD
:1010900007F3A0FBD4480078012802D114201BF0EC
:1010A000AFFA0020207204200AF0E6FBCF480022AD
:1010B00000680C2108F3A7F9FFF7BCFF28003AF0FD
:1010C00015FB70BD10B5FFF7D3FFC54900200870B0
:1010D00048704865C649086010BDC148017A0329B7
:1010E00001D0032101727047FF2800D008407047EB
:1010F000C04910B5096839F0E6EF7D22D20019F336
:1011000028EF8905800A084301D041F06EEE10BD3A
:10111000F8B50024160005000F002200002901D0B8
:101120003889C2193BF086FB002879D0AC49087A8F
:10113000032876D00228FCD0680726D5002F24D0BB
:10114000507B117B04020C430B2C08D010DC032CC9
:101150000BD0082C09D0092C07D00A2C13D1A64893
:10116000A6490088097808430BD0FF25052615E01D
:10117000102CFAD0122CF8D04F2C04D1FF250726C2
:101180000CE004208543042608E0062E06D193488F
:101190000838406819F306EEC0056CD48F4808384B
:1011A000406819F300EE01002800FFF79DFF0028BA
:1011B00061D08B484030818B002900D18683904DCF
:1011C000002C1CD0288800280FD084490420085601
:1011D000401C0AD10800083840684079FFF788FFB2
:1011E000FFF770FF002028805CE03AF07BFA0400F3
:1011F0007C4839001AF3DDFA20003AF077FA774F8D
:101200000426083F786886573BF014FB002813D06B
:10121000734C606D00280FD0A06D00280CD004E046
:101220003AE02AE0774803F043FF0DF395FF616D44
:10123000401AA16D8842F5D3694802210172701CE1
:1012400005D0B01C03D00021300007F3C3FA786842
:101250004079FF2829D0FFF74BFF2888002824D0A9
:101260003BF0E8FA002804D0FFF72CFF002028808C
:101270001BE0288819E00020F8BD680715D5002F6D
:1012800013D03AF02FFA0400564839001AF391FAB5
:1012900020003AF02BFA08E0680706D5002F04D0AA
:1012A000FFF7C8FE3800FFF789FE0120F8BD4C4863
:1012B000602110B519F3D0EC10BDF8B500200C007A
:1012C000474F1500B882B8651DE0607821780002AC
:1012D0000843FF38163819D0A1280AD12000062D5E
:1012E00007DB4179027908027D231043DB00584374
:1012F000B865E178A27808021043291A091F0D0485
:101300002D14241D0419042DDFDCF8BDE178A2782A
:1013100009021143CE082000F2009142E9D1121DCA
:1013200011040914A942E4DC0821082E00D231007E
:10133000CA00011D2A48143019F3F2EB06E0F00050
:10134000C019002114300A0006C0761C082EF6DBF6
:10135000CFE7FFB58BB00A2000261D000A96059046
:101360000B983700406907903EF09CFF06900B9861
:101370000B990089441820314118E078C00701D149
:10138000A01D01E020001230A27894461207930FAE
:10139000012B04D16046000908286CD03AE0920F76
:1013A00002D14026092034E00388174A934209D12C
:1013B0004388934206D18388934203D101263700A4
:1013C000300026E00078C00720D00826032702203E
:1013D0001FE000000400000434030004A000000427
:1013E000DC2C000408380004680500040000000438
:1013F00014070004E0B801C0643C00048C0600043B
:101400009006000488130000FFFF0000022637004A
:1014100003202880A0780007800F022873D10D9A3E
:10142000002010700B98891D0A91406902900028D5
:1014300023D0614808900A98022208A939F07DFD5E
:1014400000281AD102983BF029FA00280D8B590583
:1014500001000000EC1300000004000011450E1410
:1014600003D002988068400704D4029807F0DEF8A1
:10147000002803D00D98012101708EE05448406887
:1014800019F39AECC005F8D40620288088E0079864
:101490004079022841D10C98002827D00C98403080
:1014A0000500007D8006400F012809D9032805D8D2
:1014B0000C98183019F380EC000701D5012200E0E8
:1014C0000022A17800200B079B0F022B03D10909F2
:1014D000090700D50120024308D0287E3D4A410774
:1014E0002000490F0C301AF38DFA059004A903AAC5
:1014F0000091019206981121490140180378059A3C
:10150000079821003AF0A1FA0398002802D00D991B
:1015100001200870049800283FD02D48406819F336
:101520004CEC304239D0A0780007800F022837D128
:10153000294EB08A002833D0C120C0000025099070
:1015400026E0B84202D0254988421ED1E08A2349CC
:10155000884207D021000A981631022239F0F7FCA0
:10156000002812D1A069401C1AD00A98022209A9A9
:1015700039F0EDFC002808D10A9821001A30183102
:10158000042239F0E4FC00280AD06D1C082D04DA8E
:10159000E8008419A08A0028D3D100200FB0F0BD44
:1015A0000120FBE70A480078C00700D001207047FF
:1015B00000B53BF054F9002805D0FFF7F3FF0028F1
:1015C00001D0012000BD002000BD0000888E000079
:1015D00098000004DCCB0004DC2C0004FFFF0000BA
:1015E000F3B591B00C001198002837D0207D0E285B
:1015F00034D214264643BB4D4021A859401CA85163
:1016000001A819F334EB200001A91CF027FD677D28
:10161000607E0090206801218068800000281FDB28
:101620000098401C02062069120E002800D00021FC
:1016300011981DF09EFE206901A9002824D10E2FCB
:1016400005D21420784340194268521C4260009829
:1016500000280BD170198168491C816013B0F0BD5E
:101660002069002800D000210022E1E700200206C6
:10167000120E142353438A5C5B199C68401CA21809
:101680000E289A60F3D3E9E7E07D002804D07019B2
:101690000269521C026103E07019C268521CC260E8
:1016A00000200206120E142353438A5C5B199C68C7
:1016B000401CA2180E289A60F3D3CFE710B5FF2480
:1016C00019348849220019F3A0EA8648210019F349
:1016D000CEEA10BD70B50D00002805D00D2189019E
:1016E0004018846B002C06D1002D03D04C2128001B
:1016F00019F3E6EA70BD7C4AD1687C484368591802
:10170000794B4160403B2162596B8668711881605A
:101710006162196BC3685918C160A16211680269DE
:1017200051180161002DA163E4D0A06C290019F3C8
:1017300054EB6069291D19F350EB2900A0690831A9
:1017400019F34AEB2900E0690C3119F346EB290043
:10175000206A103119F340EB2900606A143119F343
:101760003CEB2900A06A183119F336EB2900E06A36
:101770001C3119F332EB2900206B203119F32CEBCB
:101780002900606B243119F328EB2900A06B283164
:1017900019F322EB2900E06B2C3119F31EEB290021
:1017A000A06E343119F318EB2900E06E383119F3CB
:1017B00014EB2900206F3C3119F30EEB2900606F08
:1017C000403119F30AEB1DF0FCFA2900443119F3FA
:1017D00004EB1DF0F3FA2900483119F3FEEA70BD5D
:1017E000F0B400283BD00D2292018218926B002A9F
:1017F00035D03E4C23685B1C23609B062FD14C7E6A
:10180000D36A1B19D3620B69002B23D10D682B6F90
:10181000DE78F60707D09E783607B60F022E02D183
:101820009E7CF60702D19B79DB0702D0936C5B1C90
:101830009364D36B5B1CD363AB689B000DD4002C0B
:101840000BD093695B1C012C936106D9D3695B1C97
:10185000D36102E053695B1C5361F0BC9F7A27504F
:1018600001000000E817000000040000429FDD783E
:10187000C0E6F0BC7047002808D00D229201801805
:10188000806B002802D0826951188161704700285E
:1018900010B51AD00D239B01C318986B002806D0F1
:1018A0004469641C4461986BC36B5B1CC3630E2961
:1018B0000BD214204843104B1958491C002A1950C8
:1018C00003D0C0180169491C016110BD002809D06E
:1018D0000D2189014018806B002803D080300188D9
:1018E000491C01807047FF210348193110B519F3D5
:1018F000C8E9002010BD000064C6000440A80080B4
:10190000A8000004C0207047010002A010B507F332
:1019100042FD10BD7364696F00000000F7B515004B
:1019200006000024002A1FD1002E14D0707902284E
:1019300011D002E0012004F041F82000641C0228CC
:1019400007D20022F848110019F386FE0500F1D0F5
:101950000AE0002D08D10022F448110003233DF0D5
:10196000BAFF050000D1FEBD6E61FFF7CBFF00049A
:10197000000C288108274419122120002F7319F325
:10198000AAE9300023F0B5F820731420207100205C
:1019900060717079022803D1DF20A071002001E07E
:1019A000380AA771E071B0792070F0796070019801
:1019B000143404602800FEBD10B504000321363045
:1019C00019F388E920001C21393019F384E9203407
:1019D000A07E01210843A07610BD70B50400FFF77A
:1019E000EBFF2000FF30FF220421993039F0E4EAB8
:1019F0002000FF2158304131050019F342E9FF343E
:101A0000413401210020A161E0612075280016F316
:101A1000DFFD70BD0F21890170B54418E168002910
:101A200026D10079002803D0032801D004281FD133
:101A300039F06CFE0500BE480021FF229D324A436A
:101A40008258002A0AD1FF239D33594301220E18E0
:101A500042503000FFF7C1FFE66002E0491C022956
:101A6000EBDB280039F056FEE068002800D1FEE7E5
:101A700070BD0F2189014018C168002902D00022E1
:101A80000A60C260704710B5028912311218917055
:101A9000090AD1700F213AF0FBFE10BD0A000F2198
:101AA0008901411810B5C9682A311DF07DFE10BDAD
:101AB000F0B58FB00500149E159C1700092918D1A8
:101AC000382101A819F3DCE804206B469880994876
:101AD000D88002A806223900801C19F336E804A831
:101AE00032002100801C102304F05DF96B46188140
:101AF00005E023000022310001A816F393F9280025
:101B000001A904F0D7FE0FB0F0BDFEB50C3A0D00F0
:101B100014060600240E1021102C00D821003000DD
:101B20000A00FF30290019300831070019F30CE8CA
:101B3000FF3601970094761C2B787069AA1C092146
:101B4000FFF7B6FFFEBD70B5050048790B00C00673
:101B500020D51800603081784078090201431800D0
:101B60000922633016F34CFA040013D06078102277
:101B70000C38102800D8020028002100FF300E3158
:101B8000193039F0EEF9002804D06278A11D280040
:101B9000FFF7BBFF012070BD0F218901401810B570
:101BA000C068583016F3B6FD10BD7CB50C001500AA
:101BB000069900910F21079A890140180192C06887
:101BC0002A003930210015F34AFF7CBDFFB585B0EE
:101BD00000220E001D0001894469081803902000AE
:101BE00004A9FFF79BFE070002D1012009B0F0BD58
:101BF0000F20800100962618F268039913000498BC
:101C000030332A3216F3C0FA0498817C012910D0AF
:101C1000002200920192F2680100130030332A3250
:101C200071312000FFF7C1FF04996031C873000AC9
:101C30000874079904982B00012216F38DF901000E
:101C40003800FFF720FF0020D0E70F229201801814
:101C500010B5C068393016F35DF810BD30B504001A
:101C60000D2080012018002A8FB009D0340518CC2F
:101C700001000000E41B000000040000B6F0A8CC46
:101C8000002C10D0806B00280DD08030C5886D1CD2
:101C9000C58008E0002C06D0806B002803D080307F
:101CA00045896D1C458101A816F3C6F8200001A9DD
:101CB00004F00AFE0FB030BD70B505000F208001A2
:101CC0002C18E06828220100FF312D31DC3018F398
:101CD000B0EF01212800FFF7C2FFE3680100DC3309
:101CE00001222800FFF7C4FF70BD70B544692720AA
:101CF000400125186878002801D0002070BD200020
:101D0000FFF7DAFF0F2080012018C2680121C032DE
:101D10005161C068C0308069002803D0827AFD23F9
:101D20001A4082726970E8E7F8B5446927204001DB
:101D300027183878002809D00020F8BD501A000470
:101D40007C190004884304000404000000212000E2
:101D5000FFF785FF0F2189016518EB680100FF334C
:101D60005B1D00222000FFF783FFE8680126C030DA
:101D7000C660E868C0300169002904D1066101210C
:101D8000200020F0F4F9002120003E7022F005F937
:101D9000D2E7F7B584B005000E004769008900223C
:101DA00040190290380003A9FFF7C2FD040002D1D8
:101DB000012007B0F0BD0F200022800138180092EA
:101DC000C26802991300039830332A3216F3E6F9F9
:101DD0003100039801224031002316F3C7F80700B1
:101DE000706F00280BD0607B012108436073069858
:101DF000002801D0FF4800E0FF48A06109E00698F4
:101E0000002803D0280000F094FB02E02800FFF730
:101E10006CFF39002000FFF740FE0020C9E7FEB547
:101E200000220E00018945690F18280001A9FFF75B
:101E30007FFD040001D10120FEBD0F2000228001A2
:101E400028180092C2680198130030332A323900F2
:101E500016F3A4F93100019801224031002316F352
:101E600085F8617B012211436173E449A16101009E
:101E70002000FFF712FE0020FEBDF7B58AB0052650
:101E80000A9847690F2080013D18EC6800200890EF
:101E90000120583407900020069002E0012003F052
:101EA00097FD761E03D3E86840680128F6D10A98AA
:101EB000210016F3F9FA0028099019D00898002893
:101EC0003FD1E8683E3015F38BFD002839D0E86833
:101ED0003E3015F39AFD0028E86804D0417A0A30B4
:101EE0001DF092FC02E02A3015F331FA060002D10F
:101EF00000200DB0F0BDE8683E3016F3EBF90200AB
:101F00002100D4312000503002AB07C30D00220065
:101F10004032B439019200910B9A0C9923003000A1
:101F200016F35AFA200010222900843039F023F8E1
:101F3000002804D027210020490179184870012089
:101F40000690079800280CD0220021000A98403201
:101F500020310023FFF744FE002802D00020069025
:101F600015E00698012812D1002F09D00D2080011C
:101F70003818806B002803D06030418B491C4183A6
:101F800009992000093115F32AFF0020A06706985F
:101F9000AFE7F8B5060045690F2080012818C7682B
:101FA00030005837390016F398FA040001D10020A8
:101FB000C3E620790122022800D000223900300037
:101FC000FFF7E7FE002801D02000B6E6002D09D07B
:101FD0000D2080012818806B002803D06030418BD1
:101FE000491C418321000931380015F3F8FEDEE772
:101FF000F0B50E008DB0476916F356FA040046D0CE
:1020000032005032200001A916F34BF8012070670E
:10201000F01DF9300500806807F325FE0021A96056
:1020200031002079AC313500C03502280C9130D117
:10203000200060308178407809020143200063303D
:1020400001AA16F30EF80C98102201A938F093FF9C
:10205000002805D1272001214001381801700FE028
:102060000C98282201A918F3E4ED6B46188D2882FC
:102070000020C0432721E86000204901CF79F63DC8
:1020800001000000E01F000000040000E52A7BA022
:10209000791808705F4A21001268300090470028C4
:1020A00029D100202FE720006030817806000A0245
:1020B00040782100024363310C980B9138F065FFA2
:1020C000002801D1012012E0B078717802020A43A1
:1020D0000B990C9818F34CEDA0796B468006800F95
:1020E0006882188D28820020C043E86000202721E4
:1020F000490179180870200005E7F8B50700446920
:102100000F2080012018C668380058363100FFF7CC
:1021100079FF050005D031003800FFF78AFE00285E
:1021200001D0002013E6002C09D00D2080012018DA
:10213000806B002803D06030418B491C418329000B
:102140000931300015F355FE280000E6F8B505000A
:102150000E0000891700401981790024090716D55F
:102160004079C00709D02800FFF71DFFEFE5642084
:1021700002F0C6FF641C2406240E3A003100280039
:10218000FFF785FE0028F1D1072CF0D3DFE528000A
:10219000FFF7B3FFDBE5FEB50C000600086F170084
:1021A000401C06D1E06E401C03D1200016F324FA37
:1021B000FEBD39F0BFFA050002E0002139F0A8FAAF
:1021C000154819F3C6FA0028F7D1280039F0B6FAF5
:1021D0000022300001A9FFF7B5FB0500E8D00F2071
:1021E000800136180094F2680198130030332A32C7
:1021F000390016F32FF8F0683E3016F375F8020038
:10220000F0682030417F09E0972400004F1C000057
:102210008D1C0000B8FC000468D00004807E090713
:10222000CB0F8006C10F019816F334F9E06E401C05
:102230000128E06602D1206F401C20672100019830
:1022400001224031002315F39BFE01002800FFF717
:102250002EFCFEBDF3B581B006000F2080013518BD
:10226000E8680400FF30593007000068583400283F
:1022700020D0FC20005D00901DF060FC029A21003F
:102280003000FFF788FF0098002814D0012811D1F2
:10229000E868B14A2030017E0823491C0176009885
:1022A000210016F31DFAAD4AAD49200008237E61D6
:1022B00016F302FAFEBDA84A00982100082316F37F
:1022C0000FFAE8682030C17D491CC175FEBD70B5AC
:1022D0000E0011000F2292018418E568FF22583584
:1022E00015325051E0680622303018F342ECE068B5
:1022F00006222A30310018F33CEC9A4A9A49280009
:10230000082316F3BDF970BDFFB581B005001600B6
:102310000A9F3AF0EBFA00282CD02800FFF750FC77
:102320000F2080012C18E06802990A30320018F35F
:1023300020ECE0683A00467204992800FFF7C7FFD6
:10234000E16801204860E0682821DC3018F3ACEC3B
:10235000E0682821FF30401D18F3A6ECE068282132
:10236000FF30713018F3A0EC27200021400128181D
:102370000170417005B0F0BD0F2189014018C0689F
:10238000FF304130C0690006000E70470F218901FF
:10239000401808B5C068408F009008BD020010B515
:1023A0003AF0A4FA00280BD00F2080011018C16861
:1023B00020314A7E520852004A76C068FFF710FB6F
:1023C00010BD0F2189014018C06801222030417ED4
:1023D000114341767047F0B585B00E000B9915009A
:1023E0000A9F0C9A0400002902D1002004A904903D
:1023F0000F20800120180197009303920291C0687A
:102400002B000100FF3199313930320015F3F8F912
:10241000B0E7F0B506000F2080013418E0680F0027
:10242000417A15000A308FB01DF0F8F9002810D05D
:1024300001002B003A0001A815F334FC300001A97B
:1024400004F04CFA3000FFF7BBFBE0680121C0301C
:1024500001610FB0F0BD70B505000F2080012C1890
:10246000E0682030417EC90712D0817EC9060FD5B1
:10247000007F00220007C10F2800FFF7CAFFE068B5
:1024800001222030007F0007C10F28000A1D9C3662
:1024900001000000DC23000000040000CDBBFE1D95
:1024A000FFF7C1FF70BD0FB50F2189014018C1684A
:1024B0006B46FF319A8881310A83C1681A7AFF31ED
:1024C00081318A76C068197BFF308130C1760FBDBB
:1024D00030B50F24A4010019C468FF348134257E6F
:1024E0000D70647E4C70C168FF318131897E11703E
:1024F000C068FF308130C07E187030BD30B50F2409
:10250000A4010019C4682034A57E0D70E47E4C70CF
:10251000C1682031097F1170C0682030407F187079
:1025200030BD0F21890110B54418E06800280BD098
:10253000FF304130006A002806D007F3A8FBE068AE
:102540000021FF304130016210BDEAE70F2189010F
:102550004018C068FF307130704710B50400FFF7B5
:10256000D8FB2000FFF7F4FB002010BD558531009B
:10257000409C00008185310080969800A98531003B
:1025800070B5002503891C1866784369002E17D0A2
:10259000032E20D1002B09D00D24A4011C19A46BFB
:1025A000002C03D0803465886D1C65805B79022B1C
:1025B00002D106F005F901E0FFF7D2FD01250AE09E
:1025C0005879032801D0012805D12079012802D1AA
:1025D000080012F0E9FF280070BD10B51DF04AF99F
:1025E000002010BD10B502F0A0FF002805D0A748BC
:1025F000807DC00701D040F0F2EC10BD10B5FFF7B0
:10260000F1FF23F003FE40F0F8EB23F000FE10BDD5
:1026100010B501F087FD002812D001F082FD9C4921
:10262000012000058860401101F0DCFC22F0ADFBC8
:10263000FFF7D8FF40F0E0EB22F0C3FB01F070FDA4
:1026400010BDFEB5002439F07FF8060000F096F9C1
:1026500090480168080602D5480600D5012403F019
:10266000EEFD050002D1012003F0FDFD0120C007B1
:10267000807802210840800717D4002C1BD100224B
:102680008548009200680822012101AB3AF069F9FF
:102690000122009200221100100013000DF03AFFF9
:1026A000012819D100F06AF905E07C48006800288B
:1026B00012D1002C10D0002D0ED0754CA568E0175B
:1026C000E060E70C380001F096FCFFF7A1FF38004E
:1026D00001F088FCA56001E0FFF790FF300039F0C1
:1026E00037F8FEBDADE710B539F02EF8040040F024
:1026F0007AEC22F03BFB200039F02AF810BD70B5CF
:10270000040039F021F805006248016821430160A6
:10271000600601D4200618D5480616D5080612D53D
:1027200001F078FD5A48FF21491CC16040685C49AE
:10273000086861225205904308605A494869282276
:102740009043486101E001F065FD280039F000F890
:1027500070BD10B50DF088FC002801D1524810BDA5
:10276000524810BD10B502F093FE51494000085A7E
:10277000504B4C495843096A0B071B0F18F31EECCA
:10278000080507060609090B0B06400810BD80085E
:1027900010BDC00810BD000910BD10B5FFF7E2FF65
:1027A0004549884201D1454810BD4549884201D17B
:1027B000444810BD444A4549904219D0444A904289
:1027C00001D1444810BD444A904202D14148D23818
:1027D00010BD424A904201D1414810BD414A904249
:1027E00001D1414810BD414A904201D1404810BD3D
:1027F000080010BD70B5040038F0A6FF050025489C
:102800000168A1430160600601D420061BD548067B
:1028100001D5080617D422480168612252051143E8
:10282000016001684205114301601949C00D8860CB
:1028300001F008FD1B48416928221143416102F063
:102840000DFF0CF01FFD280038F082FF70BD114A0B
:10285000010012680020914300D101207047C000A0
:1028600005D50C4820304068002800D0004770474C
:102870000300402010B5FFF7EAFF002804D018033A
:1028800002D5102000F036F810BD0000A001008035
:1028900000300080C800000400C001C0F1EDA6CFE8
:1028A00001000000D8270000000400009E612D7187
:1028B000CC06000400210080002800803F3D00007D
:1028C0007F841E00E4340400A0860100001BB700D2
:1028D00054150000405DC600B013000000F824014C
:1028E000540D000000366E01AA0A000080BA8C0167
:1028F00000F04902AA06000000751903EB0400006D
:10290000007C9200AA1A000010B52A490400002099
:10291000086029490860C020FFF776FF01F0ABFC92
:10292000E00602D51DF098F910BD1DF036F910BD76
:102930000020E9E70221032010B51EF0B2FB0028B9
:102940000FD1032108001EF0ACFB002803D040F09B
:1029500058EB002805D1FDF770FF002801D10120B8
:1029600010BD002010BD10B501F07EFC01280CD177
:10297000FFF7E0FF002808D00DF0EBFC0F480088BF
:10298000012802D001F088FC10BD01F07CFC10BDD4
:10299000084910B509680020002900D040200649E8
:1029A0000968002901D080210843FFF7B2FEFFF734
:1029B000DAFF10BD6007000464070004E2070004AA
:1029C000052804D2664983001818085C7047FF2068
:1029D00070470A00032010B5FFF7F2FF904201D1C3
:1029E000FFF7A6FF10BDFF280CD05D4A00218B0029
:1029F0005B18D35C834202D10806000E7047491C65
:102A00000529F4D3FF207047FF280ED0544A002137
:102A10008B005B189B185B78834203D188004018B9
:102A2000105C7047491C0529F2D3FF207047052828
:102A300005D24B4983001818401840787047FF2092
:102A40007047FF280ED0464A00218B005B18D35CEC
:102A5000834204D188004018801840787047491C90
:102A60000529F2D3FF207047FF280ED03C4A0021F1
:102A70008B005B18D35C834204D188004018801817
:102A800080787047491C0529F2D3FF207047344AEB
:102A900000218B005B18D35C834207D1880040186B
:102AA0008018C0784007C017401C7047491C052992
:102AB000EFD30020704710B50024FFF794FFFF28E4
:102AC00006D0274983001818401800798007C40FE2
:102AD000200010BD70B505000C00100001F074FB63
:102AE000200001F092FA2800FFF78EFF022805D09F
:102AF000032803D0042801D0052803D1200000F0CA
:102B000073F870BD2000FFF7B4FE70BD10B504006F
:102B1000C00005D50122120311040C20FFF7DAFFD3
:102B2000200105D50122D20211040B20FFF7D2FFAC
:102B3000600105D50122920211040A20FFF7CAFFA5
:102B400010BD0120C00310B501F03EFB0120C007FD
:102B500001F05BFA0349086A80229043086210BDC5
:102B6000CC00000400280080F3B581B00F0001986C
:102B7000FFF739FF05000198FFF763FF0600019892
:102B8000FFF772FF0400032D07D1042E05D110209A
:102B900001F01AFBB00401F046FA002F1ED1019893
:102BA000FFF775FF002819D0231F18F312EA061744
:102BB0001717170A04170198FFF77DFF01000D2072
:102BC0000AE00198FFF777FF264AA90049198918FA
:102BD000C978CA080100100005F338FEFF220199E8
:102BE0001000FFF7F6FEFEBD10B50400C00203D5CD
:102BF00001210220FFF7B8FFA00207D50121032021
:102C0000FFF7B2FF01210420FFF7AEFF200203D53A
:102C100001210520FFF7A8FF01200007844205D00D
:102C20004010844202D0401084421AD1FF20820614
:102C3000A11808D0891804D0C206891804D10C2024
:102C400002E00B2000E00A20FFF7DEFE022805D09C
:102C5000032803D0042801D0052802D10121FFF761
:102C600083FF10BDCC0000043EB5040002E001204B
:102C700002F05AFA03F024F90028F8D002206B463B
:102C8000187000205C709870D8700121684603F0BD
:102C90007CF93EBD01B5B84801224068694608305C
:102CA00003F04CF92020FFF7DFFF08BD230FEEF201
:102CB00001000000D42B0000000400006A0E58C57B
:102CC000B24808B5016801222031684603F040F996
:102CD0006B46187808BD10B50400AC4898B0016880
:102CE00024220FA803F034F960070ED524220FA97F
:102CF00005A817F3C6EFA6491422684617F3C0EFDC
:102D0000A34810380FC808F02CF8200704D510ABE2
:102D10009979587907F0ADFDE00609D5FFF7D0FFA6
:102D2000002805D09B48406AC030C07FFFF7BCFF39
:102D30009748242210380FA917F3A2EF18B010BD3E
:102D400010B54078FFF7C7FF03F09EF9002010BDD3
:102D50008E4800B5016889B02422684603F0F8F86F
:102D60006B4619780120002902D01979002904D076
:102D70006B465978002900D1002009B000BD834876
:102D800008B501680122491C684603F0E1F86B466A
:102D9000187808BD7D4808B501680122C91C68463D
:102DA00003F0D6F86B46187808BD784808B5016876
:102DB00001220F31684603F0CBF86B46187808BD46
:102DC000724808B5016801221F31684603F0C0F857
:102DD0006B46187808BD6D4808B5016801220B31B3
:102DE000684603F0B5F86B46187808BD674808B523
:102DF000016801220C31684603F0AAF86B46187886
:102E000008BD1CB50122614C01A821680E3103F0F8
:102E10009FF8216801221931684603F099F86B4642
:102E200019780020002903D01A798A4200D10120A4
:102E30001CBD564808B5016801220A31684603F0F6
:102E400087F86B4619780120002900D0002008BDC2
:102E5000002008B500904D480122016868460831FD
:102E600003F076F86B4619780120072900D300207B
:102E700008BD464808B5016801220D31684603F0D7
:102E800067F86B46187808BD404808B5016801220C
:102E90001831684603F05CF86B46187808BD3B486B
:102EA00008B5016801221A31684603F051F86B46F3
:102EB000187808BDF8B505000E00344C01222168D1
:102EC0006846891D03F044F86B461878324B01229E
:102ED0005843286021686846C91D03F039F86B46DD
:102EE00018782D4B58433060F8BD284808B5016864
:102EF00004221031684603F02BF8009808BD2348DF
:102F000008B5016804221431684603F021F80098DE
:102F100008BD1E4808B5016801221D31684603F04E
:102F200017F86B46187808BD184808B501680122E3
:102F30001E31684603F00CF86B46187808BD01B5E1
:102F4000124801224068694603F002F808BD01B545
:102F50000E48012240686946801C02F0F9FF08BD56
:102F600001B50A48042240686946001D02F0F0FFDE
:102F70000220FFF783FE08BD10B5040022F070FDAB
:102F8000002802D12000FFF7EBFF10BD083C040031
:102F9000D04604007CC70004710200007CB5040028
:102FA0000D00160002203DF013FA00280FD0FF217B
:102FB000CB316B461980042159801C715D71002151
:102FC0009E71D971082376216A460FF03BF97CBDCA
:102FD00070B50025FFF793FF012801D2012400E01E
:102FE0000024FFF782FF012801D2012000E0002029
:102FF000002C0AD0002808D0FFF7EDFE002804D1ED
:10300000FFF7C8FE002800D10125280070BDF9484F
:1030100040687047603010B517F30AEF80780107F9
:10302000890F022908D10009042805D00C2803D0F3
:10303000F149086A401C086210BDEF49886AC96AF4
:10304000704710B507F096FD002809D038F090FBC6
:10305000E84A117C002901D0491E117438F08CFB1C
:1030600010BDE44870B5683803F334FEE1483C38DD
:1030700003F330FEDF481838007C062813D0022006
:103080003DF0A6F907E020001BF090F8E279A17965
:1030900020001DF0CAF80400F5D13DF099F9002890
:1030A00001D01BF083F8012002F017F800200CF08B
:1030B000EBFCD248C168012292051143252F7BA069
:1030C00001000000D02F00000004000039D48BA9BB
:1030D000C160C16852001143C160CE49086902262F
:1030E000B0430861C84C0025A561CB4825746061D8
:1030F00007F063FD6561667470BDF8B504000E00ED
:103100000BF3EDFF009030060D00000E0DF0F1FC0A
:1031100061680127897800230A07920FFF03022ABA
:103120000ED10E09042E0BD18602B748009AC03882
:10313000006A0021C08880186941801B99410EE017
:10314000012A11D109090E290ED1009A80021E0010
:10315000101A2B00B341642219008018714161617B
:103160002061608838436080F8BDFEB50C00C969F5
:10317000C90408D5210020314A7A097A55066D0E16
:103180008E07B60F1BE00022130069460CC1110028
:10319000E56A0BE0CB005B191E685B6801931B03BB
:1031A0001B0F9A18491C0E29009602D2637893428D
:1031B000F0D2009949044D0E00998E07B60F89068A
:1031C0008F0FE1690A04120C29000DF02BFC012E6F
:1031D000029003D10E352D062D0E0EE0022E0CD1DD
:1031E00068060A23400F584329075F43090F401818
:1031F000390040181F3005062D0E60680123028833
:10320000E0690104090C28000BF352FD02994018F3
:103210008249096B08186087FEBDF8B502203DF0B1
:10322000E1F80500FF217E4800222D3118F350FA05
:1032300006007ED00221C020317334183081A0787E
:10324000F32280088000104008300007000F403053
:10325000A070E0784008400008431040CF210840AB
:10326000BF210840E070F1208000291806220D00DF
:10327000A01D17F3A6EC2000062229000C3017F33E
:103280000AED200006222900123017F39AEC0020E4
:1032900020801C20351830818421280017F32CED64
:1032A0002F00162060372C67787757481838009021
:1032B000007C00284AD054487838C088A080FFF7A6
:1032C00094FD002808D1FFF76FFD002804D1A088E5
:1032D0007D2149014018A0804B4878388089A8702A
:1032E00002203DF07FF870614E480079800607D4D7
:1032F000A878002804D0A868012189070843A8609D
:10330000082015252D023877FFF74EFD01240028EF
:1033100004D0012000F018FE3C4844602900300031
:103320000EF028F80098007C002806D13949086979
:1033300000E011E0022210430861334801001C3113
:1033400084614868401C48600120F8BD2E48C038A0
:10335000016A0988A180C1E72B491C318868401C9B
:1033600088600020F8BD294970B500248A6982422E
:1033700021D1254D183D287C06281CD000208861CD
:1033800021488069002803D1FFF747FF04000AE0C5
:10339000254801694069814205D024480722006818
:1033A000012139F008FB287C002804D0002C03D12F
:1033B0002C2019F091F970BD0128FCD1022028744D
:1033C000FFF76CFD00281A4806D03C30040003F3D8
:1033D0008BFC00220C2105E01030040003F384FC78
:1033E00000220521200003F331FC200003F31EFC22
:1033F00070BD10B5054CE169814204D12F2019F050
:103400006BF90020E06110BDA8470400103C0400E7
:1034100000900090C0A20080FFFFFF7F40A60080C8
:10342000C01900042CE9000400A000801408000466
:1034300030470400F8B500240600F94802218461F1
:1034400041740BF34CFEF74DE962A862FFF7ACFC48
:103450006968084303D0002000F076FD6C60002E00
:1034600004D0EF491C310868401C0860EC4C183C43
:10347000207C022808D1012001F039FEFFF70EFD63
:103480000326002801D02674F8BDE86906F31DFC68
:10349000E34DE44B0822783D0092EA88E24800219F
:1034A0001C3302F0CDFC2674FFF79CFD002807D0EA
:1034B0000BF315FE2A00383251631063E888A880A8
:1034C000D748683803F310FCF8BDD549203FF718FA
:1034D00001000000CC330000000400008611AE1A89
:1034E0001C314869401C48610120ADE7D14910B545
:1034F0001C314869401C4861322019F0F7F88CE70C
:10350000F8B5CC4C183C207C06282ED0C9488069E0
:10351000002818D10BF3EDFD05000E00200021005E
:1035200060382839C78880880A6B4B6B0021801867
:1035300059410023C0195941401BB14100280DDDFC
:1035400000F017FD0AE0BE4801694069814205D0DC
:10355000BC4807220068012139F037FA207C002896
:1035600003D0032801D105202074F8BDF8B50BF372
:10357000C0FD07000C0038F00FF9AE4DAE490090C9
:10358000287C496A08432BD128001838007C002683
:1035900000280AD0062808D02800783831002A00F0
:1035A000403A536B8088126B0CE007F0A7FA0028B2
:1035B00001D168690BE09F4AC03A106AD3698088DC
:1035C0009269310080185941C01BA14168610028EF
:1035D00006DD0EF0B5F8002802D0287C401C2874C7
:1035E000009838F0DDF8F8BDF8B50BF382FD914A8C
:1035F000403A516310639048806906F370FB8D4C2C
:103600000226183C207C2500603D00281FD0FFF7D3
:10361000F6FB002819D0FFF79BFC8B4F002801D048
:10362000667407E0FFF789FC002801D0032000E062
:1036300001206074EF80FFF746FC7D21C900414303
:103640007D200001081AA88001E0002060747A4BF8
:1036500008220092AA887D480021183302F0FAFB64
:1036600001202074744C7A4FE06801280DD138F0A5
:1036700093F80021E1607969302291437961754ABC
:10368000516AB143516238F08BF86A49A8884861A1
:103690003869B0433861FFF769FFF8BDF8B50BF33F
:1036A00028FD644A403A516310636348806906F319
:1036B00016FB604C0026183C207C2500603D00284D
:1036C00033D0FFF79CFB644F00287DD0FFF740FC10
:1036D00000282BD002206074FFF7DFFB002816D0F3
:1036E000FFF7BBFB002812D1E8887D2109014018B3
:1036F0000004000CB842E88001D9EF8004E07D218D
:10370000C901884200D2E980E88854492DE0E88860
:103710007D21C8380004000CC9018842E88000D22D
:10372000E980E9884D482DE0A880C5E0FFF705FC59
:10373000002829D003206074FFF7AFFB002816D0C3
:10374000FFF78BFB002812D1E8887D214901401842
:103750000004000CB842E88001D9EF8003E0404942
:10376000884200D2E980E8883E49081ADCE7E88808
:103770003B49C8380004000C8842E88000D2E98048
:10378000E9883848401ACFE701206074FFF785FBCD
:1037900000281AD0FFF761FB002816D1E8883249CB
:1037A000FF30F5300004000C8842E88000D9E98041
:1037B000A8887D21FF38F5380004000C49018842B3
:1037C000A88079D2A98077E012E0E8887D2164386A
:1037D0000004000C49018842E88000D2E980A888F2
:1037E000224964300004000C8842A880EAD863E0D3
:1037F000FFF7E4FA002804D01D486674E880AF8023
:103800005AE00D48016A002901D0066205E0194915
:10381000002082008A58002A01D0012703E0401CC2
:103820000828F6D33700FFF7E7FB002F009023D0DE
:103830000E4823E0A8470400103C0400F3320000C7
:1038400000A0008014080004FF7F00006732000021
:10385000C0A20080C0A80080204E0000307500008B
:10386000E02E0000606D0000D859000050460000B6
:103870004E700000F40003C07D204001A880FFF7D7
:103880000CFB002803D0FFF7E8FA00280AD0FFF766
:10389000F3FA002801D0002F04D00098002F03D0A5
:1038A000002803D1F94805E0002801D1F84801E0DB
:1038B0007D204001E880667408220092AA88F548BD
:1038C000F54B002102F0C6FA01202074F24CF34FB0
:1038D000183CE06801280DD137F05EFFDDD94D7B43
:1038E00001000000C837000000040000D5CB7D7641
:1038F000E6607969302291437961EE4A516A022388
:103900009943516237F056FFEB49A88848613969FD
:10391000022081433961FFF733FEF8BD10B5FFF790
:10392000D1FA002802D0FFF769FE80E5012001F0FE
:1039300080FBE1491C31002805D0C868401CC860E4
:10394000FFF7B6FE73E50869401C0861DA480421F8
:10395000183801746BE5FEB5050002203CF056FDF9
:103960000090D548406800284AD037F01FFFD24C5D
:103970000126183C0190207CB602002D37D000288B
:103980003BD1200060380068002836D007F0C0F82E
:10399000002832D1FFF7FAF9002803D1FFF718FA0F
:1039A00000282AD0FFF74BFA002803D0FFF710FABF
:1039B000002822D03FF050EB207C06280AD0BF48D8
:1039C0000178002906D101215022017000981300CE
:1039D00006F052F8FFF776FA002805D0300000F024
:1039E0002DFB300000F01DFBFFF798FF05E00028DD
:1039F00003D00025062804D12574019837F0DAFE9B
:103A0000FEBDAA4F183FF86906F373F9B86906F3CB
:103A100070F9FFF744FB300000F010FB300000F0BD
:103A200008FB207C0628E7D0A44801780029E3D0D1
:103A30002822057000982900130006F01DF8DBE726
:103A40001CB5002001900090694601A8FFF750FACC
:103A500099480199C03802688A4203D18288009B44
:103A60009A4226D00160009A82809349C3889C398B
:103A70009A180A80019B9A1A4389D21A4A80C388ED
:103A8000D218643A8A80C2884389D21ACA800289CD
:103A9000009B0831D2180A80019B9A1A4389D21AD6
:103AA0004A800389D218643A8A8002894089101AB0
:103AB000C8801CBD804870B5406800282ED037F003
:103AC00075FE040007F024F8002824D00020FFF73A
:103AD00042FF3FF0C2EAFFF7B3FF7948C168012215
:103AE00052051143C16073498039886AFF229204EC
:103AF000104388624D0D280000F0A0FA280000F065
:103B000090FA6D481838007C062804D0082200215D
:103B10000120FFF761FA200037F04CFE70BD6648C7
:103B200070B5406800283AD037F040FE5F4C060080
:103B3000183CA06906F3DDF80025A561A06806F32E
:103B4000D8F85B48A56041693022914341615949E9
:103B5000486A02229043486256488038816AFF22B0
:103B6000920491438162440D200000F067FA200026
:103B700000F05FFA5048C0384561FFF790FA4E48B0
:103B80001838007C062804D0002211001000FFF72E
:103B900023FA300037F00EFE0120FFF7DCFE70BD87
:103BA000424918398A6882420DD10020886001207C
:103BB000C8603F4841693022114341613D49486A2C
:103BC0000222104348627047F8B507003A4840683F
:103BD000002858D0384878380068002853D037F08B
:103BE000E5FD354C0126183C0090354D207C7605CE
:103BF000002F1CD0002808D106202074FFF7DDF824
:103C000000283DD0FFF78BFF3AE0062838D0274F39
:103C1000183FF86906F36DF8B86906F36AF80620EC
:103C20002074E868B043E860FFF739FA28E0062816
:103C300026D1FFF7C2F800280FD1FFF7A7F8002818
:103C400003D1FFF7C5F8002807D0FFF7F8F80028E0
:103C50000FD0FFF7BDF800280BD1207C06280FD12C
:103C60000020207406F054FF002809D0FFF722FF3F
:103C700006E0E8683043E8603FF0EEE9FFF74EFE0B
:103C8000009837F097FDF8BD084910B518394A6912
:103C9000824203D10020486100F06AF939E4000053
:103CA000D85900001027000067320000283C0400AB
:103CB000C0A20080C0A80080A8470400603C0400A7
:103CC0000090009038B5C94C2169814216D100207E
:103CD0002061C748007C032801D004280ED10120B0
:103CE00000F046F9606906F304F8C04B5E1526EB58
:103CF00001000000C43B00000004000021A408C231
:103D0000082200926288C0480021143302F0B6F8FD
:103D100038BDF8B5BD48446B00250BF3FEF9B84E2D
:103D2000001969417163306306F0FCFE002811D070
:103D3000B448A838406900280CD0B06805F3E3FF08
:103D40000822009219223300B148520100210833A1
:103D500002F094F8AB48007C002825D0062823D038
:103D6000012822D10BF3D9F90C00A64928390A6B96
:103D70004B6B2100821A99410B00A249A54C603976
:103D800088882900801A994100040014A0420BDAA7
:103D9000B06905F3B8FF9A4B082200929E482200B2
:103DA0000021183302F06AF8F8BD306905F3ABFF63
:103DB000082200923088924B221A00219748103333
:103DC000F0E7F8B5263801258E4A8D4E117CAD02FC
:103DD0000224030017F32EE914A30D0D390B0E7EF8
:103DE0001113361729300D0DA8A8AAAAAA0DFFF79E
:103DF0006BFEF8BDFFF79DFEF8BD012000E000203E
:103E0000FFF7B3FDF8BD8648062904D0C16801223A
:103E100052051143C160C1682143C160280000F010
:103E200017F9280000F007F9F8BD280000F010F994
:103E3000280000F008F9F8BD7248243802F372FF38
:103E4000FFF772FBFFF774FDF8BD6E4FA83F388A8D
:103E5000002807D138002C303862F8893882FFF703
:103E6000F9FD04E067498439401E39623882012037
:103E70007861280000F0DFF80BF34FF9F961B861C1
:103E8000B06905F340FF08220092386A5C4B428813
:103E900061480021183301F0F1FFF068614D0128FD
:103EA0000DD137F08DFC0021F1606969302291431A
:103EB00069615D4A516AA143516237F085FC386AF5
:103EC00081885048183041612869A0432861FFF774
:103ED00061FBF8BD4B4B1833587C002813D0401EB3
:103EE000FF24F53458745C61FFF754FBB06905F3A7
:103EF0000AFF434B08220092474822000021183352
:103F000001F0BCFFF8BD0129FCD13E4914743431E5
:103F10008869401C88610120FFF7AAFAF8BD0429CE
:103F2000FCD1FFF7CFFBF8BD012000E00020FFF738
:103F300055FEF8BD10B505F04BFF324C1834A068A3
:103F4000002812D0E06800280FD006F041FE0128BA
:103F50000BD129F0F4FA022807D0012060602D204F
:103F600018F0D8FB2A2018F0D5FBE8E42B2010B578
:103F7000FFF727FF2E20FFF724FF224900201831EA
:103F80004860DCE40322264912050028086901D0B4
:103F9000104300E0904308617047F8B502203CF000
:103FA0003FFA07000E216A460FF0A9FC050024D055
:103FB00000981E4E046F00202071607120706070A8
:103FC000FF220621A01D37F052E8F12080003918A9
:103FD000200006220C3016F312EE02203CF020FAEC
:103FE00068610098082160300177310028000DF0E9
:103FF000DFF9002801D00120F8BD0020F8BD000045
:10400000103C040090470400613B000000A60080C3
:10401000793A000034080000673200009D3B000040
:1040200000900090C0A20080C0A800800211000093
:104030000948006A704708494A6902434A61CA69E7
:104040000243CA617047044A516981435161704714
:104050000149C04308627047802200804B490A68CA
:1040600002430A608A6802438A6001207047474918
:104070000A6882430A608A6882438A600120704726
:10408000424940310868086070474049C043C860F1
:10409000012070473D4B80339969DA6909011209A3
:1040A00009091201002804D00520400701430A2015
:1040B00003E005200007014305200243D961DA61CE
:1040C00070473348016B022291430163016B402228
:1040D00091430163016B04229143016370472C48B3
:1040E000016B062291430163016BC02211430163FE
:1040F00070472748016B80229143016309541EAD2C
:1041000001000000C03F000000040000727EDBAE32
:10411000016B462211430163016B3822914318223F
:104120001143016370471F48006B810701D50020D0
:104130007047400601D5022070470120704710B536
:1041400001F039FA002804D0174988690122104388
:10415000886110BD10B501F02EFA002804D0124875
:10416000816949084900816110BD10B501F023FA49
:10417000002804D00C48806901210904084010BDC2
:1041800010B501F018FA002803D007488069C0076D
:10419000C00F10BD0348C168C2051143C16070471C
:1041A0008022008000210080C02A00807047704774
:1041B000FF484068816B090C01D000207047816B7B
:1041C000090504D5816B0904090FFBD100E0806B60
:1041D00001207047F64949688A69120C12040243AB
:1041E0008A617047F2484068816BC907FCD041681A
:1041F0000122D203914341607047ED4949680A6B3F
:10420000086348680122D203104348607047E848B9
:104210004068406A7047E649496880314A6A00014F
:10422000120F1207000902434A627047E0484068D3
:10423000C06A7047DE494968CA698243CA617047EB
:10424000DB494968CA690243CA617047D84949686D
:104250000A6D02430A657047D54949680A6A0243F4
:104260000A627047D24949680A6A82430A62704703
:10427000CF484068C0300168490849000160704774
:10428000CB48406880308188490849008180704768
:10429000C74840688030818801221143818070477F
:1042A00070B5C34D68688030016801221143016018
:1042B0000168C04C490205D50168A14301600A208C
:1042C0003EF00AEE6868803001682143016070BDED
:1042D000B74840688030016849084900016070476C
:1042E000B348406880300068C007C00F7047B048CE
:1042F000406880300168AF4A914301607047AC4824
:104300004068803001680122120611430160704745
:10431000A74840688030016801221206914301607D
:104320007047A34840688030C068704770B505008A
:1043300016003EF0AAEE9E4C6068010080300269D3
:104340000561426943618269F0228261C269C66186
:104350008A68102002438A608A6820239A438A6010
:104360006068416B426B8A42FCD0FFF7DAFF00289D
:10437000F6D1606881681943816041680122520367
:104380001143416070BD8A484068803000697047C1
:1043900087484068816820221143816070478448C3
:1043A0004068816820229143816070478049496854
:1043B0008031CA8801238340C8881A43CA80704765
:1043C0007B48406881680122D204114381607047B4
:1043D00070477748406880300168FF22521C1143C3
:1043E0000160704772484168092080010818C1695E
:1043F000012292031143C161C16952001143C1619D
:10440000C16952001143C161704769484168092080
:1044100080010818C169012292031143C161C16979
:1044200052001143C161C16952009143C16170479B
:104430005F484068816810221143816070475C4882
:104440004168092080010818C16901225204114302
:10445000C161C169D2001143C1617047544905224D
:104460004968D2018918CA69382340079A43800EE7
:104470000243CA61C86901221043C86170474C4AAF
:104480000023D3561F21C0181F2800DA0100080698
:10449000000E70470D2804D8454900228A56002A8C
:1044A00000DBECE77047F0B593B0434C206803099C
:1044B00060681B010109A06809010209E068120196
:1044C00000090001C01C12902069491C050960699F
:1044D0002D0100090001401D1190A069921C0009E6
:1044E0000001801D1090E0692D1D0609206A36012B
:1044F0000009000108300F90606AF61D00090001F4
:1045000009300E90A06A000900010A304757505444
:1045100001000000BC43000000040000708703B8E5
:104520000D90E06A000900010B300C90206B00092F
:1045300000010C300B90606B0709A06B3F01000974
:1045400000010D300A90E06B0D37000900010D30BD
:104550008646F020814310310991129985434035F8
:104560000895119D8243854350350795109D203253
:104570008543503506950F9D9446854350350595E6
:104580000E9D0C9A8543503504950D9D82438543BD
:10459000503503950B9D50328543503501950A9D4A
:1045A000029281438643874385437246824330317A
:1045B000503650375035834350321F20000283431A
:1045C000964605E000010004000040003C2D000478
:1045D000009513252D025B192360099B81438343BA
:1045E0005B196360634683435B194919A360E1600B
:1045F000089D0B21854349026A182261079D864365
:1046000085436A186261069D874385436918A161E5
:104610000321C9027218E261059D85436A1822626E
:10462000049D85436A186262039D85436A18A262ED
:10463000029A82435218E262019D85436A182263FE
:104640007A186263009D85436A18A26372468243AA
:10465000511800250700E163AE00A059C004C00E48
:10466000FFF717FFA159C006C00CB9436D1C0143E9
:104670002D062D0E102DA151EED313B0F0BDF0B5C7
:1046800088B0FF490A6A1206130F4A6A1206120F0F
:10469000120113438A6A1206120F12021343CA6AE6
:1046A0001206120F120313430A6B1206120F1204A2
:1046B00013434A6B1206120F120513438A6BC96B20
:1046C0001206120F09061206090F134309070B43BE
:1046D000EC494A68D11DFF31FA310C690B610C6B52
:1046E0000B630924A4011219D468D360E44BDC687D
:1046F0002406260F04969C6835012406240F039493
:104700002C431D692D062E0F350237032C430597C8
:1047100000962600A6465C693E432406240F0194B9
:10472000240426430694019C27059C693E432406E5
:10473000240F2506DC692E432406240F2407264374
:10474000029607965B68BC461B061F0F039B1E0163
:104750003B003343049E059F36023343009E3B4398
:1047600036041E4367463E432E432643072803D0A4
:10477000062801D00A2809D1906802989060C8687C
:104780000798C860C86ACE6208B0F0BD0528FBD1A2
:104790009068019E704636033043069E304366465D
:1047A0003043284320439060CA68C860C86A0698AE
:1047B0000343604603432B432343CB62E4E7F0B556
:1047C000AF480168426809071207090F120E11432A
:1047D0008268036B1207120D1143C2681207120C94
:1047E000114302691207120B114342691207120AA0
:1047F00011438269120712091143C26994461207D4
:1048000011439646026A1407426A240F1207120ED9
:104810001443826A1207120D1443C26A1207120C63
:1048200014431A07120F15042C43456B26002D075D
:104830002D0A2E43856BC06B2D072D092E430007D3
:10484000064390484568E81DFF30FA3047684160EC
:104850008768866016053443120614431A0714430A
:1048600009229201AA1813681160536854606246C5
:104870001207120F1301134314022343140323439B
:1048800014042343140523431206134372461343AF
:10489000426A4162816A8362F0BDF0B57849086876
:1048A0004A69C004C50E4868D204C004C00E400165
:1048B00005438868D20EC004C00E80020543C86854
:1048C0005206C004C00EC00305430869CB69C0048A
:1048D000C00E0405254315438A69DB04D204DB0EB0
:1048E000D20E5B011A430B6AAC46DB04DB0E9B0263
:1048F0001A434B6A4D6BDB04DB0EDB031A438B6AF6
:10490000ED04DB04DB0E1B051A43CB6AED0EDB0462
:10491000DB0E5B061A430B6B6D01DB0494DD3B7809
:1049200001000000B847000000040000235DD0D45F
:10493000DB0E2B438D6BC96BED04ED0EAD022B43EB
:10494000C904C90E470106003E4387023E43C70320
:104950003E4326434006064348010C0004438802B8
:1049600004434D48CD0340682B430100FF302C43E6
:10497000FF30801C45696546456187698261C7696A
:10498000C361436B33004663866B8363C66BC3634B
:1049900008000921890140180169056141694261E6
:1049A00081698461F0BD10B50400FFF712FF20009B
:1049B000FFF76FFEFFF77BFF10BD37494968FF31F6
:1049C000FF31891C0A68000712091201000F024317
:1049D0000A60704730B504002F4D04280CD2112016
:1049E000FFF76CFD6968092292018918C969890479
:1049F000C90E884200D204246868FF30FF30801C52
:104A000001680F22120291432207120D1143016027
:104A100030BD214A10B553680522D2019A18136996
:104A20001F246406C006A343800803431361106972
:104A30006311C9069843C9090843106110BD164A9D
:104A400010B553680522D2019A1813691F24E40394
:104A5000C006A343000B0343136110696311C90629
:104A60009843490C0843106110BD0B4A10B55268B9
:104A70000523DB01D21813691F246401C006A34378
:104A8000800D034313611069C90640094001C90E36
:104A9000084303E03C2D000400010004106110BD38
:104AA000F84A10B552680523DB01D21853691F2458
:104AB0006401C006A343800D034353615069C906D6
:104AC00040094001C90E0843506110BD0C2010B5CB
:104AD000FFF7E9FC04001120FFF7E5FC2100FFF7D8
:104AE000DFFF1220FFF7DFFC04001320FFF7DBFCE1
:104AF0002100FFF78EFF1420FFF7D5FC04001620DD
:104B0000FFF7D1FC2100FFF79AFF1720FFF7CBFC3E
:104B100004001920FFF7C7FC2100FFF7A6FF10BD16
:104B2000D84905224968D20189180A699205D20E2E
:104B3000824206D30A69D206D20E824201D80820E8
:104B400070470A691203D20E824206D30A695204E0
:104B5000D20E824201D8042070470A699200D20E18
:104B6000824206D30A69D201D20E824201D80220C3
:104B700070474A699205D20E824206D34969C90636
:104B8000C90E814201D80120704700207047BD49FD
:104B900049688031CA6AFF23E13300079A43C00D98
:104BA0000243CA627047B74900B549688031CA6A92
:104BB000C30652095201DB0E1A43CA62FFF7B0FF67
:104BC0000006000EFFF7E3FF00BDAE494968C031A3
:104BD0004A69FF23E13300079A43C00D02434A614B
:104BE0007047A84900B54968C0314A69C3065209EF
:104BF0005201DB0E1A434A61FFF792FF0006000ED6
:104C0000FFF7E3FF00BD9F494968FF3141314A6B1F
:104C1000FF23E13300079A43C00D02434A63704704
:104C2000984900B54968FF3141314A6BC3065209C2
:104C30005201DB0E1A434A63FFF772FF0006000EB3
:104C4000FFF7E1FF00BD8F494968FF31491C4A6900
:104C5000FF23E13300079A43C00D02434A617047C6
:104C6000884900B54968FF31491C4A69C3065209A1
:104C70005201DB0E1A434A61FFF752FF0006000E95
:104C8000FFF7E1FF00BD7F494968FF31FF31891C13
:104C90000A6A0F235B0600079A43C00802430A62B0
:104CA0007047784900B54968FF31FF31891C0A6AAD
:104CB0001F231B059A43C306DB091A430A62FFF749
:104CC0002FFF0006000EFFF7DEFF00BD70B50500E8
:104CD0000D20FFF7F3FB6B494E680921890171181C
:104CE000CA699204D20E904201D2012200E0002251
:104CF00064480024401C035DAB4204D0641C2406BD
:104D0000240E022CF7D3086A182555435D4A000C7F
:104D100000040832535B18430862486A000C000420
:104D2000AA18538818434862886A938885B5D5A81D
:104D300001000000B44B000000040000D732A56061
:104D4000000C000418438862C86AD388000C000471
:104D50001843C862086B1389000C000418430863E9
:104D6000486B5389000C000418434863886B93898F
:104D7000000C000418438863C86BD389000C00043E
:104D80001843C8630520C00130180368168A1B0C3D
:104D90001B04334303604368568A1B0C1B043343D4
:104DA00043608368968A1B0C1B0433438360C3688B
:104DB000D28A1B0C1B041343C3603023364A63435F
:104DC00038329A18535B0C6A1B042404240C2343C6
:104DD0000B62521953884C6A1B042404240C23438D
:104DE0004B6293888C6A1B042404240C23438B623B
:104DF000D388CC6A1B042404240C2343CB6213897C
:104E00000C6B1B042404240C23430B6353894C6B4D
:104E10001B042404240C23434B6393898C6B1B04D5
:104E20002404240C23438B63D389CC6B1B042404FC
:104E3000240C2343CB63118A036809041B041B0C55
:104E400019430160518A436809041B041B0C194370
:104E50004160918A836809041B041B0C194381601B
:104E6000D18AC26809041204120C1143C16070BDDA
:104E700009494A68092189015118CA691F235B023F
:104E8000C0069A43800C0243CA61C8690122920499
:104E90009043C86170470000000100044E49496812
:104EA000C0314A690F239B0300079A43800B0243DA
:104EB0004A61EFE7484900B54968C0314A691F2394
:104EC0005B029A43C3069B0C1A434A61FFF732FE0A
:104ED0000006000EFFF7E2FF00BD3F494A680921C6
:104EE00089015118CA69FF23E13300079A43C00DB5
:104EF0000243CA61CEE7384900B54A6809218901F1
:104F00005118CA69C30652095201DB0E1A43CA611D
:104F1000FFF710FE0006000EFFF7DFFF00BD10B523
:104F200004000D20FFF7D4FAFFF7A2FF1620FFF7C9
:104F3000C4FAFFF7C0FEE00614D50120C007C07C0C
:104F4000C1070FD00007400F02282AD0032809D13B
:104F50001620FFF7BDFAFFF78BFF1620FFF7ADFA1B
:104F6000FFF7A9FE1620FFF7A8FAFFF7C4FF1620E7
:104F7000FFF7A3FAFFF79EFF1820FFF79EFAFFF74F
:104F80001CFE1620FFF799FAFFF735FE1620FFF7F3
:104F900094FAFFF74FFE1620FFF78FFAFFF76AFE2D
:104FA00010BD1120FFF794FAFFF762FFDAE70B4814
:104FB00080690007000F6DE7084881680122120729
:104FC000914381608168C20591438160816852107C
:104FD000914381605EE7000000010004802A0080A8
:104FE00070B504F0D5F8764D0226002818D000F0F0
:104FF000E0F8002814D004F3CDFA724C226A636AF8
:10500000801A9941E162A062E868B043E860A06854
:10501000002802D00020A062E06206F000F870BD17
:1050200005F039FD002803D105F005FD0028F6D074
:1050300000F0BFF80028F2D0E868B043E86070BD27
:1050400010B5604CA16981420ED1FFF7C9FF6069BC
:105050004004400CFFF71FF860694004400CFFF764
:105060001FF80020A061606110BD042010B5FFF79B
:1050700012F80420FFF714F8524CA069002804D05D
:1050800004F369FE0020A061606110BD4C48C06857
:1050900002210840704738B5052840D2494D484C98
:1050A0002969803400290BD004F374FA69622862FC
:1050B00002E0052000F092F8E06A4000F9D530E007
:1050C00001218140E8680143E960FFF7DFFF002824
:1050D00001D1012038BDE06A400022D400F069F817
:1050E00000281CD10420FEF7DBFF0420FEF7CBFFD5
:1050F0002C68FDF7DCFF002800D06C68686904218B
:10510000084368612F4B082200922F48220000219B
:10511000183300F0DBFE04F33DFA696228620020D8
:1051200038BD2748C16802229143C160D1E70528F4
:1051300010B501D3002010BD01218140E28C9C31CB
:1051400001000000B04F00000004000084E8760C6D
:105150002148C2681143C160FFF7A2FF002814D0A4
:1051600000F031F800280BD0FFF789FFFDF7A9FF09
:10517000002805D01A48007C042801D105F059FF09
:105180001449C86802229043C860012010BD052858
:1051900010B516D2104C0123E16883400A009943F0
:1051A000E1600ED1002A0CD000F00DF8002801D0EB
:1051B000FFF765FF0749C86802221043C860012055
:1051C00010BD002010BD04488069002800D00120D7
:1051D0007047000000900090C8010004B54E000028
:1051E00090470400F849086B802290430863704799
:1051F000F64910B5096836F006E88905800A0843C3
:1052000001D03DF092EE10BDF148016A0F2211432A
:1052100001620220ECE7EE48016A09090901016216
:105220000120E5E7EB4970B5086808229043086063
:10523000E94A506840084000506010690B2108435B
:105240001061E64908009369DB0601D4401EFAD2DA
:105250009069800601D4491EFAD236F0E3FAE0499B
:105260000A680124A406A2430A60DD4A803213685A
:10527000DC4D2B4013601368ED432B4313600A6829
:1052800022430A6036F0D2FA0120FFF7B1FFFFF7A0
:10529000BBFF20F051FC70BDD349FF22C432888B84
:1052A0001042FCD17047F8B5D04C6069002806D098
:1052B00036F0B8FACE48FAF7D5FF00F0AFFC36F07A
:1052C000B1FA60610021012020F09CFB002810D081
:1052D000C54EB488012080020440B088C24D3527F5
:1052E000A0433F012035B84204D1287D0121084365
:1052F0002875F8BD022000F042FB0028F9D03C439D
:10530000B480297D012001432975F8BDB74810B547
:10531000446900214161FF210170B3482030017DC3
:10532000490849000175012020F08EFB200036F06D
:105330007DFA10BD70B5FEF2FAE9AC4D0400287894
:10534000022813D1A869401CA861200605D4A848EA
:105350002030FAF787FF00F061FC802C02D1FEF2CA
:10536000E6E970BD2000FEF2ECE970BD6869002836
:1053700005D09F481630FAF775FF00F04FFC00216A
:10538000012020F03FFB0028EFD002206C61287044
:105390000120A861974800680028E6D1924DAC88AA
:1053A000012080020440A8886B26A043F600B0428A
:1053B000DBD0022000F0E3FA0028D6D03443AC80E2
:1053C00070BD8A4910B58869401E88610FD14C694B
:1053D0004861FF200870012020F036FB802C02D1AC
:1053E000FEF2A4E910BD2000FEF2AAE910BD0028DB
:1053F000FCDAFEF29CE97E481730FAF733FF00F042
:105400000DFC10BD70B5794E7069002807D036F0DC
:1054100009FA7748001FFAF725FF00F0FFFB36F086
:1054200001FA70610021012020F0ECFA002814D06C
:105430006D4DAC88012080020440A888A0438228DA
:105440000BD02888F080002000F099FA002804D0C2
:10545000A888308182200443AC8070BD634810B5B9
:105460006149028944698A80C2880A8000214161B9
:10547000FF210170012020F0E7FA200036F0D6F974
:1054800010BD70B5594D6869002807D036F0CAF9CB
:105490005748C01EFAF7E6FE00F0C0FB36F0C2F92E
:1054A00068610021012020F0ADFA00281BD04E4E8B
:1054B000B488012080020440B088A043022812D0A2
:1054C000FEF759FE002803D0012803D13F2002E057
:1054D0001A2000E07F203188E9803080B088288160
:1054E00002200443B48070BD404810B53E49028993
:1054F00044698A80C2880A8000214161FF210170CD
:10550000012020F0A1FA200036F090F910BD30B54E
:1055100005000C00FFF7C0FE334B20331D81FFF761
:10552000BBFE9C80FFF7B8FE30BD10B50400FFF74E
:10553000B3FE2D4B20331C81FFF7AEFE187910BD52
:1055400030B504000D00FFF7F0FF284351E49E82C0
:1055500001000000AC530000000400003B2D53BFCD
:1055600001002000FFF7DDFF30BD30B504000D0065
:10557000FFF7E5FFA84301002000FFF7D2FF30BD91
:105580001F484178002909D12049096801220902F0
:105590004270090F02002432515C8170807870479C
:1055A000174910B5C878002815D108611748406818
:1055B0000A008007800F103210230124002807D032
:1055C000012803D0022803D0032803D1136001E08F
:1055D00030201060CC70086910BD0000400C0090B5
:1055E000E0B801C080A1008000A3008040A6008038
:1055F0008813000000210080FF7FFFEF000800906B
:10560000F801000437000100EC07000400200080CE
:10561000E54800880006000E704700B5FFF7F8FF68
:10562000022806D1E048803840688007800F0128B2
:1056300000D0002000BDDD4B596838229143104056
:10564000084358607047D94B59680F229201914323
:10565000104008435860704710B50C00FFF7F3FF87
:105660002000FFF7E8FFB7E7D14810B544690021F3
:105670004161FF210170012020F0F0F9200036F097
:10568000DFF8A9E770B5CA4C6069002806D036F08B
:10569000D3F8C848FAF7F0FD00F0CAFA36F0CCF8B3
:1056A00060610021012020F0B7F9002811D0C24D1F
:1056B000AC88012080020440A888B526A0433601AA
:1056C000B04206D0022000F064F9002801D0344333
:1056D000AC8070BDB4480068B8498874010CB74804
:1056E00020380186B64949698163704710B50400C6
:1056F0000BF098F9002802D1200020F09BFD6BE709
:1057000070B50500AD480C0020384169A14212D0A7
:1057100044610021200020F0DBF90021200020F06E
:10572000E3F9002D07D10021200020F0D7F9002156
:10573000200020F0DFF970BDA0482038016A002069
:10574000DEE79E482038C1690020D9E79B48203811
:1057500081690020D4E799482038416881610020A0
:10576000CEE796482038816881610020C8E79348D9
:105770002038C16881610020C2E790482038016963
:1057800081610020BCE788488E4A8030016811435F
:105790000160704784498B4A8031086890430860F3
:1057A00070478948C16889008908C160C1680322BF
:1057B00092071143C160810C7C488030416183496C
:1057C000016183494161052101617047814800B54C
:1057D0000068002801D0FFF7E4FF7F480D21C16376
:1057E0002D21416300BD714980398868CA0C9043FE
:1057F000886047E76D4880388168C20C114381603A
:1058000032E7694880380068000701D501207047F9
:10581000002070476648C068704700207047F7B5A1
:1058200086B004000D0036F007F80090002101203A
:1058300020F0F2F800286FD0032160000A008240B7
:1058400005902000083840000E008640039020009C
:1058500010380492020047000800B840029020006F
:105860001838430008009840012186460800A040EF
:105870009C460B00019059489340584A4030002DF7
:1058800037D0082C04D21568049EB543156012E089
:10589000102C03D25568B54355600CE0182C04D287
:1058A000C569029EB543C56105E0202C03D2056A97
:1058B0007646B5430562089D002D14D0102C04D205
:1058C0009368019C2343936002E0426A1A43426258
:1058D00082680A438260404BC03358680122120636
:1058E0001043586044E03C48C030016804229143B2
:1058F00046E0082C07D21568059E049FB140BD43C1
:105900000D4315601BE0102C07D25568039FB5436B
:10591000B9400D43556012E033E0182C06D2C5693A
:10592000029EB940B5430D43C56108E0202C06D264
:10593000056A6646B1407746BD430D430562089946
:10594000002918D0102C04D29168019B99439160D2
:1059500002E0416A9943416281684908DDC717EE58
:1059600001000000A85700000004000068F780D381
:10597000490081601D48C0304168012212069143F0
:10598000416000211B48416005E01848C0300168B3
:10599000042211430160012020F06AF8009835F0DC
:1059A00059FF09B0F0BD10210A2803D20549400073
:1059B0003431095A05480180012070478020008059
:1059C00000290080F8010004370001000008009061
:1059D0009CC7000400A8008000044010002A00803A
:1059E000170000FF102000002C9301C080220080CF
:1059F00000020090E0B801C070B50024FFF717FE68
:105A0000002808D0FEF7F8FB002803D1FEF7E9FBD9
:105A1000002800D0012435F019FF0500002C07D123
:105A200002203DF065FD002802D01B4901200860DE
:105A3000002101201FF0FAFF280035F00BFF0020A5
:105A400070BDF8B5002015491FF076FA124E0024FB
:105A5000361D0F273F0308E02104090C39430020BD
:105A60001FF06AFA70598047641CA500705900281D
:105A7000F2D10B480C49026800920A4A0B480C4BC1
:105A800002F322FA19F096FF0A480168002901D0B2
:105A900000208847F8BD00002C9301C05F5F000024
:105AA00068070004C8DA0004881900047C1900049F
:105AB000803C04C038020004FEB50D001600089FAB
:105AC0000A9A0999002800D1FEE70468002C00D149
:105AD000FEE702920191320029002000009720F099
:105AE0002FFCFEBD10B500F3E3FF0006000E10BD55
:105AF00010B500F36FFF0006000E10BD002810B5B2
:105B000001D000F3A3FF10BD38B514006A4600F3BE
:105B1000FDFE00982070002038BD10B5040000F391
:105B20004FFE2060002010BD10B500F31FFF10BD18
:105B30007CB50D001600079A0699002800D1FEE7F3
:105B40000468002C00D1FEE7019200913200290088
:105B5000200020F0EEFC002800D165637CBD10B56C
:105B6000416B20F0FDFC10BD7CB50C001500069AC1
:105B7000002800D1FEE70068002800D1FEE70021E0
:105B8000019200912A00210020F008FC7CBD10B594
:105B900020F024FC10BD002810B500D1FEE70068FD
:105BA000002800D1FEE720F090FC10BD002810B5C1
:105BB00000D1FEE70068002800D1FEE720F09FFC3E
:105BC00010BD10B520F0A5FC10BD10B520F0A9FC4B
:105BD00010BD10B504003DF0E2E9002801D000201E
:105BE00010BDFDF2B8ED606000F3EAFD2200002177
:105BF00000F348FE0028F3D06068802802D1FDF24F
:105C0000AAED01E0FDF2B0ED012010BD38B50400B1
:105C10003DF0C4E9002801D0002038BD00F3D0FDDC
:105C200021686A4600F32EFE002808D160688028AB
:105C300002D1FDF290EDEFE7FDF296EDECE70120E9
:105C400038BD0000F8B59749486B0222904348637D
:105C50009548017801297ED00121017035F0F6FDCB
:105C600000909248422115F3ACE801218F4AC90700
:105C700000200B781354491C401C0A28F9DB8C497E
:105C800000200B781418491C401C0B28A372F8DB69
:105C90008748903801785175017991754179D175AE
:105CA000017A1176417A5176017B9176407B804969
:105CB000D076803900200B781418491C401C0A2823
:105CC0002377F8DB7A4950390A7E78482030827190
:105CD0000A7FC271497F0172754930390A78427270
:105CE0004A7882728A78C2720A7902734A79427358
:105CF0008A7982730A7AC2734A7A02748A7A4274FF
:105D00000A7B82744A7BC2748A7B0275CA7B4275A5
:105D10000A7C82754A7CC2758A7C0276C97C41768F
:105D2000634930310A7882764A78C2760A790277F6
:105D30004A7942775F4A137C8377927CC2770A7FE5
:105D400020300270497F4170594E08201036844639
:105D5000B078EE2800E041E0FAD16046F070FF2014
:105D6000B07000222FE0B078EE28FCD19B7EBCD52D
:105D700001000000A45B0000000400009C98F5678F
:105D80000C245443514B1959F170080A3071080C16
:105D90007071080EB071FF20B070002903D1B07887
:105DA000FE28FCD11BE0474FE51869681A37B07828
:105DB000EE28FCD1434813300B780370491C401C7B
:105DC000B842F9D9414B68681B59C018884210D8AD
:105DD000287AB070521C1206120E6245CDD300987C
:105DE00035F042FD34483A4941633448002101709E
:105DF000F8BDFF20B070DAE7324810B51030807877
:105E0000EE2804D13348FAF74BFAFFF725FF10BD0F
:105E1000F8B5FCF7F4FC304D284E274F2C6804E011
:105E20006068002800D080472468002CF8D1FFF774
:105E3000E3FF7078401C0006000E7070FAF730FA2D
:105E4000786BFF21491C08437863FCF7D7FCE5E732
:105E5000224810B500F3C8FD10BD10B5184C203C09
:105E60006360E260A16020603DF000E920613DF0E8
:105E70000EE960613DF01AE9A0613DF028E9E061BA
:105E80000D48416B022291434163FFF7E5FE10BDCF
:105E900010B5040035F0E4FC0F4B19680A0000E06F
:105EA0000968002902D0A142FAD101E022601C60F9
:105EB00035F0DAFC10BD000000340080440200041C
:105EC000742F0004900100808000008034350400AD
:105ED000F20101007000010004180004E0B90004A0
:105EE00007E003788B4207D04378801CD21A921EB9
:105EF0001818022AF5DA0020704710B51C009A42E3
:105F000000D81400220014F3CAEE200010BD0000D7
:105F10002A48816A0422114381627047FFB581B02B
:105F200000241D00FDF220EC009003F335FE244E0A
:105F30000027B06800281DD004004069B0603068B8
:105F4000401C306001D1012030600198206002982F
:105F500060603068206103986761A0600A982073D0
:105F600003F306FE0100706803F34CFE2100301DB0
:105F700003F36CFE7068002806D03169002903D154
:105F8000806803F315FEF060002C07D0206900281C
:105F900004D0002D00D02860012403E0002D00D0A3
:105FA0002F6000240098802802D1FDF2DEEB02E091
:105FB0000098FDF2E4EB200005B0F0BD0034008055
:105FC00020760400FF4841680068814201D1012029
:105FD000704700207047FB4810B5416800680122F7
:105FE00092070B00040093439443A34205D1114050
:105FF0001040814201D0012010BD002010BDF249A7
:1060000000204861F14A5060EE4A1060C860704755
:10601000EC48416801600168EB4841610021C160C2
:1060200070470021032010B51FF00AFDE6480178F3
:10603000002901D18068016003201FF023FD10BDFD
:10604000F8B504000D00160035F00AFC0700002129
:1060500003201FF0F5FC002C0ED0002D0CD03200D8
:106060002900200014F31AEE03201FF00BFD380066
:1060700035F0FAFB0020F8BD380035F0F5FBFEE7FF
:10608000D14810B58068342114F3A4EE10BDF8B5E2
:106090000C000700002600281CD0CB4D28780128D2
:1060A00018D1012C02D135F0DBFB060000210320C2
:1060B0001FF0C6FCFEF79FF800280DD0FFF79FFFEA
:1060C0000020287003201FF0DDFC012C02D13000DD
:1060D00035F0CAFB0120F8BD35F0C2FB8446FFF75E
:1060E0007AFF002804D0604635F0BEFB002013E0A4
:1060F000E868401CE860B34800680C210004000C0C
:106100004143B3480818002105000A000B000EC0E7
:10611000604635F0A9FB2800002800D1FEE7FA7898
:10612000082A01D8121D00E00C22390014F3B6ED44
:10613000A44800F071F9A749C86B01221043C86355
:1061400003201FF09FFC012C02D1300035F08CFBA6
:106150000020F8BD1CB50024E4439F480122032120
:1061600001AB0094FFF27CF801980028F5D00128DB
:10617000F3D100F061F9F0E710B535F02F755D3916
:1061800001000000A05F000000040000CF42260BC9
:1061900071FB0400002103201FF05CFC9048001DEF
:1061A00000F044F99049886BCA0D104388630320BE
:1061B0001FF072FC200035F061FB10BD002810B507
:1061C0000AD00078012807D1FFF72CFFFFF7DEFF88
:1061D00017F021F9002010BD012010BD10B5017885
:1061E000042901D0012010BD7C494A68521C4A6034
:1061F0000969002901D0884701E0FFF7C7FF0020A7
:1062000010BD0EB504216B46197001215970022191
:10621000D970017819714078587170484168491CEB
:106220004160FFF7B3FF01216846FFF73AFF002006
:106230000EBDF0B587B035F01DFB070081200003CF
:10624000FDF766FF6A490120000588600820FEF717
:1062500041F80820FEF74AF8644866492830016092
:1062600065490161654941605C4C00262661012257
:106270000A200592020003906148012189026B46C1
:10628000049607C3002359485E4AA8385EA100F36C
:10629000EDF9002802D0012007B0F0BD53485CA101
:1062A000FEF276FF0021032026701FF0D3FBA068CA
:1062B0005A4D0068A84207D1FDF7A7FF00280AD071
:1062C000FDF7AEFF002806D0FFF7E4FEA0680560EA
:1062D000FFF79FFE0DE0FFF7A5FE41484660012055
:1062E0006B461874DE742070002104A8FFF7D9FEF5
:1062F000267003201FF0D0FB380035F0BFFA0020D5
:10630000CAE700290CD005280AD2042802D1334854
:10631000016103E0354A80002832115000207047A7
:106320000120704770B5FDF770FF2C4C002802D09B
:106330000020207014E035F09DFA274D060008E09B
:10634000E168002910D02548491E1430E16000F0B2
:106350006DF8606969688842F2D1300035F08EFAD4
:1063600030492F48C86070BDFEE71B48016840688F
:10637000814201D0012000E0002019494A680968E3
:106380008A4201D0012100E0002108430121484058
:10639000704701001548002210B5FEF2FBFF10BD4A
:1063A00010B504000D480178012901D001210170C8
:1063B00020030BD51B491C48C8600820FDF790FF3F
:1063C0000820FDF787FF0120FFF7E3FFE00401D578
:1063D000FFF7A8FF10BD0000801300C008B901C07E
:1063E000001300C0881300C0802A008024FD02C072
:1063F0000030008013600000ED5F0000CD5F000002
:106400007CF802C0795F00004963635461736B00DC
:1064100049636351466C616773000000CDAB0000B7
:10642000FFEFFFFF80220080FFFFF7FF02680123DC
:106430001104090C9B07491C1A4011430A009A4396
:10644000082A01D35940194001607047F8B535F06A
:1064500011FA144C144E154D07001BE0FDF7D5FE44
:10646000002803D012490020087017E070680C2340
:106470000004000C584340190CD00178052905D2BE
:106480008A00A258002A01D0002902D12168884739
:1064900000E09047706831688842DFD1380035F0FD
:1064A000EDF9F8BD4CFD02C0001300C0081300C098
:1064B00008B901C070B535F0DDF90500FF4803F3F8
:1064C0006FFA040009D020005421083014F38CEC3A
:1064D000FA4821000C3003F38DFA280035F0CEF98C
:1064E000200070BD70B5040035F0C4F90500002C23
:1064F0000DD020005421083014F376ECEF48210031
:106500000C3003F3B5FA0100EC4803F373FA2800EA
:1065100035F0B4F970BD10B501F082FB002010BD5C
:1065200070477047002803D02030407D0007C00F1F
:106530007047002807D02030427DF723C9071A4052
:10654000090F0A4342757047002807D02030827D2A
:10655000FB23C9071A40490F0A4382757047002878
:1065600006D08268C90752085200C90F0A438260E8
:106570007047002806D082680223C9079A43890F12
:106580000A4382607047002806D08268F677024589
:10659000010000009C63000000040000E7D3A3B6E4
:1065A0001023C9079A43C90E0A4382607047F8B5A1
:1065B00000250E0017002C00002824D00D21890191
:1065C0004218516A002901D00D000835D16900290F
:1065D00001D00C000834330022002900009704F396
:1065E0001DFE002E06D0002D04D0280048210C30BE
:1065F00014F304EC002F06D0002C04D02000482116
:106600000C3014F3FCEBF8BD70B5040000680028F2
:106610000BD0806D0025002803D0FFF76DFF2068A8
:1066200085652068FFF768FF256070BDFFB589B0FC
:106630001C00A8A605A88ECE139D8EC000210A00BE
:106640000B000E0001A84EC00F001298204302D18B
:1066500001200DB0F0BDE878A9780002AE1D084316
:10666000C00700D0129C002C10D0A07AC0070DD01B
:10667000206D002804D1FFF727FF0028206505D0F2
:10668000206D54220830210014F386EBE878A978B5
:106690000002084380071ED50A98002808D0914AB6
:1066A00009981268012190476B46187D401C1875A7
:1066B0000B9905270622200014F304EB8A4A099857
:1066C000126801219047894A099812680121904770
:1066D00002212D200155E878A97800020843C0075F
:1066E00007D012270621200014F388EB01212D206A
:1066F000015569782A780902E079114300090907F0
:106700000001090F0843E0710320A071687929791D
:106710000002084331002081223110220D0001A81F
:10672000E77234F0DCFC00280CD1200010222E305F
:1067300005A914F3C8EA200010223E3005A914F37D
:10674000C2EA0BE02000102229002E3006F36CFD77
:106750002000102229003E3006F366FD30782073B9
:1067600020001022B11C1D3014F3ACEA31002000CF
:10677000102212310D3014F3A6EAA07A0121084349
:10678000A072002065E770B51B2100224901411865
:106790008A820D21531E890141181D240B631100AB
:1067A00064010725ED014E003618361932828E003D
:1067B00036187619491C04293362F4DB70BDFFB525
:1067C00087B000200C001500109E1F00002E0390C3
:1067D00067D07078317800020843032841D10798C8
:1067E0000196009540790121022800D00021404AFD
:1067F000079823008218FFF719FF002C039007D099
:10680000E07901210007000FE071E07A0843E072AF
:10681000002D07D0E87902210007000FE871E87A1F
:106820000843E872002F07D0F87940210007000FD5
:10683000F871F87A0843F8727078317803020B43E4
:1068400007990F208001081806902000403005901D
:1068500028004030049014F352EC050C2525BFD0DD
:10686000DE0007983B002A002100009604F30AFD91
:10687000C3E70799112040010918B2790120CB79AB
:1068800090408343002DCB7104D00499049A497A37
:1068900001435172002C9BD00599497A0143059818
:1068A0004172B8E0F078B178000208438107079898
:1068B0000D2292018018002984462EDA002C31D056
:1068C000A07AC0072BD0079800281AD0604611E0A4
:1068D000E8E401C0365C365C365C365C365C365CBF
:1068E000365C365C64F800045CF8000458F8000478
:1068F00029020000806B002803D080308188491C69
:10690000818000202086401EE0620798FFF73BFF51
:10691000002060630120208701E0002C02D005994F
:1069200000200874002D02D0049800210174002F6B
:1069300002D0002040373874F078B1780002084364
:10694000C0070FD0002D0DD0A87AC0070AD0079835
:10695000002807D06046806B002803D08030018972
:10696000491C018107984079022829D1F078B17833
:1069700000020843800723D5002C21D0A07AC0074D
:106980001ED0079839F060FD0700079839F083FDA5
:106990002037797889060BD506990969BA6EA83728
:1069A000010000009867000000040000B40970DADC
:1069B0006031097CC90705D080300069002801D00A
:1069C000012100E00021079821F0B7FAA07AFD210B
:1069D0000840A072F078B17800020843C10724D0C3
:1069E000002D09D00006810F04980174F078B17869
:1069F00000020843C00718D0069800696030007C88
:106A0000C00712D1079800211BF06FFC0DE0002F8A
:106A10000BD0F078B17800020843400505D50798FF
:106A200040790328EED00128ECD01AF079FD002C33
:106A300005D0A07AC00702D007983CF08EEB0398EF
:106A40000BB0F0BDF3B581B000260198002866D0E8
:106A500001980D2189014418606A002802D1FFF7CE
:106A60003DFD6062019839F0F9FC019949790229EC
:106A700025D1050020304078C10903D1010701D498
:106A8000800641D52F0080373868002804D1FFF7F1
:106A900025FD0028386042D03868E061019821F077
:106AA00062FA002806D0FFF719FD85218900002829
:106AB000485134D0FF35FF35AD1C68691FE003290C
:106AC0000ED1206A002803D1FFF708FD206207E0FD
:106AD000E169002907D008310830542214F366E92F
:106AE000E069002802D1FFF7F9FCE061019821F08C
:106AF0003AFA002801D1A06A02E0FFF7EFFCA06299
:106B0000002801D006000836606A002807D0E06936
:106B1000002804D0019821F026FA002802D0002095
:106B2000C043FEBD616AE069029A0830009202002B
:106B3000019808313300FFF74CFEFEBD70B514001C
:106B40001D0000290AD0012809D0022801D00428FC
:106B500004D10A002900200014F3BEE870BD102201
:106B60002900200014F3B8E810352000082229007D
:106B7000103014F3B2E82900083108222000183040
:106B8000EAE7F8B5040039F090FC200039F066FC23
:106B9000210020314B7DF72213404B75A568042658
:106BA000B5432122A560125C97070AD50D229201F8
:106BB000C56FA218D561C06F5062082003434B75A2
:106BC00005E0100701D4900601D53543A5602000EB
:106BD0003CF0C2EA0020F8BD30B4C27903231209A8
:106BE0001201121DC271102583710581C37A4024E0
:106BF0002343C372CC8C50231C54837A0124234337
:106C000083728B8C03870B6A43630023140703860C
:106C1000C362240F0B0002000C322900200030BC9C
:106C20008CE7F7B58CB0060039F03FFC00903000DF
:106C300039F014FC2121095C04000A0701D48906FB
:106C400067D5B168042211430D22B1600D999201FC
:106C5000B518012910D137210901471820008030CB
:106C60000B900068002803D1FFF738FC0B990860EF
:106C70000B980068E86113E00E99012912D1772181
:106C8000C9004718300021F06EF9002804D0FFF742
:106C900025FC852189000851852080000059A862C3
:106CA000050007E06D6A28222900343101A814F399
:106CB0007EE801AF002D02D101200FB0F0BD0D988C
:106CC0000835012804D100202200E832287013E0A2
:106CD0000E98012805D1FF220121280034F034EA62
:106CE0000DE0112040013018407A2870B06803216F
:106CF0000843B060009A30320E98002804D0390062
:106D00002800FFF769FF04E00D983B00290004F319
:106D1000ABFD30003CF020EA0020CEE710B50400C7
:106D200002008034206800280FD0C17B2032090780
:106D3000090F01290AD0022908D0032905D150786A
:106D4000C00902D12000FFF769FC10BD51780A0785
:106D5000FBD48906F9D4FFF7D9FB0020206010BDD1
:106D6000FFB5002091B00E0014001A9F1D00002BEB
:106D70000B9004D0E8790007000F2030E871002C58
:106D800004D0E0790007000F2030E071002F04D01C
:106D9000F8790007000F2030F8712100F37A0C31E8
:106DA000109129000C310F9121003000BCA7A8F4EC
:106DB00001000000946B0000000400004066056EB6
:106DC00040310E300E9114F3AEE905047E7EFE7E56
:106DD0007D000700002C75D0002DFCD0B07A04286F
:106DE00070D2707B317B000208434007A07A02D545
:106DF0000121084301E040084000A072E079F17AE7
:106E0000000909070001090F0843E0717878397813
:106E10000002084320810320A0710E98B27A417AC3
:106E20000120904001430E980D224172B07AB91CA6
:106E30000301181A00190C300A90801C13F356EF46
:106E400078783978000208430D28E07A04D10821C7
:106E50000843E072012003E0F7210840E0720020BF
:106E60000A9948700A98B17A0170707B317B0002F0
:106E70000843000702D50E99B07A0872A07AC007BD
:106E80001FD0119801218068022208431043119AF3
:106E90009060A87AC20702D0EA79120711D108439C
:106EA000A872E8793F2200090001E8710320A87167
:106EB0007878397800020843288110990F9813F3E5
:106EC00080EF06E2DBE10A9011980F21890140185A
:106ED0000D9030001830002D0C906ED0707B317BFF
:106EE00000020843810768D54007A87A02D501212E
:106EF000084301E040084000A872E879F17A0009EF
:106F000009070001090F0843E8710A98417A027ADB
:106F10000802104328810320A871B17A50204155FE
:106F20000121E972A87AC00734D011980321806842
:106F300008431199886000202886401EE862119855
:106F4000FFF735FC002068630120288711984079FD
:106F5000022842D1119839F08BFA0990119839F032
:106F6000AEFA09992031497889060BD50D9909693E
:106F70006031097CC90705D080300069002801D044
:106F8000012100E00021119820F0E1FFA87AFD2105
:106F90000840A8720D980069FF302130C07F00289A
:106FA00001D001200B900A980C9B417A007A0902CB
:106FB0000143F07A0F9AFFF7CBFD002C6BD0707B6A
:106FC000317B000200E0C2E00843C10763D0400704
:106FD000A07A06D50121084305E0A87A02210843DA
:106FE000D7E740084000A072E079F17A000909076C
:106FF0000001090F0843E0710A98417A027A0802F9
:10700000104320810320A0710E99B07A0874E07AB1
:1070100002210843E072A07AC0072AD0707B317B3E
:1070200000020843800614D50A9920000A7820300F
:107030000274497841740A990422891C0C3013F3B4
:1070400056EE208E002804D1E06A002801D1401EAF
:10705000E062707B317B00020843C00603D500204C
:1070600060630120208711980321806808431199EB
:1070700088600D9800696030007CC00701D1012054
:107080000B900A980C9B417A007A09020143F07A2E
:10709000109AFFF75DFD002F7ED0707B317B0002E0
:1070A0000843410578D54007B87A02D50121084345
:1070B00001E040084000B872F879F17A0009090748
:1070C0000001090F0843F8710A98417A027A080210
:1070D000104338810320B871B17A5020C155F87A35
:1070E00040210843F872B87AC00724D0707B317B06
:1070F00000020843800614D50A9938000A78203027
:107100000274497841740A990422891C0C3013F3E3
:10711000EEED388E002804D1F86A002801D1401E17
:10712000F862707B317B00020843C00603D5002063
:107130007863012038870A983A00417A007A090278
:107140000143F07A0C9B0C32FFF702FDBDE00021F9
:10715000099005A80A91FF4F8ECF8EC000210A002A
:107160000B000F0001A88EC0707B317B000208432A
:10717000810700D50A95C00700D00A940A98002814
:107180007DD00A98807AC00712D00A98006D002836
:1071900007D1FFF7ADF900E094E00A9900280865EF
:1071A00006D00A980A99006D5422083013F308EEAD
:1071B0001199012449792000022900D0A54020C856
:1071C00001000000906F00000004000013BCD60214
:1071D0000020717B327B0902114389071FD50028EB
:1071E00009D01198102180686B4608431199886076
:1071F000187D401C18750A980521C172DB49119849
:10720000062241180A9813F37CED1198119A8068B0
:1072100002212043084390600A9820304173707B1C
:10722000317B00020843C0070BD00A991220C872B4
:107230000A98062113F300EE0A98203044730120C7
:107240000B900A98F17AC079090700090001090F2B
:1072500008430A99C8710A99032088710998417CEA
:10726000027C08020A99104308810999102201A89A
:1072700033F053FF00280DD10A9810222E3005A9B3
:1072800013F33EED0A9810223E3005A913F338EDB2
:107290000CE035E00A98099910222E3005F3E2FF40
:1072A0000A98099910223E3005F3DCFF0A98B17A5A
:1072B000017309990A98102212311D3013F320ED41
:1072C00009990A98102222310D3013F31AED0A9809
:1072D0000A99807A204388720B98002803D011986D
:1072E00000211BF016F81AF02FF9002D05D0A87A0E
:1072F000C00702D011983BF044EF002015B0F0BD5C
:107300000120FBE7F7B582B0002702983E00019705
:1073100039F0B8F80299029B0D22497992019C1824
:1073200002292AD1050020304078C10903D1010784
:1073300001D480064AD52F0080373868002804D150
:10734000FFF7E0F8002838600ED03F68E761029848
:10735000083720F01CFE00280AD0FFF7D3F885215B
:1073600089000028485103D10020C04305B0F0BD7A
:10737000FF35FF35AD1C686923E003290ED1206A73
:10738000002803D1FFF7BEF8206207E0E169002979
:1073900007D008310830542213F31CEDE0690028AF
:1073A00004D1FFF7AFF80028E06101D0E7690837A2
:1073B000029820F0ECFD002801D1A06A02E0FFF75E
:1073C000A1F8A062002801D008300190606A00286E
:1073D00004D1FFF797F80028606201D0666A08368A
:1073E000019A00920499029833003A00FFF7CCFC0E
:1073F000BCE770B505000C000026081D31F049F807
:10740000002815D1201D31F035F8002810D1F120C9
:10741000800029180622201D33F07FFE002807D0A7
:10742000201D39F0ADF8050001D1012070BD012605
:10743000220031002800FFF765FF70BDFFB589B05D
:1074400004001F00129E002E77D0002CFCD02000DC
:10745000403008902338079010380690401E059061
:1074600010300490083003903801C01B00190290BE
:1074700020003E30FF29019004D1E0790009022864
:10748000E2D0E4E00229FCD1FF209D303070000AF8
:1074900070700A20B0700020F0700B990622301D29
:1074A00013F32EECE0790007000FF072E07A41064A
:1074B00002D50121890204E0800701D5012100E005
:1074C00002213173090A7173E07903071B0F300041
:1074D0001900103013F330EE05043232323231002D
:1074E000042F2AD2B7720899097AB94208D1717B60
:1074F000327B09021143082211433173090A717367
:107500000299497B002901D1052100E00D21B173C9
:10751000090AF173F17BB37B0A0202991A430E3117
:1075200013F3EEEBF078B2780102F07B1143B27BFB
:10753000000210430818801C31E02AE13500303584
:10754000032944D1217BB1722021070081730020DF
:10755000F87330000E3001991022009013F3D0EB35
:1075600010223000203003E0D06600002902000025
:10757000079913F3C6EB06991022280013F3C0EB0A
:1075800001990098102205F36DFEF078B1780002A1
:107590000843F97BBA7B0902114340181230B070DE
:1075A000000AF070A07AC00708D0707B317B00021F
:1075B0000843042108433073000A7073F078B178EF
:1075C00000020843001D0004000C0DB09C8D0BFD53
:1075D000010000008C73000000040000AC79F3B1DE
:1075E000F0BD08990A7CB2722289B275120AF2754E
:1075F000228E21001378B3735278F27304222C3157
:1076000013F388EB002131757175E07901073000C3
:10761000090F1830012911D12021B1750021F17510
:107620000599102213F376EB3000049908222830D4
:1076300013F370EB08220399280005E02189B17546
:10764000090AF1752289059913F364EBF078B27891
:107650000102F07D1143B27D0002104308180A3088
:10766000A7E7E079351D0007000F3071000A70713F
:10767000FF20401C3070000A00227070B270F2705F
:10768000E07A410602D50120800204E0800701D59E
:10769000012000E00220A870000AE870E0790107EC
:1076A0001ED1A81D042F7ED221892971090A697172
:1076B0000899097AB94202D10121417000E0427073
:1076C0000770029922890E31801C13F324EBF178A4
:1076D000B07809020143891CB170090AF17041E0D8
:1076E0000007000F012813D12020287100206871A5
:1076F00005991022A81D13F30EEB28000499082207
:10770000163013F308EB0822280003991E300AE014
:10771000022801D0042809D11020287100206871A6
:1077200005991022A81D13F3F6EA1BE0032853D194
:1077300020892871000A6871207BA8710120E871F6
:10774000AF1D07991022B81C13F3E4EA380006991C
:107750001022123013F3DEEA380001991022223091
:1077600005F38AFDA07AC00708D0E878A97800025E
:10777000084304210843A870000AE870F178B27841
:107780000802697910432A79090211434018801DC3
:10779000020AB070001D0504F270E0792D0C00079C
:1077A00018D0741900E017E0FF2121312170090A77
:1077B00061700621A1700021E1700B990622201D45
:1077C00013F3A8EAE178A278080210432D1D4019AE
:1077D00005042D0C280002E7002000E7FFB581B06A
:1077E000002501980A9EC079000718D1042B16D3F2
:1077F000019F002440370120797AA04001420AD03D
:10780000230601A8009607C81B0EFFF721FE3618B5
:10781000281805042D0C641C042CECDB05E001A8E1
:10782000009607C8FFF714FE05002800A8E5FFB57D
:1078300081B000240500160080681F0040051DD59A
:10784000287901281AD0022818D1280038F024FEFF
:10785000002E13D1002811D08030006800280DD0F0
:10786000F90745D00B9AF121890000926A18029914
:1078700008300023FFF7ECFD040039E0F049B807B9
:107880006E180D2189016D1800280EDA686A00282B
:107890000BD00B9A00920A9B029908303200FFF736
:1078A0009DFF0B99091804000B91F80710D0E869A7
:1078B00000280DD00B9A00920A9B029908303200E2
:1078C000FFF78CFF0B99091820180404240C0B9166
:1078D00078050DD5A86A00280AD00B9A00920A9B59
:1078E000029908303200FFF779FF20180404240CB5
:1078F000200045E5FFB587B0FF2100261F00089C4A
:10790000D04B35003000062C059607D202000798B0
:1079100001970091FFF78BFF06007BE0140071E0F8
:10792000C8480490FF2003900020029060782178DE
:1079300000020843C11FF9390FD103990197009143
:10794000E179A0790B020343029A07980021FFF71F
:107950006EFF05003F18301844E00100FF399D39E3
:1079600042D107980690E078A178000208430628E3
:1079700029D3201D30F097FD002814D1201D30F0B0
:1079800083FD00280FD10798F121890041180622B4
:10799000201D33F0CCFB002805D0201D38F0FAFD67
:1079A000069001200290E178A278080210430A288C
:1079B00009D3A07A0390627B237BA248110219436A
:1079C00000D0080004900698002809D00399019778
:1079D0000091049B029A06980221FFF768FA840A34
:1079E000010000008877000000040000FFA320DDF4
:1079F00028FF05007F1970190604360CE078A1787D
:107A00000002084305998300091D41180904090C67
:107A1000181804191434059108990598884203D25E
:107A200019208001864285D330000BB0F0BD70B5BF
:107A3000060004680834E07903071B0F934201D065
:107A4000012070BD000712D1042910D22500403555
:107A50000122687A8A40904368720801401A00192E
:107A60000C300F2113F326EA687A002804D130681D
:107A7000FEF774FD00203060002070BDFFB581B0BE
:107A8000040000201D000A9F0090A0680026400509
:107A9000002827DA2079012824D0022801D00328E1
:107AA00020D1200038F002FD2179032902D161792B
:107AB000022917D1002F15D1002813D080300700DC
:107AC000006800280ED0E90752D0C17B0A0703994D
:107AD000120F8A4202D00399FF2949D1FEF73EFDD9
:107AE0003E6045E00D21029889016718FF281BD1EF
:107AF0005A48854218D1786A002802D0FEF72EFD38
:107B00007E62F869002808D0FEF728FDFE61386A19
:107B1000002802D0FEF722FD3E62B86A002827D076
:107B2000FEF71CFDBE6223E0786A002808D0A80793
:107B300006D5D9208000039A02992018FFF777FF15
:107B4000F869002808D0E80706D0D7208000039AFB
:107B500002992018FFF76BFFB86A002808D0680563
:107B600006D56D20C000039A02992018FFF75FFF29
:107B700000980FE4F7B586B0002707983E00062866
:107B800064D314005EE0FF20049003900020029074
:107B90006078217800020843304DC11FF93901D1C6
:107BA000012643E00100FF399D393FD10698059039
:107BB000E078A1780002084306282BD3201D30F07E
:107BC0007CFC002814D1201D30F068FC00280FD167
:107BD0000698F121890041180622201D33F0B1FAE0
:107BE000002805D0201D38F0DFFC05900120029010
:107BF000E178A278080210430A280BD3A07A0490F7
:107C0000E07A0390617B207B0D020543124805401A
:107C100000D1124D0598002808D0029A0092039ACC
:107C2000049905982B00FFF729FF0643E078A17817
:107C3000000208433F1DC11983000F0418183F0CB0
:107C400004191434079887429DD300E001263000C0
:107C500009B0F0BD2902000003040000FFFF00008E
:107C6000002810D00D2189014218916B00290AD0FB
:107C70000B695B1C0B61916BCB685B1CCB60916BE0
:107C80000A6E521C0A66112149014018C1798022EE
:107C90001143C171704770470548142110B513F3A3
:107CA000E0E804480121017000218160C16010BD3D
:107CB00060FD02C020B901C070B538F01EFC0400A0
:107CC00033F014FE0500206C02F3B3F80021280005
:107CD000216433F00FFE70BD70B50D00080038F060
:107CE000E5FB0600280038F008FC04002C34A179DC
:107CF0003000227AE830042905D86030407C824286
:107D000013D30F2204E06030807C82420DD3102216
:107D1000022901D001290DD120002030017E012946
:107D200008D1217202210176A1790022280000F0F9
:107D30002CFA70BDFF48291828002AF021FF0A20DC
:107D4000A07170BD38B5040038F0D7FB02002032B6
:107D50000168937CE8315D1E032D01D8496F03E073
:107D60005B1F032B1CD8896F137D002B05D07D234F
:107D7000DB00994200D30B001900127A012A04D1CA
:107D8000ED4A914200D30A001100002200927D22A8
:107D9000D2004A430300E94840332100FEF704F9CA
:107DA00038BDF8B5002844D0002942D00500603520
:107DB0002A7CEB7B12021A431206120E84187134CD
:107DC000DD271C2027706070DD480278A2704278A1
:107DD000E27080782071092060715020405CA071B1
:107DE0000A8E2281CA6A20000A3004C06D90C68BB8
:107DF00001000000847B0000000400000BCC5569EA
:107E0000060010220C3112F39AEF297CEA7B09025A
:107E10001143627830008918891C0A0AE9732A74B0
:107E200010300822511A4C07640F0CD00770611EE5
:107E3000401C13F34AE8287CE97B00020843001940
:107E4000E873000A2874F8BDF7B582B01400060084
:107E500038F05DFB0500300038F032FB07002200EF
:107E6000300001A9F9F754FE04002AD0F0686061DF
:107E700020890721001901730198722113F324E866
:107E8000F12080003218B0483118019810F322F91F
:107E90002C35687901231A00062800D000222879A1
:107EA000000704D4E037387A000700D40023A8780C
:107EB0008006C10F019810F3D3FB0398019901606C
:107EC000200005B0F0BDF3B587B00A000025079883
:107ED00005A9FFF7B9FF0028089002D1012009B0D9
:107EE000F0BD079838F013FB0490079838F0E8FAD3
:107EF0000700049804002C34200000F0AAFD20693B
:107F00000290E06803907320C0003A180092A078B5
:107F100039008006C00FC203E8310598803202ABF9
:107F2000069102F310FF0598069B010060310A7C60
:107F3000C97B16020E43372109017A18A11C03F3ED
:107F4000B3F8059802006030017CC77B0B023B430D
:107F5000991B182902DD18390D042D0C0499803164
:107F60000969002911D007990D26B60189198E6A71
:107F7000002E0AD0002D03D05B1BC3731B0A0374B1
:107F8000896A10000831FFF716FF21000598221DAD
:107F9000283102F3B6FF0598017D4B0738210A5DB1
:107FA00021005B0F183110F3D1F801000898F9F7A0
:107FB00064FE002093E7F3B589B00A0007000020B3
:107FC00005000390380007A9FFF73EFF00280A903C
:107FD00002D101200BB0F0BD380038F098FA06004D
:107FE000380038F06DFA06900D208001381808909E
:107FF000406A340014302C340290200000F029FD37
:1080000020690490E068029A05900092A0781121FE
:108010008006C00FC003C90142180798211D04AB98
:1080200002F391FEC037B86801894018A1780A07A9
:1080300008D504220092484B0822DD210BF380FE74
:10804000039009E0890607D500220092082230211A
:1080500000230BF375FE0500039A07982B00A11C63
:1080600002F3E2FF002838D0A078800639D50798BF
:10807000069A03006030017CC07B0F02074306981C
:108080003721090141180025E832180002F3D2FE19
:10809000079802006030017CC37B09021943CB1BA7
:1080A000182B02DD183B1D042D0C80363369002B84
:1080B0000BD0002D03D0491BC173090A0174089825
:1080C000816A10000831FFF776FE21000798221D13
:1080D000283102F316FF002803D10A9813F38CFB12
:1080E00077E70798017D4B0738210A5D21005B0F78
:1080F000183110F32BF801000A98F9F7BEFD0020A3
:1081000068E77FB506000D0038F001FA04002A0088
:10811000300003A9FFF798FE050002D1012004B04A
:1081200070BD0D2080013018466A2C3414362000B2
:1081300000F08FFC20690190E0680290202130005F
:108140000FF3A4FA012209E029020000B80B000095
:10815000717A000047F731004EF731000398D202E0
:10816000211D01AB009602F3EEFD039A20341000AE
:108170006030017CC37B080218435F300104207E1D
:108180009073090C0320D07308020B0A1843107473
:10819000000A50742800F9F770FD0020BFE7F7B51A
:1081A00082B00C00029838F0B2F90700029838F05B
:1081B00087F96846FDF767FD386C002802D0029801
:1081C000FFF784FDE00702D1641E2406240E3D0063
:1081D0002035AC7402991122287A52018E18012898
:1081E0000AD180373878002806D1718A0298012296
:1081F0000DF071FB002426E0012C04D1B8F2D2016D
:1082000001000000807F0000000400005816860571
:1082100004990298FFF77FFF0EE0032C04D1049924
:108220000298FFF7D2FE07E0052C01D0072C1FD1E2
:1082300004990298FFF751FE040002D1A87C401C6B
:10824000A87402980FF03CFD002804D0718A0298AF
:1082500000220DF04AFB002C02D1287D401C28751D
:108260000298FFF783FD6846FDF734FD200032E6F3
:108270000498002802D0049813F3C8FA6846FDF762
:1082800029FD012027E610B513E0200038F049F958
:10829000A1682C30C90407D580790A2804D10022AE
:1082A00007212000FFF785FFE279A179200018F06F
:1082B0008EF80400E9D110BDFF4910B50988C184CA
:1082C000012181840021016210210FF3E9F910BD21
:1082D00070B5050038F0FEF84B210400C9004018C5
:1082E000F12189006A180100FF31FF304131193056
:1082F00002F325FF2120005D800611D50F208001AB
:10830000281800696030007CC00709D07720C000C1
:108310002018FFF7D1FF012200212800FEF7BDFC45
:10832000002201212800FEF7B8FC70BD70B50500E1
:1083300038F0D0F8060033F0EDFA04000F20800189
:108340003118CA6A002A0ED0521ECA620BD1886A3E
:10835000C8622800FFF7BCFF200033F0DFFA2800D6
:10836000FFF791FF70BD200033F0D8FA70BDF8B56B
:10837000050038F0AFF807000400F120F83780005E
:10838000732137233E002A18C9001B0141366118AA
:10839000E01802F3D4FE0D2189016418E069012878
:1083A00009D1A820415D280033003A0088300FF33E
:1083B00037F90020E061F8BDF0B50600A9B04569C5
:1083C000280038F0AEF80B90280038F083F80A90B7
:1083D0000B980CAA04000D2080012818476A3089E8
:1083E0002C3486190A98289030006330417814376D
:1083F000891C2FF08FFC28980122E0308446807A77
:108400000990289807A903008033D86E08900E9829
:108410000490069205916046C089189AA11C0392A7
:1084200002910190986E0090089B099A2100280003
:108430002BF072F8012804D11121280000F007FB6D
:1084400024E00A9B6179FF333A330120062900D0EA
:1084500000200200200039002031283004920391CE
:108460002200310002909548183211310091140019
:10847000291801922A001800AC323B0002F3B1FD2A
:10848000210030000FF340FE002802D1012029B066
:10849000F0BD2800FFF724FC0B9800212030017567
:1084A0000A0003212800FFF784FEF0E7012805D029
:1084B000022803D0FF38401E01D10620704700205B
:1084C0007047FFB583B0060000250D990C98029106
:1084D00011780191077804993020012900D0DD201E
:1084E00030700498002806D075490322684612F3BC
:1084F00030ECB41C0AE073490322684612F328ECFE
:1085000070490422B01C12F324ECB41D0120207029
:1085100000206070A41C03222000694612F318ECAE
:10852000002F04D0380001F343FB05042D0C28066E
:10853000000E03F3B3F9E0700698241D207006982E
:10854000000C6070A41C002515E06B4618782070A4
:10855000587860709878A070019801F329FB07049F
:108560003F0C3806000E03F399F9E0700198241DC2
:10857000B8436D1C019006988542E6DB0E9820708A
:108580000E98000C6070A41C002514E06B4618784F
:108590002070587860709878A070029801F308FBFA
:1085A0000104090C0800FFF781FFE0700298241D08
:1085B00088436D1C02900E988542E7DB04980028E2
:1085C0002ED00F98002827D00F980178217040787E
:1085D00060701098A41C20701098000A6070A41C91
:1085E000002509E011991022200012F3B2EB119836
:1085F000103410306D1C119010988542F2DB0F98EA
:108600000078C0090CD02E490322200085CCF0163A
:10861000010000007C830000000400000E3FE545DF
:1086200012F3A0EB0620E070241D03E00020207070
:108630006070A41CA01B0004000C811E717007B0A8
:10864000F0BDF0B587B004008C4696460CAD0FA87F
:10865000E0CD07C8009503AD0297019607C520003D
:1086600072466146FFF737FF0004000CE7E7F0B5FC
:108670000E000700002189B01BF093FDFF2291320C
:10868000512307A908A809F032FE002836D0380087
:1086900037F02AFF07990022103103000D00E8335C
:1086A0000392049205921A89D9880093029201914B
:1086B000B07808358006AC1CC10F321D20000123A4
:1086C000FFF7BFFF20782870000A07E04602000489
:1086D0002902000047F731004EF7310068706078DA
:1086E000A870010AE9700799001D8872000AC87213
:1086F000FD48089A3918380009F0D3FE03E4F8B5AC
:1087000006004769380037F016FF050004000D2009
:1087100080013818406A2C351430009030892900C7
:10872000801918310FF3FAFC002801D10120F8BD9F
:1087300000980121403000268180009832000664B4
:1087400031003800FEF7B3FA002804D001213800C8
:1087500000F087F9EAE73800FFF7CCFA3420065535
:1087600020682030407880060DD50F208001381811
:1087700000696030007CC00705D080342069002883
:1087800001D0012100E0002138001FF01CFCA87876
:10879000800607D529003800FFF769FF0A20A87175
:1087A0000020F8BD002205213800FFF70CFDF8BDC0
:1087B000F8B5018946690F18300037F0BCFE040097
:1087C000010005002C34443138000FF3A7FC0028C9
:1087D00005D11121300000F044F90120F8BD30002E
:1087E000FFF788FA002020352875A079062803D1E4
:1087F00021003000FFF73BFF0A20A0710020F8BDE8
:1088000070B50E00C1790500807937F0A4FE06E04E
:10881000AC4206D1E279A179200017F0E2FD040014
:1088200018E0200037F087FE010020318A7CD20753
:10883000F0D0097A002905D00129EBD18021095C0B
:108840000029E7D02030817C32002000FFF7BBFCFC
:10885000012070BD002CDBD1002070BD10B50400DC
:1088600037F042FE002811D06179E83002290DD19D
:10887000A16849070AD55021095C002906D0408922
:10888000C10703D1800701D4012010BD002010BD15
:10889000F8B50E0033F048F8002E009027D03000D5
:1088A00037F022FE040022D01B2040012518287832
:1088B000002701281CD0022816D1E820005D4007BF
:1088C00009D53000FFF7CAFF002804D00F2080012F
:1088D0002018816AC1620D20800120182F708762E4
:1088E0003900300000F0B1F8009833F021F8F8BDFD
:1088F0002F70F9E7F1B582B0029837F0F5FD0D2140
:10890000890104004518686A00283CD033F00CF84F
:1089100001901B204001261830780127002833D011
:1089200001282DD10220AF623070E86A01F39FFA6E
:10893000DB2000228000231800926C4A6C480299C8
:10894000FDF750FB019832F0F3FF0298272129F040
:1089500091FFE820005D40070CD50298FFF77EFFED
:10896000002807D00F21890100206118C8620298F1
:10897000FFF7B8FCA86A01040298090C00F065F83A
:10898000019832F0D5FFFEBDDB20002280002318C5
:108990000092564A56480299FDF724FB3770EFE7DC
:1089A00070B505004669300037F0C5FD0400B068B9
:1089B000C00407D5288941194879400703D53000FC
:1089C000FFF798FF70BD200009312C3000F05DF8F2
:1089D0000028F7D02034A07C022803D12800FFF71C
:1089E000F5FC70BD042803D12800FFF788FE70BD98
:1089F000062801D00828FAD12800FFF7D9FE70BD5B
:108A00003EB5FF220400062101A832F0E4EB00226B
:108A1000009220000E2301AA01A90BF0F9794E81E2
:108A20000100000078870000000400005DE53629A1
:108A3000DFF832F083FF0500E179A07937F095FD8A
:108A400007E020002AF0BFFBE279A179200017F0AF
:108A5000D2FC0400F5D1280032F074FF3EBD13B5FE
:108A6000040037F04BFD284B20001C684C210223EA
:108A700001AAA0471CBD70B504000D00FFF744F922
:108A80001E482A00211820002AF0A2F870BDC168F3
:108A9000491CC16002D10169491C016170477CB564
:108AA00004000D00042201A812F366E90422291D26
:108AB000684612F362E90198FF21090202000A40A8
:108AC000030612029D1803000A0213401B0AEB184A
:108AD000000E18182369984218D100980140030627
:108AE00009025B1801001140090A5918000E081804
:108AF000E16888420AD101207CBD00002902000003
:108B000000879303ED85000088F800040020F3E758
:108B1000FD4900201422424352189268002A01D0D5
:108B200000207047401C0128F4DB01207047F0B59D
:108B30008C001025AC4315012C43F44DF44E2C4011
:108B40000125AD05651900278400A6193560F04D93
:108B5000403564192360EC4C0501583C2C19402623
:108B600027736673E84EC907583E73516360E37B11
:108B7000C90F5B085B000B43FD210B40D107890F38
:108B80000B43042119430228E37302D31900FB208D
:108B90000140E173A773A760F0BDDE4870B5012303
:108BA00001688A09C16992011A4343049943194330
:108BB000C1610260D8494161D8494162C162D84966
:108BC0008160D849C160D04D0024283D1420604305
:108BD00000224019402112F3B9FE641C022CF5D387
:108BE000C94D00241420604300224019402112F393
:108BF000ADFE641C012CF5D370BD70B5FCF745FECD
:108C0000FFF7CBFFC84D0024E000001B000200214D
:108C100043190A002000FFF78AFF641C2406240E73
:108C2000032CF1D370BDF8B505000020009032F0A0
:108C300085FEB54E07000024283E142060438019AD
:108C400012F3B4FE08E04169A94204D1380032F0C1
:108C500079FE0120F8BD00680028F4D1641C022CC4
:108C6000EBD3380032F06EFE0098F8BDF3B589B052
:108C70000998A749800008904018006A4022C10165
:108C8000C90D571A09990406CB00A74A240E5B1A8E
:108C900014201B0248439A182500029402290792C7
:108CA00055D2994928394018069012F37FFE0600E4
:108CB0004AE070690A99884245D130898019006F6D
:108CC00004900020039701902BE01C21614307983A
:108CD000049A4118486890420BD100963668009972
:108CE000069838F0FDFD0098002132F015FE7F1E39
:108CF0001AE01C226A43079880181C2212F3A6E887
:108D000000210800402D00D0681C05062D0E402CC7
:108D100000D0611C01980C06401C240E0006000EB9
:108D2000019003998842D0D30399019888420BD1CE
:108D3000009636680099069838F0D2FD0098002118
:108D400032F0EAFD00E03668002EB2D14EE009991B
:108D5000891E01294AD26C4940182838059012F31F
:108D600025FE060040E070690A9988423BD13089AF
:108D70008019603012F342E90490002003970190BB
:108D80002AE01C2161430798049A411848689042E0
:108D90000AD1009636680099059838F0A1FD009830
:108DA00034F06BFB7F1E1AE01C226A430798801880
:108DB0001C2212F34CE800210800402D00D0681C52
:108DC00005062D0E402C00D0611C01980C06401C9D
:108DD000240E0006000E019003998842D1D3019918
:108DE0000398814200D13668002EBCD11C23029921
:108DF0003C0059435C4307982200411812F326E8CF
:108E0000099800F095F8424A01200899C0073843B4
:108E100040328918086209983B49079A000158397D
:108E20000A50079A4018121900214260EB84ED1194
:108E300001000000748B000000040000A98A439D1B
:108E400001734021C91B41730BB0F0BDF1B582B075
:108E5000FCF725FD00240127BF073248A1000E18AA
:108E60003568280038433060306A4000FCD532F065
:108E70006FFD0190680704D420060299000EFFF7E9
:108E8000FFFEBD433560019832F066FD641C032C83
:108E9000E3D3FEBDFFB583B0FCF701FD00262148FA
:108EA000B1000F1838680121890701900843386024
:108EB000386A4000FCD514201849704328394018FE
:108EC00012F37EFD04001E4806990818029017E070
:108ED00020890599051928784007400F88420ED14E
:108EE000286F0299801D062232F05DF9002806D114
:108EF00004997C2041550698290034F0D9FA246859
:108F0000002CE5D101980121890788433860761C3F
:108F10003606360E022EC2D307B0F0BD68610400DB
:108F2000FFFF00FE00A1009000A0009098DB01C0B0
:108F30000700070F40A0008050E8008000E901C052
:108F4000290200008100034808180168012211432A
:108F50000160704700A10090FF490020087248722C
:108F600060390867C8664867FF31491C8860C86077
:108F7000B0398864C8648865C8658866C86608674B
:108F80004867086448648867C8678031086048603B
:108F90007047FEB5040032F0DBFC00900120102C7D
:108FA00004D0202C02D0402C00D00020EA496039A7
:108FB0000A780E00303EA24210D1E84F820092198A
:108FC00053697D6EAB4209D19268BB6E9A4205D15E
:108FD0004200921952887B8A9A4264D042009219C8
:108FE00002925288D20702D07D25ED0000E00125D3
:108FF00080008619B2686B461004000C120C988031
:10900000DA807769D449381A68436039002A886061
:1090100010D1102C07D1D248D249784312F306EC74
:109020006B46D8800EE0CE48CF49784312F3FEEB72
:109030006B46D880402C05D1FAF721F87D23DB0060
:10904000584303E06B46D888381A6843C2496039F0
:10905000C86070690A00C44968431161C34950601F
:10906000091A1162C0494942401850616006400F18
:109070000BD002984088010A02D0000A684300E041
:10908000BB485064BB489064D064FFF765FFBA49A1
:1090900001200860B148147071694166B168816649
:1090A000029949884182009832F056FCFEBDAA48D8
:1090B0000021017241727047F3B581B00D00A80024
:1090C000A54CA64E603CB1780719B8688D4209D10D
:1090D00072780199914205D1F16E884202D1616B9B
:1090E00000291ED19C4A903A116A401AC10F0818F3
:1090F00041106163506A814200DC010061630091AC
:109100000098032111F3A4EF00222264E063009988
:109110002163A063E270A270B868F066B570019830
:109120007070FEBD70B504268C4C944D00280ED096
:10913000F9F741FF002803D0F9F7DBFF002805D03D
:10914000E088401CE080E868B043E86070BD20899A
:10915000401C2081E8683043F7E78048C078012848
:1091600000D0002070477D4810B5C07801282BD072
:109170000020FCF7A2F80120FFF7D4FF764C603CFA
:1091800020784006400F1FD100F3A4FA734A8032C2
:109190005164106422005032D36B926B801A994153
:1091A000A16AE26A401A521A824200DB1000626829
:1091B000511A814200DC0800216C081870492064B3
:1091C000884200DD0100216410BD402010B5F9F790
:1091D00042FC002807D06048008B000A02D0032020
:1091E00013F00BFE10BD6749002008606649088037
:1091F000032013F002FE032013F054FB10BD564968
:1092000010B560390A6D82420DD1002008650878DA
:10921000012801D0022807D14F480121890201838A
:10922000222013F03FFB10BDFFF79DFF4B490120AB
:10923000C87010BD484910B560394A6D0F78813348
:1092400001000000708F000000040000FA5090F14F
:10925000824219D10020464A48650320D070087820
:109260004006400F10D041480121890204006034BB
:109270000183A06A002804D102F067FDA062FCF718
:10928000F1FA222013F018FB10BD70B5374E603E86
:1092900030784006400F24D13548C078022820D1CC
:1092A000324C0821200070380C22615682569142BF
:1092B00017DA32F057FB050008F028FB00280DD024
:1092C000207A401C20723178022901D0082905D16A
:1092D00000F30AFA254A103A51631063280032F06D
:1092E00045FB70BD10B5F9F78CFF002806D02C485F
:1092F000007C00280AD0062808D005E01C48C07869
:10930000002803D0042801D0012010BD002010BD8A
:1093100070B50D00154C603CA16D814207D1002055
:10932000A06520784006400F02D0FFF758FF70BDBF
:1093300013F078FD0028FAD00221280001F051FD39
:109340000028F4D0FFF7CEFF0028F0D02078074C9B
:109350006034042826D1FFF798FF606A0028E6D021
:109360000021280011F07CFB70BD00001062040099
:10937000603C04001027000050C30000204E000095
:109380006EBE0000983A0000B80B000064B901C03E
:10939000009000906079FEFF14070004A00600040E
:1093A000904704000828DFD108F06CFA002802D0AA
:1093B000FFF76BFF70BD606A0028FBD0280011F03A
:1093C0006EFB70BDF94870B50024007812F3FAFD09
:1093D0000500092012F3F6FD4300181880088542A5
:1093E00000D20124F1482038C07F012800D901248F
:1093F000200070BDF8B50027EC4AED4CE03AD16D85
:109400002600803E814275D1EA4BD868042188430A
:10941000D8601000C7655030C36C826CC16D806D20
:10942000851A306B9941401C3063E91725606160F3
:10943000A268E368A81A994103D261682068E160D4
:10944000A0602269206863696168121A8B4103D2A7
:1094500061682068616120612268206A6368616ACE
:109460008018594161622062326B3B0011F376EA49
:10947000CE4FE161E03FA061786C7D22D2003C00DC
:10948000811A0A23C034A94227DA79789200890028
:10949000C9198C468968891AA94210DA607F0028A8
:1094A00002D0401E60774BE063777069002847D197
:1094B000B562706A401C70620120A06140E0637771
:1094C000F169BD4A40186146786489688918884204
:1094D00000DB08007864F06232E0F1698C46411AE2
:1094E0008A1AAA422CD96377227F002A03D0521EFF
:1094F000227722E03BE07A78AF4B9200D219926853
:10950000D218904205D1B1696246891A4018786430
:1095100000E07964796CFF20F530814200DD0800BD
:109520007864FFF74FFF002805D0A448796C81428A
:1095300000DD08007864306A2077786CF06201E022
:10954000306A20777878002803D0022801D00328D9
:1095500004D1E06A002801D098487864B86D0028EA
:1095600002D1706B401C7063252013F0A5F9F8BD83
:1095700010B58E4CE03CE06D00F397FC0020E065F8
:1095800010BD8A4970B5E0390A6E824220D10026AA
:109590000E66C86D00281BD00C005034A26E206FE0
:1095A000E36E616F851A994100F39EF8A26CE36C3B
:1095B000801A9941002D08DCFF22F532801AB14152
:1095C00003D308F0A9FB002803D0272013F074F977
:1095D00070BDFFF7CDFF00210800FFF70BFF70BD46
:1095E00010B5724CE03C606D00F35FFC00206065DC
:1095F00010BD6E4910B5E0394A6E824217D1002085
:109600004866486D002812D008005030C36F826F42
:10961000803003C8801A9941002805DC68486949F0
:1096200000680968884203D9282013F045F910BD65
:10963000FFF7D6FF00210800FFF706FE10BDF7B5C3
:1096400082B01400594EE03E7068401868E0A54EA4
:10965000010000006C930000000400004595B54235
:109660007D218002C90012F3F6E80700002505F30A
:1096700030FE3178380010290AD1717889008919B3
:109680008969002904D00D00002C03D140190AE09B
:10969000002C08D071684919A14204D37D21A00291
:1096A000C90012F3D8E80022454B009202004B4853
:1096B0000299883BFCF7BEFC00F320F8414A803A4F
:1096C000D167906705B0F0BD70B532F055F93C4DEB
:1096D0000600E03D286D0024002802D000F3EFFBD7
:1096E0002C65686D002802D000F3E9FB6C65E96D1C
:1096F000080002D000F3E3FBEC65286E002802D0DE
:1097000000F3DDFB2C66686E002802D000F3D7FB67
:109710006C66300032F034F970BD70B532F02CF95F
:1097200005001DF0A3F9040007D02D4800218A0090
:109730008258491CA41A0929F9DD280032F020F9C1
:1097400003F0F6F8002815D02648016940698142E7
:1097500010D1002C0ED1002033F036FA002809D1A8
:1097600033F032FA002805D11F480078002801D1D3
:10977000012400E0002408F073FC012C01D1012831
:1097800007D11A480068002803D1194C2078002816
:1097900003D1192013F09AF870BD012002F0B6F938
:1097A00020781449401E2070FF20F53010F0E2FAB6
:1097B00070BD0A6882421FD100200860ADE700003A
:1097C00090620400E03C04000090009048F4FFFF29
:1097D00010270000C8050004C405000431900000F3
:1097E000F40003C000A000800C1800041806000458
:1097F000B7050004BF94000070477CB5040005F372
:1098000068FD05000E00684615F0CEFA0098019933
:10981000421BB1410B00E117121B8B4101DA012001
:109820007CBD00207CBDF0B501250024F948FA4F2D
:10983000017885B04806420FF648002A40787ED06D
:10984000F44B1E00726CE036012846D110292FD14E
:10985000FFF254FF3A008032D36A926A801A99412B
:1098600003910290F9F709FC002808D0F9F7E5FB0D
:10987000002804D1E749BA898878904279D3E6482C
:1098800003998030436B026B0298801A994109D387
:10989000E1488030C16A806A6140084302D0F878AC
:1098A000012878D1DB4A9470D0688FE0080096E0F8
:1098B000D84B402910D19C70D8681900801A3039D3
:1098C000D862096A884200DC0800D449D86288421C
:1098D00000DA0100D962DC70A8E0002872D1F9F743
:1098E00089FB002804D0CB49FA898878904240D37C
:1098F000FFF204FFC84A8032D36A926A801A994103
:1099000003910290F9F74AFB002845D0C148C24AAA
:109910004168926B406C891A081ABE493039096A4D
:10992000814200DB08000190B07812F355FB07007C
:10993000092012F351FB874205D8B74800E078E0D0
:10994000018AB448817015F09FFEB34FF96B8842CD
:109950000AD30198FFF751FF002805D0AD48847065
:10996000C470019956E004E0AA493A8A8878904286
:1099700003D2401C8870CD7058E04A6C8868801A09
:10998000A44AC862303A126A904200DC1000C862F1
:109990008C70CC704AE012E09F4803998030C36B12
:1099A000826B0298801A99410DD39B488030C16A1E
:1099B000806A6140084306D0F878012803D09548B2
:1099C00081781EE00EE0934A94709068516C401AC2
:1099D0009049D0623039096A884200DC66E7D0627B
:1099E000D47023E0022819D1F9F7EEFA002803D148
:1099F000F9F7DFFA00280FD086483A8A8178914239
:109A000003D2491C8170C57010E08470C470426C30
:109A10000169891AC16209E07E48F6E77D49032899
:109A200004D18C70CC704869801AC8620A207470A6
:109A300010E0784E01281BD1F9F71FFB00280BD04E
:109A4000F9F7FBFA002807D1B0787989884203D268
:109A5000401CF570B0703DE0B470F068EF4FE3A3C8
:109A6000010000006897000000040000164F662EF9
:109A7000B062B26B316B53009A188918401AF062C9
:109A8000F47031E0F9F7C0FA002802D0F5703464C0
:109A90002AE0F9F78DFA002803D063483038006ACD
:109AA00000E0B068316C604F431AB362303F7268B7
:109AB000BF6AD21B9A4200DC1300B362B76B9C46AC
:109AC000326B7B00DB19D21863469A1A564BF2624E
:109AD000303B1B6A9A4202DA081AF57003E06246CC
:109AE000101A0818F47030644F48C078F4E510B5C7
:109AF00010F02DFD002801D0012010BD10F03DFD1B
:109B0000002801D0022010BD4748C03080690028DD
:109B100020D1454830380088042813D0102813D1AC
:109B20004148407801280DD1F9F7BCFA002809D046
:109B300001208002FAF765FB01204002FAF761FB81
:109B4000402010BD102010BD10F0D1FF002801D022
:109B5000082010BD042010BD33483021303810B526
:109B600011F3CEE9FF213048113111F3CAE92E4833
:109B70001021303801802F4941612F498160002137
:109B8000418081802D4AC18082612D4AC2602D4A68
:109B90007D23C261DB002C4A036202612B4A4262D0
:109BA0005A00826202000124203214730324547389
:109BB0001E4AC385F030D1708161126A02770A2291
:109BC00081774277C82242638163403041602049F7
:109BD000016010BD10B501F06EF8002805D0F9F74E
:109BE000DCF9002801D1012010BD002010BD19486A
:109BF0000021C1607047174800218160704710B58F
:109C0000FF24CC340470240A447006248470002499
:109C1000C47001714471110A8271C171190A037211
:109C200041720A2010BD0000B0610400603C0400D5
:109C30003C730000204E00001027102750C3000086
:109C4000307510275CC100004E70F22B941100009B
:109C5000F0550000B06204003EB504006846FFF70E
:109C6000CEFF0300762120006A4608F0F9FB3EBDD6
:109C700038B5FF4C6078012803D12078402822D0E5
:109C80000AE0FB49C031C96A002803D0022801D08C
:109C9000032801D1002916D1F648006EE064606EF9
:109CA00000F317F9F24B08220092F348E26C643398
:109CB0000021FCF7C9F9FFF22BFDED4A5032D167C4
:109CC0009067803203C238BDF8B5FFF221FDE84A43
:109CD0005032536C126C861A99410D00F9F768F9ED
:109CE000002814D1E2494878012802D10878402898
:109CF0000DD0E048006EC864CC6A4000E317C1177D
:109D000080196941001B994101D20120F8BD002052
:109D1000F8BD38B5D64C6078012803D120784028AA
:109D200022D00AE0D249C031C96A002803D00228F3
:109D300001D0032801D1002916D1CE48C06DA064FE
:109D4000206E00F3C6F8CA4B08220092CB48A26CE2
:109D500060330021FCF778F9FFF2DAFCC44A503294
:109D60009066D1665167106738BDF8B5FFF2D0FC38
:109D7000BF4ABF4C5032D36C926C861A60789941BE
:109D80000D00012811D0F9F713F900280DD1B948B9
:109D9000C06DA064646C4000E317C117801969416D
:109DA000001B994101D20120F8BD0020F8BD38B553
:109DB000AF4C606D00F38DF8B148C16804221143C7
:109DC000C160082223000092AE48E26A54330021A9
:109DD000FCF73AF9FFF29CFC220050325164106407
:109DE00038BD10B5A24CC034E06B002810D0A1489B
:109DF000406F00F36EF8E06B00F36BF80021200079
:109E00004030E1634160A04901600420FBF773FA30
:109E100008E7F8B5002036F0E9FB0600FF219B4873
:109E200000222D3111F358FD050056D00220287371
:109E3000C0202C182881A078F321800880000840D9
:109E400008300007000F4030A070E078012108437F
:109E5000F1210840102108439F210840E070F120C3
:109E60008000311806220E00A01D10F3650E24722A
:109E700001000000649B000000040000E220139A2F
:109E8000AEEF2000062231000C3011F312E8200062
:109E900006223100123010F3A2EF002020801C2097
:109EA0002E1828818421300011F334E83700172060
:109EB0006037346778777B48A0800920B070002035
:109EC00036F09EFB686178480079800607D4B07848
:109ED000002804D0B068012189070843B060082039
:109EE000152138770902280007F052FB0120F8BD40
:109EF0006549496F814200D195E77047614938B59E
:109F0000C031C96B814220D1684C6068002815D0EF
:109F10000420FBF788F9664820605B48406FFFF239
:109F2000E2FF0822009220687D210901564B421A67
:109F3000604800217433FCF791F804E00420FBF73B
:109F4000E4F95648206000F001F838BD38B5F9F75B
:109F500070F8002829D0F9F735F8002825D1F9F74D
:109F600026F8002821D1F9F76AF900281DD100F060
:109F70001FFF012819D123F0D2FB022815D04B4C2A
:109F800001206168002900D0002060604748403807
:109F9000C06BFFF2A8FF454B08220092464822689A
:109FA0001B1F0021FCF75AF838BDFFF724FF38BD0E
:109FB00010B53E4C403C206B002809D0FFF293FFC7
:109FC00000202063A063C82060630320FBF79DF995
:109FD00032E6F3B5502087B00390029000F0E8FE1F
:109FE00001282ED1FFF79CF9002805D108983D28BB
:109FF00002D008983728F4D1224F089B38005030FF
:10A00000069098303C000126C034282B05907BD068
:10A0100018DC172B79D008DC022B05D00A2B75D061
:10A020000B2B74D0122BDCD10CE3192B70D0262B08
:10A030006FD0272BD5D1FFF7A2FE002801D0FFF764
:10A0400072FE5BE30F4D353B603511F3E4E80DEC38
:10A05000ECEBBDBDBDBDBD08EAE9BDE8BD00FFF745
:10A06000A7FFFFF773FF0848C0780428E9D0F8F786
:10A07000A9FF002826D1F9F71FF8002820D1F8F70A
:10A08000C2FF1BE0B0610400603C040013930000B9
:10A09000A392000000900090698F0000F05500002E
:10A0A000C0190004B03600002CE90004B0620400BE
:10A0B00050460000D59B0000E19B0000002801D025
:10A0C0007E7029E0F8F77EFF002803D0F8F758FFEC
:10A0D00000280AD0F8F781FF002806D1F8F788FF9A
:10A0E000002804D03878102801D1022013E0F8F7B6
:10A0F0008AFF00280ED0F9F724F800280AD0387813
:10A10000102807D1032006E04EE2EBE2E1E20FE285
:10A1100045E259E100207870FFF766FD00287DD008
:10A12000FB480778FFF7EDFCFEF75BFFF948C078C6
:10A130000028F748007848D14006400F28D000F0AA
:10A140004AFEA06A002802D101F01DFEA062079815
:10A1500003F098F800280BD0079811214901401806
:10A16000EC49027D0A71407D4871079814F003F9AB
:10A17000E84F387800280ED1F8F724FF00280AD1DC
:10A180003E70029B039A07983100FFF76FFD02E0D3
:10A19000012000F00AFEDF4F0120FE7000F069FD93
:10A1A000012005F089FDDA48417801292AD100789B
:10A1B000402827D10020FE70FBF7A7F8FF20401CA5
:10A1C0002883222012F096FB98E2B8421AD040066B
:10A1D000400F0BD07806400F14D100F0FCFDA06AB0
:10A1E00000280FD101F0CFFDA0620BE07806400FF0
:10A1F00008D0012000F0D9FDA06A002802D00598FF
:10A2000001F027FE00272F83FFF772FA00F026FDEA
:10A21000FAF7F3FF3800BE4FF86605E028E0CAE120
:10A22000B9E187E14EE20DE2FEF7BEFE3878410665
:10A23000490F02D17978FEF767FF31F0B1FB049046
:10A24000FFF705FB002853D0B248C6700020FBF78B
:10A250005CF83878012804D0022802D04006400F6C
:10A2600005D0FF20401C2883222012F043FB95E0FC
:10A27000A84DE878002835D0042833D094657B1B9E
:10A2800001000000609F000000040000B1FAC0F669
:10A29000FFF738FA00F0ECFCFAF7B9FF0026FE668B
:10A2A000079814F0A5F82878002806D028222E70E8
:10A2B000079831001300FFF7E3FC0020FBF72FF8AD
:10A2C0000020FEF761FFA06A002802D0059801F087
:10A2D000CAFDEE70A6610A20A6776077286A20770B
:10A2E000002000F0D0FC002005F0F0FC387840069B
:10A2F000400F01D0FEF79BFF8C48C1680422114338
:10A30000C16005E2FFF707FC402806D00020FAF7FD
:10A3100094FF002801D1FE660EE1834DE878012804
:10A3200005D1FFF209FA2A008032D1629062FFF271
:10A3300003FA7C4A5032D16390630020FEF724FF79
:10A340000220E8707948C16804221143C16007986F
:10A3500014F01BF838784006400F1FD0002002F0A0
:10A36000C5FAA06A002802D0059801F07CFD787833
:10A3700000280AD0022808D0032806D0012817D1C7
:10A380003878102801D0402812D1FFF724FDFFF7BC
:10A39000AFFC00280CD0FFF77FFC09E008220092F8
:10A3A000BA6A6348069B0021FBF762FEFFF713FDC4
:10A3B000387808280FD004280DD04106490F7CD0EA
:10A3C0007978002907D0022905D0032903D0012973
:10A3D00073D11028FCD1002211009EE031F0EAFA7E
:10A3E000002604903D00FE66FEF7A4FF002893D0EF
:10A3F0004D4FF878012805D1FFF29EF93A008032DE
:10A40000D1629062FFF298F9464A5032D16390636C
:10A410000020FEF7B9FE0220F8704448C16804220B
:10A420001143C160079813F0B0FF2878414F4006F0
:10A43000400F1DD0002002F059FAA06A002802D077
:10A44000059801F010FD6878002808D0022806D091
:10A45000032804D001284AD12878102847D1FFF7D3
:10A46000BAFCFFF745FC002841D0FFF715FC3EE0A1
:10A47000A86A3A68C1177B688018A862AA6B59411C
:10A48000296B53009A188918411AE9620822009230
:10A4900002002748069B0021FBF7EAFDFFF79BFC23
:10A4A000287804280AD1FEF718FF606A00281ED019
:10A4B0000798002110F0FCFA19E031E0082801D0DB
:10A4C000022819D107F006FA002802D0FEF705FF8E
:10A4D0000CE02878082801D1606A02E0022805D142
:10A4E000286F002802D0079810F001FB2E6728780B
:10A4F000082810D004280ED029784806400F0FD025
:10A500006878002807D0022805D0032803D0012846
:10A5100006D1102904D1396800220798FFF7B7F84F
:10A52000049896E0B0610400603C04000090009044
:10A53000338F0000F0010004049831F03FFA00204E
:10A5400009B0F0BD6662E3E0FFF7DCF8FAF75FFE02
:10A550000020F8663878012825D0022823D0042866
:10A5600001D008280BD100F083FBFEF72EFEFF4838
:10A57000C67000206062288B000AE4D113E0400618
:10A58000400FE0D0288B000A0DD0FBF79DF9A06AA0
:10A59000002802D101F001FCA062F448C178022930
:10A5A000D1D103219DE02E83B2E038784006400FE0
:10A5B000C9D0FEF70AFEED48C670A9E0FFF798FB88
:10A5C0000028C0D0FFF768FBA2E031F0F3F939783A
:10A5D00005004806400F3BD07878002807D00228B5
:10A5E00005D0032803D0012832D1102930D1FFF241
:10A5F000A3F8DE4CA26FE36F801A7A789941012AA2
:10A6000001D1246C08E0022A01D1A46C04E0032AE1
:10A6100001D1E46C00E0646C00260B003100201ACC
:10A62000994115D2797800208900CA1991690029C9
:10A6300000D00800796808189168441A08D0A04230
:10A6400006D300F015FB079822000021FFF71FF842
:10A65000280031F0B3F95BE00020FEF795FDA06A19
:10A66000002802D0059801F0FEFBFFF74BF800F040
:10A67000FFFAFAF7CCFD0025FD66079813F0B8FE47
:10A68000002005F023FBFFF7CAFAFFF7D8279AE36B
:10A69000010000005CA3000000040000996B454B22
:10A6A000C4FA0020FAF745FEB64AD06804210843F0
:10A6B000D0600898352802D00898362802D1B048D2
:10A6C000C1700BE0AE482900C5700278002A05D0A1
:10A6D0002822017007981300FFF7DCFA0A20A577FB
:10A6E0006077A748A561006A20771BE0A448C1787D
:10A6F000042917D10021C17014E00020FAF719FED7
:10A70000A048C16804221143C1605EE7FFF704F866
:10A7100000F0B8FAFAF785FD0020F866FFF789FA2D
:10A72000FFF783FA012015E710B5FEF70DFE0028AC
:10A7300006D0954800784006400F01D001205BE428
:10A74000002059E410B50400FEF7FEFD002813D0E8
:10A75000FFF7EAFF002811D18948C07802280DD1FF
:10A760008948092160304156012901DB002C05D0C0
:10A7700007F36AF9002801D001203DE400203BE402
:10A7800010B5FEF7E1FD002806D07D490120C9780B
:10A79000022900D000202FE401202DE410B5FEF79F
:10A7A000D3FD002810D0784800784006400F0BD029
:10A7B00002F0EFF8002807D173486030008BC11F0A
:10A7C000F93901D0012017E4002015E46E48C06E6D
:10A7D00070476D490120086770476B48406F7047AC
:10A7E00069490120486770476749002048677047FA
:10A7F00066488068704765480121816070476348FA
:10A80000C068704761480121C16070475E481038D8
:10A81000407B704710B50400FEF796FD00288ED0EF
:10A82000002C8CD1FEF292FF574A503251631063D4
:10A8300010001030417A491C417280E710B5FEF7D4
:10A8400083FD002815D0504C2078012801D0042821
:10A8500006D14D486030017A491E0172FEF747FD6E
:10A8600020784006400F04D0FEF270FF474A303A8D
:10A8700003C264E7FFB587B00D00FEF765FD002851
:10A880007DD0414F00263C002100387838310691B8
:10A89000083960340128059101D0042831D1FEF235
:10A8A00055FF0B00F96B069A05000598019003927D
:10A8B00002917A6B344800925030416B006B2A0051
:10A8C00000F05FFC607A401E607231F07DF82C4D24
:10A8D0000490E878032869D1386D002802D0FFF28F
:10A8E00016FB3E653878012806D1012040022083FE
:10A8F000222012F013F859E0FEF771FC0120E870F5
:10A9000054E0022802D0204908286BD10A98002878
:10A91000B6D002F003F8002831D107F0C9FB0128B6
:10A92000AED0FEF213FF070017480B00C16B069A6A
:10A9300005980190144803920291426B00925030A6
:10A94000416B006B3A0000F01CFC207A401E207224
:10A950000120002D00D000200D4908700998002822
:10A9600001D0002D6FD00020099031F02DF8044F58
:10A970000490F87803281DD1034D286D0AE02AE0E1
:10A98000603C040000900090B0610400B0620400DC
:10A99000B3050004002802D0FFF2B9FA2E6528782A
:10A9A0000228A2D0FEF71BFC0120F870049831F0B9
:10A9B0000FF848E0049831F00BF812F065FA00281F
:10A9C00041D0BB48006800283DD106F08DFF00282B
:10A9D00002D0FEF78CFC36E0002D34D0079810F042
:10A9E00090F830E0B34C4006400F2CD0486B0290FA
:10A9F000C517FEF2ABFE2700703F3A6B7B6B801AE7
:10AA0000029A99412B00121A8B410BD2A07F401C55
:10AA10000006000E0A28A07705D3A749086D401C40
:10AA20000865A661A67704F37CFC79653865FEF2BB
:10AA30008DFEA04AF965B865109B403A13637967AB
:10AA40005032386703C209980BB0F0BD994970B510
:10AA5000C039097815004906490F1CD0603010F341
:10AA600014EB80780009042815D00C2813D0914CE1
:10AA700020346078002808D0280011F3D5FA0600A9
:10AA8000A07811F3D1FA864200D2A5706078FF2831
:10AA900001D2401C607070BD10B5FEF72EEC2FE99E
:10AAA0000100000058A7000000040000CAB196276A
:10AAB00055FC002805D0844901206039098B012903
:10AAC00000D1002045E680487021C0380078084059
:10AAD00070477D486038008B000A0002704710B54F
:10AAE00030F07CFF30F07EFF33E6FEB5764DC03DA2
:10AAF0006878012833D12878402806D1FEF230FE4C
:10AB00002A005032536C126C04E0FEF229FE6F4AA8
:10AB1000D36F926F871A68789941800040198068D6
:10AB20000190C317686C0C00C117019AC0196141EC
:10AB3000121A8B4113D26878800040198068C117BF
:10AB4000C01BA14161494A6D521C4A65FF22F53282
:10AB5000904203DA10008A6D521C8A656864E86DC1
:10AB6000FFF2DFF9584B0822009259486A6C643BA7
:10AB70000021FBF791FAFEF2F3FD534A703A90641C
:10AB8000D164D165906507F003F9FEBD10B54E4C58
:10AB9000C03C206EFFF2C5F900202066D9E510B553
:10ABA000494CC03C606EFFF2BCF900206066D0E505
:10ABB00045492031087070474349C877704742497A
:10ABC000C8627047434A506B010C3F480904F03893
:10ABD000C08D014351633F4AC03A116B0904090C0F
:10ABE000000408431063704710B5F8F740FA0028D6
:10ABF00005D0F8F705FA002801D10120A9E50020C9
:10AC0000A7E53148C06B002800D00120704738B557
:10AC100001202D4CA16B002900D00020A063206BE7
:10AC2000FFF27FF9284B082200922B48626B3033E9
:10AC30000021FBF731FA38BD10B5234C216B81425E
:10AC40000ED1A06B002804D00320FAF70AFB23489A
:10AC500003E00320FAF777FB21486063FFF7D7FF93
:10AC600077E51948006B002800D00120704710B527
:10AC7000F8F703FB00280DD100F045F8002809D0B3
:10AC8000F8F7B3F9002805D1F8F734FA002801D114
:10AC900001205EE500205CE510B50B4CC03CA06DCA
:10ACA000002803D0FFF23DF90020A06551E50D49D1
:10ACB000064A002803D0086810670B4800E0106FB0
:10ACC000086070471806000470620400603C0400CD
:10ACD00015910000C0900090E1A8000030750000C0
:10ACE000204E0000C0A9008001000300FF4810B5FD
:10ACF0004068002805D0FEF731FB002801D1012073
:10AD000010BD002010BDF94810B50078012815D1FC
:10AD1000F8F754F9002803D1F8F772F900280DD09C
:10AD2000F8F7A5F9002803D0F8F76AF9002805D04C
:10AD300022F013FD022801D0012010BD002010BD1B
:10AD400010B5F8F79AFA002808D0F8F74EF900285D
:10AD500012D0E748007C06280ED00BE0FFF7D3FFA7
:10AD6000002809D0F8F741F9002805D0FEF7F6FAD7
:10AD7000002801D1012010BD002010BD10B5FFF743
:10AD8000C2FF002809D0F8F730F9002805D001F0FB
:10AD9000CFFD002801D0012010BD002010BD10B54E
:10ADA000FFF7B1FF002803D014F045F9002807D0C1
:10ADB00012F0A7F8002803D105F046FC002800D0C7
:10ADC000012010BD10B5FEF7C9FA002802D0FFF728
:10ADD000E1FC10BD012010BD10B5FFF77AFE10BDDB
:10ADE000C24840687047C14948607047BF48007812
:10ADF0007047BE490870704710B5FEF7AFFA0028DB
:10AE000005D0FFF760FE002801D0002010BD012012
:10AE100010BDB649002010B5486006F00CFE10BD0C
:10AE200010B5FEF79BFA002802D0FEF76AFA10BDB3
:10AE3000002000F09FFA10BD10B506F05FFD00285D
:10AE400009D100F087FA002805D1FFF7C9FC0028D6
:10AE500001D1012010BD002010BDF3B50C0081B060
:10AE600007D0022C05D0032C03D0042C01D0012CD8
:10AE700003D19E480078012814D135F0F4FB002856
:10AE800003D016F061FC00280CD00127994D9A4E92
:10AE900023007F0610F3DCE9050484070E7C99008B
:10AEA00000F090FB91E001983D21FFF74E697B791E
:10AEB0000100000054AB0000000400003EDEE393FC
:10AEC000B0F8002875D005E0032C03D101982621A5
:10AED000FFF7A7F8FFF73EFF0124A402002837D0B0
:10AEE000874801214160019813F06DFA00F039FBA9
:10AEF000012006F0EEF80FF0C6FD00280DD0E86B3B
:10AF000008210843E8632000F9F7BAF92000F9F7AF
:10AF1000AAF9E86BF721884306E00FF01AFE002833
:10AF200003D0E86BFF210843E863B0683843B060A2
:10AF30000FF0A9FD002808D00FF03BFB00284ED1F0
:10AF400000F014FC00284AD130E0FFF773FF46E020
:10AF5000FEF70EFA002818D106F0BBF8E86B000ADD
:10AF60000002E863B068B843B0602000F9F783F9E5
:10AF7000FFF732FEFFF757FF6548016858308142FE
:10AF80002DD1232011F0DEFC29E0012006F0A1F8EC
:10AF9000E86B000A0002E863B068B843B060FFF7EE
:10AFA0001BFED2E7FFF7ACFE002818D0FFF73BFFEF
:10AFB00015E015E000F02DFB019813F037FA019829
:10AFC0000221FFF72EF8FFF72EFF002006F081F890
:10AFD000E86B000A0002E863B068B843B060012083
:10AFE000FEBD0FB40020F0B58BB035F031FB0390FF
:10AFF00001A8FAF7C0FEF8F74AF910AB197E18ABB2
:10B000000A911E7F10AB1F7819790991D97818AB76
:10B01000089119790791197A0691D97910AB0591A0
:10B020005C7818AB5D79002842D022F0A0FB0228A2
:10B0300070D0AC4205D0012D01D12A20ABE02B20ED
:10B04000A9E0002F02D0099800281BD008980028FA
:10B050000ED1002C0CD10798002802D006980028A9
:10B0600004D00598002801D1002D01D02D2092E0B8
:10B07000002F02D00998002804D00898002801D198
:10B08000002C0CD00798002802D00698002806D083
:10B090000598002803D1002D01D12E207BE00A98CD
:10B0A000B0427AD0012E01D1302074E0312072E01C
:10B0B0000398002871D01248007801286DD122F041
:10B0C00056FB13495831022804914ED01048049978
:10B0D0000068884249D1002F02D0099800281DD06D
:10B0E000089800281AD1002C18D10798002802D0FF
:10B0F0000698002810D0059800280DD1002D0AE0F0
:10B100004802000490470400C0A200800090009014
:10B1100080D400040AE00AD024203CE0AC4206D0EF
:10B12000012C3AD103980221FFF7A1FE35E0002F50
:10B1300002D00998002804D00898002801D1002CDA
:10B140000AD00798002802D00698002804D0059855
:10B15000002801D1002DE5D00A98002802D1002E48
:10B16000E0D11AE0002EDDD017E032480078012847
:10B1700013D122F0FCFA02280FD02F48016804985E
:10B1800081420AD00A98002802D1002E05D001E0A1
:10B19000002E02D1032011F0D5FB01A8FAF708FE1A
:10B1A0000BB0F0BC08BC04B01847F8B506AC171AD1
:10B1B00070CC8B411900002F01DC0020F8BDA742A4
:10B1C00000D92700286803214000C0190FF390EF31
:10B1D0003900B842286000DB0100B84200DC0700FB
:10B1E000C81BB04200D93000099909684900081805
:10B1F00003210FF37EEF099908600120F8BD262096
:10B2000010B511F09FFB10BD10B51FF087FD094C64
:10B21000002803D120F0E4F8002801D0002000E04D
:10B220000120207000F097F900F0D6F9FEF7C6FC77
:10B2300010BD00004802000480D4000410B530F0B6
:10B24000D7FBFF490A69002A03D030F0D5FB012063
:10B2500010BD01220A6130F0CFFB002010BDF94B78
:10B26000586B020CF8481204C1680A435A634268DA
:10B2700009040A43F349C0390A6301686439016269
:10B28000002181621E2281614262C1617047EC49E6
:10B2900010B54A69824215D1002008704861FFF755
:10B2A000DEFFEA480068002801D0172008E00FF010
:10B2B000EAFB002803D10FF04CFC00285D6D06F678
:10B2C0000100000050AF0000000400006D0430FFDA
:10B2D00002D0212011F040FB10BD38B5DD4C606973
:10B2E000FEF233FE082223000092DE48A26900210C
:10B2F0001433FAF7E5FE38BD70B530F083FB060075
:10B30000D94801694069814201D0012400E000244C
:10B31000D04D2878697808431BD0300030F076FB98
:10B320006878002813D0002C0CD0686A0722401CD3
:10B330006862CE480121006831F07DFC212011F0C7
:10B340000BFB04E0A86A401CA8620120A870012041
:10B3500070BD06F397FB002808D1300030F056FB93
:10B36000E86A401CE862FFF7B8FFF0E72878401C65
:10B370002870300030F04AFB002070BD10B530F06E
:10B3800041FBB4490A7849690A4303D030F03EFBD7
:10B39000012010BD30F03AFB002010BD10B50400B4
:10B3A00006F0C0FA002822D0FFF7E8FF00281ED1DF
:10B3B000FFF7B0FC002803D00FF0D5FB002802D126
:10B3C000002C14D008E0002C06D1FFF795FF0028D0
:10B3D0000DD1FFF782FF08E09E490020C870FFF7FB
:10B3E00037FF002803D1FFF744FF06F0DFFA10BD56
:10B3F00098498A68824204D100208860086101204F
:10B40000CCE7704738B5934CA068FEF29EFD082249
:10B41000230000929648E26800210833FAF750FEB4
:10B4200038BD10B58B4CA068FEF28FFD0020A060E7
:10B4300010BD10B5874C6069FEF287FD0020606189
:10B4400010BDFEB50A21040001AA08F07AFB814F65
:10B4500005000026002843D0112040012018408A12
:10B460000321890308430199096F8880200006F0B1
:10B470009FF9010001987F4A817000927E4A1279FB
:10B48000920606D4002904D0816801229207114354
:10B490008160006F1022C178784C1143C17002E0C6
:10B4A0000220F9F795FF06F007FB002801D1641E82
:10B4B000F6D2FFF712FF012078700099280006F0FD
:10B4C00099F800280AD1280010F318FA30F09AFAF7
:10B4D0003E707E7030F09AFA0020FEBD0120FEBD65
:10B4E00030F090FA3E70F5E770B506000C001500DC
:10B4F000002B38D00FF037FB002834D001F02CFAA5
:10B50000002830D106F0F2FD01282CD00120002CBB
:10B5100000D000205A490870FFF77CFC012808D1B0
:10B52000FFF787FF30F06EFA4A4A0021117030F0C1
:10B530006DFA11F0C7FC002815D0494800680028B2
:10B5400011D106F0EFF9002803D00020FFF726FF05
:10B5500008E0002C07D04B480078002803D13000C9
:10B560000FF0EDFA0025280070BD4748C16B474A2F
:10B570001143C16370477CB5F7F74BFD3D4E444D19
:10B58000344CE03600280AD0694601A8F7F7DCFD04
:10B5900000990198884204D8606B401C6063009653
:10B5A00001952E4D0198E968814203D12969009ADD
:10B5B00091421AD0E8600099421A2A604B22D200C8
:10B5C00029618918334A8218914200D811006960B4
:10B5D000216A401AA8600FF0C6FA002803D0A868B4
:10B5E000FF38F538A860FFF744FE7CBD70B530F039
:10B5F00009FA0600FFF71DFF164C00257D20257077
:10B60000C00065702062FFF7B6FF06F038F9FFF75B
:10B6100008FF11482561416B420611434163300028
:10B6200030F0F4F970BD10B5FDF7ACFE002837D14D
:10B63000FFF7F0FB012833D1FFF7FBFE30F0E2F912
:10B6400005494A6B4B061A434A63024900220A70B5
:10B65000024921E050020004C0900090B82F00047D
:10B660001806000423AF000000A0008014080004A6
:10B6700071B00000020400002CE900047017000003
:10B68000B3050004B4050004C0A2008000020080DD
:10B69000A60E000048F4FFFF8A61CA6130F0B6F9D7
:10B6A00010BDF94AD368181A401A010410008068C6
:10B6B000090C5368F5490204086B120C000C0004D5
:10B6C000104308637047F0B5040085B044D8B97CD6
:10B6D000010000004CB3000000040000D2C1154C72
:10B6E000FFF7A2FB012853D101F040F900284FD108
:10B6F0000FF0DDF9002801D0FFF7A5FE0FF0D7F914
:10B70000002807D10FF039FA00282CD04034207ED1
:10B71000C00628D5E14C206A0490A56AFEF23EF8E6
:10B720002368220007000E002832590810000093F9
:10B73000083801AB07C33300E169A0693A00FFF79D
:10B7400048FD606A002808D0A26A216A8A18049914
:10B7500049198A4201DA401E04E0A16A206AFFF713
:10B76000AAFF1E20606230F057F9CD490400C031B5
:10B77000486B4A06104348630FF099F9002804D03B
:10B78000C8490020087006F01BF9200030F048F985
:10B7900005B0F0BDC34800797047F8B5040000203B
:10B7A00034F06AFF0500F7F786FD00285CD1002D14
:10B7B0005AD0A868C00457D501F0D8F8002853D152
:10B7C000FFF732FB01284FD121F0E5FF02284BD0D3
:10B7D000F7F729FC002847D030F01EF90090200030
:10B7E000B049B14CAE4EB14F11D0012008710020CC
:10B7F00005F083FCE06B000A0002E063B068B84328
:10B80000B060600DF8F74BFDFFF7FAF929E0002072
:10B8100008710120FFF705FB280012F0E8FDFFF793
:10B82000B4FE012005F069FC0FF041F9002807D0B3
:10B83000E06B08210843E063E06BF721884306E0F2
:10B840000FF09BF9002803D0E06BFF210843E06371
:10B85000B0683843B0600FF02AF9002801D1FFF733
:10B86000FDFA009830F0DCF8F8BD70B505008B4C9F
:10B870000026E169A0697140704008430FD0A269B9
:10B88000E3693100A81A994109D28649086B401C26
:10B890000863A269E369501BB341E361A06170BD15
:10B8A00070B504000D00FDF279FF7C4AD161906112
:10B8B0002900200035F026F8FFF7D7FF70BDF7B557
:10B8C00082B00D001600F7F7F6FC00280AD0FFF74B
:10B8D0002BFA002811D0002D7ED07C20405D072857
:10B8E0000BD80DE0286F80780007800F06D1FFF796
:10B8F00063FA002802D0FFF78FFDEDE0002DEBD0BA
:10B9000030690028E8D0286F80780007800F02286F
:10B910000BD101F02BF8002807D10FF02EF90028E9
:10B9200003D0FFF701FA00280CD1FFF745FA0028F1
:10B9300004D0286F80780007800F03D0F7F7BBFC96
:10B940000028DAD05A4807685A48007800020743AE
:10B9500030F062F801905748346800781434810060
:10B9600055484058010604D00006000E001F384319
:10B9700001E0FC2038430068A0427ED1F7F79BFC31
:10B98000002833D00020F07560880007000F0128E0
:10B9900031D03168606860318A7F801C521E120687
:10B9A000120E8A7775D04178090714D401780A07F6
:10B9B000920F022A02D1090908290CD03F49096BCC
:10B9C00001220909D20289180A0161680B8B1B0741
:10B9D0001B0F13430B8300E076E0417808221143EC
:10B9E000417002982100F7F70AFD04E030686030EA
:10B9F000817F491E817730686030807F002848D081
:10BA0000F07D002845D1FC20384306683800042129
:10BA10000843FC2239002FF05EEC3E60254828499F
:10BA2000007880000A58521C0A5026490A58121DF4
:10BA30000A50F7F740FC002804D160680822C1785A
:10BA40001143C17001202070F7F735FC002804D0A5
:10BA5000F7F74BFCF7F7CAFE16E01149C031486B07
:10BA60004A0610434863FFF7EEFC0E4800210170C0
:10BA7000286F80780007800F00E00AE001D10120E4
:10BA800000E00020FFF794FC01982FF0C9FF01208F
:10BA90007EE601982FF0C4FF1EE00000B82F0004DE
:10BAA0000090009050020004C0A20080000000023C
:10BAB00000A0008058B901C01C0103C0C0A60080CE
:10BAC000F40003C0440103C027480078002803D0D5
:10BAD00002983100FFF7E4FE002059E60D18C7B1C7
:10BAE0000100000048B7000000040000811BC620D0
:10BAF00010B5040037290CD007DC21290DD03529D9
:10BB000001D0362908D1012004E0382901D0392993
:10BB100002D10020FFF74BFE10BD00F031FF0028DE
:10BB200026D10EF0CEFF002812D014494878002804
:10BB300007D0C869022804D2401CC861FFF7E1FBA6
:10BB400010BD0020C861010020000EF0EDFF10BD07
:10BB50000FF01DF80028FAD005F0F8FE002803D0F9
:10BB60000020FFF72FFC10BD20000EF0FCFF10BDE1
:10BB70000120F6E701490020487070475002000498
:10BB8000002800D00120FC4988607047FA48C0684E
:10BB90007047002800D00120F74908607047F64838
:10BBA000406870470020704710B541690979012944
:10BBB00003D100212AF019F810BD05F03CFC10BD9E
:10BBC0000100EE4810B5C069072231F048F80020A6
:10BBD00010BDF7B584B000242500EA480194E84E72
:10BBE00042690499430619430A434261E64BD96806
:10BBF00004229143D960E34980310A6907231B0479
:10BC00001A430A61DF4BC033196808229143196057
:10BC1000DE4B196802229143196080690290FDF29F
:10BC2000C7FD0F0000902DE0D6486D1C8069029082
:10BC3000D74800697F214905084003D00121490503
:10BC4000411A03D1864201D1641C00E000240600A1
:10BC5000FDF2AEFD009A0023801ACE4AB941121AB5
:10BC60008B410FD2CA480169C448C94A8160FF218B
:10BC70003331803A1161C6498031C968C160022000
:10BC8000019002E006988442CED3FDF291FD009A25
:10BC9000801ABA4AB94151661066029904988843DD
:10BCA00004D00198002801D101200190B748016813
:10BCB000022211430160B349C031086808221043D1
:10BCC0000860B04880300169072212049143016185
:10BCD000AD49C86804221043C86005980560019802
:10BCE00007B0F0BDF8B50700FDF262FD0C00009052
:10BCF0001DF00EF8A14D0026002804D0A6490888A2
:10BD0000B843088003E0A549380002F33AF9FDF290
:10BD10004FFD009A801AA1410B000400686D3100AC
:10BD2000001B994100D36C6D6C65F8BDF1B584B012
:10BD3000924C206C401C20641CF0EAFF002806D0C6
:10BD40009549049A08881043088005B0F0BDFDF2BB
:10BD50002FFD02908D480D004038C66A9049C1629F
:10BD6000884FB869854901908E481E223431FFF70B
:10BD700030FF022803D16068401C606004E00128A5
:10BD800002D1206D401C206580484038C662B869E9
:10BD9000E063FDF20DFD029AE76C861AA9410D00E1
:10BDA0007A1C0020A06CE16C00234843002180191C
:10BDB00069410EF338EEA064E06C401CE064606CF6
:10BDC0000021801BA94100D3666C6664606BA16B87
:10BDD000884201D9606B00E0A06BA063049A0199CE
:10BDE00070481143884301D0FFF77CFF226D616CDE
:10BDF00011202BF0D1FFA8E76B480088002804D061
:10BE00006A4901200978042900D0002070472020C9
:10BE1000D6E6F8B500242600584D2869002801D13F
:10BE20002000F8BD2FF002FE0090E86A01210B000F
:10BE3000002800D00023002001218140EA6A0F0081
:10BE4000174202D10C000A43EA62401C002C01D1C7
:10BE50001F28F1DD002B12D0FEF798FC002807D038
:10BE600005F03EFE002800D001263000FEF7CFFE90
:10BE7000002E04D103F3C1FBFF20FFF757FF00980A
:10BE80002FF0D8FDCCE7F8B500243C4D28690028F8
:10BE900001D12000F8BD2FF0C9FD0090286B0127CB
:10BEA0003B00002800D000230020390081402A6B8D
:10BEB0000E00164202D10C000A432A63401C002CDB
:10BEC00001D11F28F1DD002B05D003F396FB0320E1
:10BED0000002FFF72BFF00982FF0ACFDD9E770B5FB
:10BEE00004002FF0A3FD050024480022A722A1DAB8
:10BEF0000100000044BB0000000400007574B3940E
:10BF00000169002901D1226070BD2368C16A99438B
:10BF1000C162226007D02B48006881430FD1FF2007
:10BF2000FFF7EAFE0BE01CF0FDFE002807D1FF2022
:10BF3000FFF7E2FE03F363FB0120FFF74BFE28004F
:10BF40002FF082FD70BD70B504002FF079FD050063
:10BF50000F4800220169002901D1226070BD2368C9
:10BF6000016B9943016322600CD11CF0DBFE0028B9
:10BF700008D103200002FFF7BFFE03F340FB0220BD
:10BF8000FFF728FE28002FF05FFD70BD30B901C01B
:10BF9000880200044523010040A200800090009028
:10BFA00000A7008080A80080A08601002E3D04002C
:10BFB000FFFF0000FF7FFF7FFF030000643C0004E1
:10BFC0008D060004383D0400F8B504004669008978
:10BFD0000519FEF705FF002818D0F7F780F90028AB
:10BFE00014D1286F80780007800F0FD1200036F021
:10BFF0005CFF200005F0C8FC002803D00120FFF7FB
:10C00000EBF9F8BD200036F077FF0CE0310020009E
:10C0100000236A4633F0D6FB002802D12000FFF748
:10C02000CDFD0028EDD120000FF386FCF8BD38B51A
:10C03000E04C606A30F028FEE0690522002130F013
:10C0400018FEDD4805220068002130F012FE02E0F3
:10C0500000980FF371FC206A04220023694630F037
:10C0600004FE0F28F4D1D54800250570D4481221CC
:10C070000EF3A0EFD34865700560002038BD70B5A1
:10C080000E00A8214143D04800250C18A088E18863
:10C09000814201D1012070BD810061188968316041
:10C0A0002621401C0FF33AECA1808034206A401E08
:10C0B000206230681C3844696179022905D1290061
:10C0C00013F0D5FD20000BF0F8FD002070BDF8B591
:10C0D00004000D0040791600022815D120000CF054
:10C0E0005DFC012810D1300002211C3813F0BFFD87
:10C0F0000700012120000CF0C4F8012F04D1AD4944
:10C10000886D401C88650BE0A8216943AE480C1877
:10C11000E5882621681C0FF302ECA088884201D133
:10C120000120F8BDA80020188660E1808034206AD4
:10C13000401C20620020F8BDA348A82110B50EF3D2
:10C140003AEF9C490020886210BD001F10B504061C
:10C15000240E042C13D2A82060439B494018A82128
:10C160000EF328EF934A0120916AA0400843102162
:10C17000A1400143FF20401CA0408143916210BDBB
:10C18000F8B5041F042C24D22FF05AFC0600894D68
:10C19000FF20401CA96AA04008420AD003E0009892
:10C1A0001C3831F056FA20006946FFF768FF002876
:10C1B000F5D0FF211231A86AA1408843A862A820C7
:10C1C000604381494018A8210EF3F4EE30002FF0AF
:10C1D0003BFCF8BDF8B5041F042C25D22FF030FC31
:10C1E0000600744DFF20401CA96AA04008420BD0F5
:10C1F00004E0009800211C382FF010FC2000694654
:10C20000FFF73DFF0028F4D0FF211231A86AA140BA
:10C210008843A862A82060436B494018A8210EF308
:10C22000CAEE30002FF010FCF8BDF8B50024250050
:10C23000654EFF277F1CA82060435E4935543800B7
:10C24000896AA040084202D00120FFF7C3FC641CA9
:10C25000042CF0DBF8BDF1B582B02FF0F1FB0090BB
:10C260005A495B4837F04EE8FFF7DDFD0190029830
:10C27000FCF764FE574F0024260001202506386095
:10C280002D0E029928001DF062FB029928001DF076
:10C29000BFFC641C042C3E60EFDB01A8FFF729FE05
:10C2A00000982FF0D1FBFEBDF7B582B00025060047
:10C2B00015F015F8002801D1002050E5002168464E
:10C2C00021F03EFAFF212D31300007F039FC040047
:10C2D0001DD01C202700C0372518208120213800C0
:10C2E0000EF392EEB878F321800880000840001D1C
:10C2F0000007000FB030B8706B462F67D0A02C003D
:10C300000100000040BF00000004000026AE60F8FD
:10C3100018788007800F012801D1052000E0002057
:10C32000A870270041D0314801902C6F03992171EA
:10C33000090A6171002121706170E07806224108CC
:10C340004900FD2001402A48E1703118A01D0EF37C
:10C35000A0EDF12080003118200006220C300EF3F1
:10C3600098EDCC2060357E6168770498022402281D
:10C3700019D004DC002807D0012816D104E00328D6
:10C3800004D0FF2811D10820287700E02C770199EC
:10C39000380005F057F9002807D0164908692043EE
:10C3A00008610120E5E40320EEE738000FF3CEFA40
:10C3B0008CE711480088002805D01048017803292F
:10C3C00001D10421017070478802000414080004A0
:10C3D0000C18000468CB000400080004C8C800045E
:10C3E0001111FFFFBBBBBBBB343C040002150000B6
:10C3F00029020000C0A20080643C00048D060004F5
:10C40000FF4840787047FE4948707047FC4900205B
:10C4100088607047FA490020C8607047F7B582B05D
:10C420000600F74D1700E86800285FD10398FEF773
:10C43000CFF900285AD0FF21F24800222D310FF306
:10C44000AFFA040052D001200221E8602173666136
:10C45000617B0143EC486173A061C0202081112001
:10C4600040013018428AE94800920068320003799E
:10C47000F12080003118AC32200001F304FC01905F
:10C480001C2025182081842128000EF39EED280011
:10C49000390060300700417701982867300005F0C7
:10C4A000AFF9DB4EA870FEF76AFC002800D1D94E28
:10C4B000D9480079800607D4A878002804D0A86855
:10C4C000012189070843A860FCF784FF002802D0F7
:10C4D000FEF7E2F900E0032038773100200005F094
:10C4E000B1F8002805D120000FF330FA002005B084
:10C4F000F0BD0398FEF7D4F90120F8E7FFB589B045
:10C500000700002005900C9800281AD0BC488168CC
:10C51000002916D0C1490A6949698A420BD041688D
:10C520000722491C4160BE480121006830F0ABFB86
:10C53000212010F039FA0DB0F0BD0120F9F7E2FB2F
:10C5400001E0FF242D342100380007F003FB050033
:10C55000F3D0288939794619F12080003C18380039
:10C56000AC300629089002D10C2006900BE0380070
:10C5700034F066F9002801D00C2000E00420069079
:10C58000387906280DD1A748089A3B180192069AD7
:10C5900002213000009401F3B3FBF0784008400022
:10C5A0000BE0089A0192089B069A02213000009441
:10C5B00001F3A6FBF07801210843F070F078EF2139
:10C5C00008400A992C00C907C90E0843F070FF20E3
:10C5D000C01C3071000A70710020307070701C2017
:10C5E000288102202900287330311C3404918421D1
:10C5F00020000EF3EAEC21006031139807917728B0
:10C60000487701D0782804D1A06801214906084361
:10C61000A06026670C9800280AD00120C007A060FF
:10C62000774801218160687B084368737E48A86170
:10C630000020208006980C281FD10B99380034F078
:10C640000BF941072078490FC008C0000843410793
:10C650002070490F380034F02AFA0101206F028B54
:10C660001207120F0A430283206F017E0909090194
:10C67000017620789F21084020700B9A2100380015
:10C68000002334F018F91298002827D1FEF792F809
:10C69000002818D0079908200877002138002AF0D0
:10C6A0006FFAA0700A99002914D00FF303FD060059
:10C6B00009200FF3FFFC864201D90920A070A07861
:10C6C000FEF7B2FA06E0079809210177380005F075
:10C6D00097F823E001200003059021E000213800B5
:10C6E0002AF04EFA0328A0701AD94B480079C006E8
:10C6F00003D53420C05DFE280CD0787902280FD1F4
:10C700000F2080013818806A0521C901D21C16A6A5
:10C71000010000003CC30000000400002457B8EEF4
:10C7200040180078000705D50321380004F0DEFF2B
:10C73000A070D9E70798407F772803D0782801D0E8
:10C74000412804D10520A07001200003059037483E
:10C750000079800607D4A078002804D0A0680121C1
:10C7600089070843A06004990598C861390028002A
:10C77000002303AA33F03AF8012800D1E5E6FEF7DA
:10C7800075FB002812D0129800280FD0280036F030
:10C79000A0FB0599280005F026F9002802D0FEF735
:10C7A00085FBD2E6280036F0BBFB05E005992800A2
:10C7B00004F052FF0028F4D1280018F02DFC2800C6
:10C7C0000FF3CEF8C1E6FFB5FF212D31060085B08D
:10C7D00007F0CAF907007ED01748317934180129CB
:10C7E00002D07079022804D12100300034F024F8FE
:10C7F00002E0300034F02EF86B460390187EF321EF
:10C800000840083018760399002919D00007000F56
:10C81000C03018E040B901C0C019000445C0000094
:10C82000C000000402040000021400002CE900040F
:10C8300000A0008014080004290200003DC0000090
:10C840000007000F40306B46187638893200C51952
:10C85000F1208000AC32311801920091187E0490D2
:10C8600002090007810F2300280001F353FAFF207B
:10C87000C01C2871000A687104986B46A870587E25
:10C88000E870707902280DD1022130000AF0CBFD4A
:10C89000E9788A06D20F1043C007DF22800E1140CC
:10C8A0000143E9701C203C1838813800256708993D
:10C8B0007C3041770E9901770398002835D06B467C
:10C8C000988B20807079032820D1300018F0BFFAAF
:10C8D0000100300000E03EE033F0C8FF410720785F
:10C8E000490FC008C000084341072070490F3000BD
:10C8F00034F0E7F80101206F028B1207120F0A4390
:10C90000028320789F21084020700EE0A64A5088BC
:10C910000101401C5080687E2A7E000210430007FF
:10C92000000F08432876000A6876002130002AF0BC
:10C9300031F9A0700898382810D00898312812D002
:10C9400031003800002302AA32F050FF01280AD13A
:10C950000298002811D0012009B0F0BD9349086960
:10C960000222104308610021380004F075FE0128FE
:10C9700003D038000EF3F4FFEDE70020ECE70200EF
:10C980008B4810B5006804210023F9F70EFA00283F
:10C9900004D10220FFF732F9002010BD012010BDA4
:10C9A00070B50400834D28680079A04201D031F0B1
:10C9B00078FF286804718048446170BD10B533F079
:10C9C0007CF8002801D1012010BD002010BD77495E
:10C9D00070B501258031096B490719D5FF2804D1AD
:10C9E000002405F0A1F9010001E001000400734BEF
:10C9F0001E1F0AE0E000C218126880190068824217
:10CA000000D00025641C012D08D18C42F2D905E02C
:10CA10006B48816AC06A814200D00025280070BD41
:10CA2000FF2010B5FFF7D3FF002801D005F076F8FE
:10CA300010BD644870B5007800284BD162480022D0
:10CA400000680821FCF2A1FE002843D1FFF7E8FFAF
:10CA500000283FD05D48FBF294FB04005B480821AE
:10CA6000FBF21EFB050059481021FBF219FB2818A8
:10CA700084422FD15648FBF284FB0400544808211D
:10CA8000FBF20EFB050052481021FBF209FB2818AF
:10CA900084421FD14F48FBF274FB04004D4808212B
:10CAA000FBF2FEFA05004B481021FBF2F9FA2818B8
:10CAB00084420FD14848FBF264FB04004648082139
:10CAC000FBF2EEFA050044481021FBF2E9FA2818BF
:10CAD000844201D0002070BD012070BD70B50120DE
:10CAE00014F0ADFE00285ED12F4C364D364E08E0D6
:10CAF0002078401C20700120FFF780F80120F9F712
:10CB00000BF928780028F3D1306800220821FCF2C4
:10CB10003CFE0028ECD102E00120F9F7AC835DB9BE
:10CB20000100000038C7000000040000778D6B8210
:10CB3000FDF8FFF77FFF0028F8D02948FBF22BFB18
:10CB4000040027480821FBF2B5FA0500244810210B
:10CB5000FBF2B0FA28188442E8D12248FBF21BFB12
:10CB6000040020480821FBF2A5FA05001D48102109
:10CB7000FBF2A0FA28188442D8D11B48FBF20BFB29
:10CB8000040019480821FBF295FA05001648102107
:10CB9000FBF290FA28188442C8D11448FBF2FBFA41
:10CBA000040012480821FBF285FA05000F48102105
:10CBB000FBF280FA28188442B8D170BD40B901C098
:10CBC000C0A20080A8020004C000000440A60080AB
:10CBD00034A9008000A000800C18000400000004AC
:10CBE0007C190004C0190004B41A0004501A00048F
:10CBF00009229201801889080E2210B50AF34DFA15
:10CC0000800010BD70B505000C0016002EF036FF38
:10CC100000212560A171E67108340A0006C42EF0D7
:10CC200031FF012070BD10B504000C235843FF49AB
:10CC3000401800210A000B000EC0200002F38CFEF9
:10CC4000200002F394FE200002F37BFE10BDF7B536
:10CC500086B014000600F64A00200092049007985F
:10CC6000210004AA03AB00F31AFE6B46187C001FD8
:10CC700003286AD82006000E05900FF359FB0FF326
:10CC800068FB05007079032806D16B461B7B05996C
:10CC90002A00300018F0F4F82EF0F0FE0190E5487C
:10CCA00047690124AC402740FFF7DBF82404240C3B
:10CCB00002902000FFF73EF86B46187BB823DB4A52
:10CCC0005843303280180021A0300173D7496B4699
:10CCD000D94A187C383900F397FD6B46197C187BCC
:10CCE00004F3CFFB6B46187CFFF768FA6B46187CA1
:10CCF000059A29003300FCF763F96B46197B28007D
:10CD000004F3CDFA6B46187C320029001CF0CBFEF0
:10CD10006B46187C29001CF067FF002F02D0200012
:10CD2000FFF72CF802A8FFF702F901982EF0AAFEEF
:10CD30006B46197B079A30001DF0FFFE6B46187B8F
:10CD4000FFF771FF012009B0F0BD0020FBE7F7B548
:10CD500084B005001600B64A009200240598310000
:10CD600003AA02AB039400F39AFDB54FB349380010
:10CD700036F0E6EA6B46187B001F032847D8F91304
:10CD8000380036F0DEEA3006000E0FF3D1FA0FF36A
:10CD9000E0FA2EF073FE0600FFF763F86B46019091
:10CDA000187AB823A149584330314018A0306B4657
:10CDB0000473A14A187B683900F326FD6B46197B82
:10CDC000187A04F35EFB6B46187BFFF721FA280004
:10CDD000FCF7D2F86B46187A04F3FAFA6B46187B24
:10CDE00029001CF0D2FD6B46187B29001CF02EFF99
:10CDF00001A8FFF79CF830002EF044FE6B46197A2C
:10CE0000059A28001DF099FE012007B0F0BD002012
:10CE1000FBE7F8B50D00060000242EF02FFE844A33
:10CE200007002906090E603230000EF3ADFF0A2814
:10CE30000DD27F4A00210001603211548018C16078
:10CE40002900300004F366FC14F05AFC0124380079
:10CE50002EF018FE2000F8BDF0B50400002085B0CB
:10CE6000019008780D000007400F16D104F3F7F881
:10CE70000700042811D0704800F3F9FC0600401C9C
:10CE80000BD03806000E3106090E020004900F0088
:10CE9000280004F3A1F9002802D1002005B0F0BD5C
:10CEA000607902280FD1200033F0C8FB0521C901A9
:10CEB0004018807A80070BD55F20005D800707D57A
:10CEC0000120019004E0200029F06DFD0028F7D139
:10CED000019904981CF0A5FF2A000499143220003F
:10CEE0001DF015FE281D0EF32AE90006000E0FF3B3
:10CEF0001FFA0FF32EFA029052480068012807D15A
:10CF0000B420005B03214902884201D336F01CEAB9
:10CF1000607903280AD1281D0EF310E90106049B4D
:10CF2000090E3A00200017F0ABFF01E0793305430A
:10CF30000100000034CB00000004000083E21E3634
:10CF4000022803D10299300018F055F81F20400143
:10CF500020180079002806D002200FF304FA0100FF
:10CF6000300018F03EF83D483D4A416A02984000C2
:10CF7000A430085A904201D18031C8690104090CDB
:10CF8000380003F04AFF012004F0F3F8300004F306
:10CF900035FB2B4A0120B100383A5050294A009203
:10CFA000049A3B002900200000F368FB3800FFF7DB
:10CFB000F4F82EF06DFD0600FEF75DFF0390281DCE
:10CFC0000EF3C6E802060298120E23003900FCF7A1
:10CFD00001F8281D0EF3BCE802060299120E230088
:10CFE00038001CF0B3FD281D0EF3B2E802061D4800
:10CFF00002992318120E38001CF0B5FE03A8FEF7A4
:10D00000A0FF30002EF048FD012051E7F3B581B0BC
:10D0100006002EF03DFD0B4F0024009018206043C9
:10D02000395C00290BD0C51968780FF38BF90FF321
:10D030009AF9B04203D1E878029903F0EEFE13E0CA
:10D04000B4CC00047CCB000440A20080141800047F
:10D050006666FFFFBBBBBBBBD00600047CC70004F9
:10D06000FFFF000029020000641C2406240E042C8B
:10D07000D4D300982EF010FDFEBDF8B500252D4F3D
:10D0800018206843395C002924D0C419201D33F0CE
:10D090005DFB06001ED061780022300014F0B4FD64
:10D0A0006B46198800010907090F014300911878A0
:10D0B000000900011870A078009904F363F86B462A
:10D0C00018882900000960810020207360733000F7
:10D0D00000F05DFE6D1C2D062D0E042DD0D3F8BD85
:10D0E00070B505000C0002F34CFC0C216943124B97
:10D0F0005A5812185A50226070BD70B505000C00C5
:10D1000002F334FC0C226A430B4951188A68121846
:10D110008A60226070BD70B505000C0002F31BFC34
:10D120000C226A43044951184A6812184A60226066
:10D1300070BD00007CCB0004B4CC000470B50500C9
:10D14000002433F085FA0600280013F054FB0F2169
:10D1500089012B7969180EF3D6E807050F0505112B
:10D16000110F11006979022902D1340064340CE0F6
:10D1700000290AD0046808E08C6A06E02EF088FCDA
:10D18000FF48F3F7A5F9F8F77FFE200070BD70B5F2
:10D190000500002413F02FFB2979002908D001296C
:10D1A00008D003290CD16979032901D001290FD1B5
:10D1B00044680DE00F2080012818846A183407E0C5
:10D1C0002EF066FCEE48401CF3F782F9F8F75CFE9F
:10D1D000200070BD70B50500002413F00CFB297908
:10D1E000002908D0012908D003290CD16979032925
:10D1F00001D001290FD1C4680DE00F20800128184B
:10D20000846A253407E02EF043FCDD48801CF3F7E8
:10D210005FF9F8F739FE200070BD0179012905D1C9
:10D220000F2189014018806A353070475D307047A2
:10D2300070B50400FFF782FF0500200033F008FA04
:10D240006179022904D10521C9014018807A0CE0D6
:10D2500006F03CFB0F21890161180128086902D101
:10D260002030807F01E02030007FC006C10F08D051
:10D27000200029005D3000F335FF002801D0012097
:10D2800070BD002070BD70B504000D0033F0E0F9F2
:10D290006179022904D10521C9014018807A12E080
:10D2A0002079062802D15F20005D0CE006F00EFB1D
:10D2B0000F21890161180128086902D12030807F7F
:10D2C00001E02030007F81064006C30FCA0F200016
:10D2D00029005D3000F314FF70BD70B50400407983
:10D2E000022802D02079062806D12000FFF726FF69
:10D2F000C0784007C00F70BD2000FFF71FFF05007A
:10D3000006F0E4FA0F218901020061180969002082
:10D31000012A02D12031897F01E02031097F89076C
:10D32000E9D5E9788907E6D0012070BD81688904D4
:10D330000AD57030817B427B08021043F451B0164D
:10D340000100000030CF000000040000D038CD5AAA
:10D3500080059149400F800008587047092000025D
:10D3600070470100603040788A688007800F92041F
:10D3700009D570318A7B4B7B110219438905490F0E
:10D38000884200D80800704780684006C00F704788
:10D390000100896800204A0602D5090600D501204F
:10D3A0007047F7B584B0002406000F00FFF7D0FEE9
:10D3B00005003000FFF7F5FE03903000FFF714FF83
:10D3C00002003000FFF733FF0300B0684006C00FD3
:10D3D0000AD0039800216E4607C61A000699380045
:10D3E0002B0000F3AEFE0400200007B0F0BD08B52E
:10D3F0000168836A01290AD1002202600100674A9C
:10D4000018000092664A674B1C3100F311FF08BDFB
:10D41000F8B50D00FF21040017002D3106F0C2FB06
:10D420000028286011D0018922004618AC32F12171
:10D43000890000923A0061180D2306F007FC0320D2
:10D44000203630702968C0200881F8BDF7B5FF216B
:10D4500005002D31544882B02E18280006F0A2FB9A
:10D4600004001BD020892A00AC32F1212718890042
:10D4700000922000320069180D2306F0E7FB04201B
:10D4800020373870C0202081049A0399200001F3CE
:10D4900029FA200006F018FC05B0F0BD0020C043BA
:10D4A000FAE7FFB587B01C000600002006903F4851
:10D4B0004068002802D03D480BF386FB3B4F08989C
:10D4C0001837002830D12079E178000208432BD1A9
:10D4D0003079012804D07179022901D0062807D1BA
:10D4E000607900228006010F300014F097FB05E000
:10D4F00060798006010F300017F0D6FD05006079D5
:10D500006B461875A0795875244AF1208000039263
:10D510002349099A30180291019000927A89059B5B
:10D520002900300000F3F6FF30001FF079FB050002
:10D530006079C3210840397A23008906090F8900E0
:10D5400008436071069A0092099A0899280000F32E
:10D55000B2FF28001FF0DBFB0BB0F0BD7CB5040070
:10D560002EF0A0FA1249050048686B46401C48603E
:10D57000E0799870207AD870A07A617A0002084326
:10D580009880E068631C012269461FF00DFD2800A9
:10D5900010E000000300010094350400CFCF00002C
:10D5A0007CCB0004DCCB000429020000400003C057
:10D5B00050B901C02EF07AFA7CBD7FB504002EF080
:10D5C00071FA0500FE4A210001A801F375F900284F
:10D5D00007D0012200922069621C022101ABFFF7F3
:10D5E00060FF28002EF062FA7FBDF8B50D0001241F
:10D5F0004179022915D10F218901411809680129B2
:10D600000FD133F056F8060028000EF3A5FE852151
:10D61000895D0091010000980AF0A0FD002800D06B
:10D6200000242000F8BDFEB50400401C33F098F83B
:10D63000E44F05004AD0A8684006C00F46D0207AC3
:10D640008006010F2800FFF7D0FF00283ED0207A87
:10D650008006010F01916879032801D001280BD1C0
:10D66000280033F021F9217A0600C3200140300759
:10D67000800E0143217200E00E00D34932002000E9
:10D6800000F3EAFF411C39D0621C280002A9FFF711
:10D69000BFFE0298002819D000223100280014F0A3
:10D6A000BDFA01000298220000F3AEFF207AC321E8
:10D6B000084001990907890E08432072C048E179A2
:10D6C0000170029806F000FB401C01D1380013E005
:10D6D000BE480E2221000DF304ECBC480561183849
:10D6E0000BF302FAB94864220092B94AB74B012100
:10D6F00018380BF338FA0120411C16D1617B227BCC
:10D7000009021143E181E17AA27A090211432173EE
:10D71000090A6173217AA172617AE1720121002202
:10D72000217262722170A6490A70FEBD7CB50400A8
:10D73000401C33F015F8A34E050012D0A86840062F
:10D74000C00F0ED0621C280001A9FFF7D49FE4ADE2
:10D75000010000002CD30000000400006FFDE8E988
:10D7600061FE0198002806D0210000F399FF01987E
:10D7700006F0B4FA0600701C02D10120207020E0EF
:10D78000607A217A000208431BD1974A0092974A97
:10D7900000212B00200001F3CEF8A07A934A8006E6
:10D7A000010F601C0EF30EFB0A280AD2E17AA27A5E
:10D7B000090211438A098E49000141182800FFF728
:10D7C0003FFA30007CBDFEB50400401C32F0D2FFB1
:10D7D000814E050003D0A8684006C00F01D130007B
:10D7E000FEBD6879032801D001280AD1207A0109F9
:10D7F000280033F063F8217A0907090F000101437B
:10D800002172E0796B461872207A58720298019062
:10D81000A07A617A07020F43621C28006946FFF76D
:10D8200001FE0098002801D1300006E001993A007D
:10D8300000F38FFD009806F051FA411C02D101213E
:10D840002170FEBD0028FCD165480B2221002C3040
:10D850000DF350EB62482C30C56018380BF34EF9CD
:10D860005F486422143003000092624A0121183399
:10D870000BF383F90120FEBD70B50B004A780D78DB
:10D8800011020F22920180180069002429435C30A4
:10D89000012902D10422991C02E001000422981CF3
:10D8A0000DF328EB200070BD10B5FFF7D9FD00285F
:10D8B00000D1012010BDF7B582B005000E004F6BFE
:10D8C0008C6BFFF74FFCA9684906C90F0BD029796B
:10D8D000012909D1484A2B0000924848049AAC33E8
:10D8E000310000F323FFE1E56979032901D0012923
:10D8F000F9D1002CF7D0002FF5D001794A07D30FCA
:10D9000022795207D20F934204D0FB231940920090
:10D91000114301710179CA06D30F2279D206D20FC1
:10D92000934204D0EF231940120111430171C178D1
:10D930000A07D30FE2781207D20F934204D0F723DD
:10D940001940D2001143C170017922798B079207E7
:10D950009B0F920F934203D08908890011430171F4
:10D960002800FFF779FC02000021280029F0A7FB1E
:10D970009CE570B50400C8798A7905020F20800102
:10D980001543201802698B782032012D02D0022D18
:10D9900036D109E01377CB78537700690A794030A4
:10D9A00002704979417008E09377CB78D3770069AA
:10D9B0000A79403082704979C170200010F048FB2C
:10D9C0002000FFF749FC02000021200029F077FB2E
:10D9D00070BD000050B901C0FFFFFFFF7CCB000409
:10D9E000580003C09BD10000CFCF0000DCCB000467
:10D9F000C8CF00043DD10000404B4C0030E900048A
:10DA00001377CB78537702690B79403213704B79D7
:10DA1000537002698B782032C6E710B5CA798C79C9
:10DA200013020F2292018218106923432030022B27
:10DA30000AD1837F8B70C07FC870106940308278B4
:10DA40000A71C078487110BD037F8B70407FC87029
:10DA50001069403002780A714078F3E7F8B50500A4
:10DA60000E000024FE4B310020006A46FFF279FED2
:10DA7000012808D121003000FFF7E9F90022210038
:10DA8000300000F31EFCF74A31002000FFF298FE40
:10DA9000012809D1220031002800FFF776F9012280
:10DAA0002100300000F30DFC641C2406240E082C19
:10DAB000D8D3F8BD38B50400FFF754FB0500A068C3
:10DAC000C02188430022A060E748110013000092A3
:10DAD00000F369FE207901280AD100220F2080017D
:10DAE00020180092806A11003530130000F35BFEAD
:10DAF000DE4A20000092DE4A29005D30002300F358
:10DB000052FEDC4821182000FFF7A8FF0022110078
:10DB1000200029F0D4FA38BD0022010010B54031B0
:10DB200082870A80C2874A8020390A7F20231A43CD
:10DB30000A778A7F44301A4342231A438A7718218E
:10DB40000DF374EA10BDF8B50E0001894569091896
:10DB50000C6F28001AF011FB002807D0F62CA8350E
:10DB60000100000028D70000000400003C273B858E
:10DB7000E078400604D52188200020300F1801E00D
:10DB800027002037380000F378FE002813D0BB4A66
:10DB9000A31D483200921C002A003900300000F317
:10DBA0002FFE0006000E05D02300320039002800A9
:10DBB0001FF00EFAF8BD380000F369FE0028F9D016
:10DBC00028790228F6D03200390028001FF015FA13
:10DBD000F8BDFFB583B01400039832F057FD4B2118
:10DBE000C90040180290002001906078217800025E
:10DBF0000843052864D9401F04060498240E401DDC
:10DC000000900398C179007912F0D5FA32F065FDE1
:10DC1000092686570700007A083780063500800FEE
:10DC20000B2101280BD1F21E012A00DDF01E050692
:10DC300008002D16F11D0B290FDAF01D0DE0032849
:10DC400039D10120F21F012A00DDF01F050608006E
:10DC50002D16F11C0B2900DAF01C060636162AE0F8
:10DC6000009822004921F8F771FA010028D04A787B
:10DC7000901C0006000E84460020521E96460EE0C0
:10DC80000B18DA78AA4207DBB24205DC7B789342B4
:10DC900002D00120019004E0401C0006000E8645E1
:10DCA000EED80098081A221A6046101A0406240EAC
:10DCB000604608180090002C02D001980028CFD0B0
:10DCC00002982030807C80070BD5049800794007AB
:10DCD000800F02D10198012803D10398002108F098
:10DCE000ADFE04980921007908420BD048206B460C
:10DCF000187001205870002098700398032269461C
:10DD0000FFF7B8FB012007B0F0BDFEB50500160017
:10DD100048780C0001270C36002818D001281CD0A8
:10DD200002282FD1A868C0042DD52879002808D151
:10DD3000E078000905D15548002182680B002EF0DB
:10DD4000B8FB22003100280000F383FB1BE0220017
:10DD50003100280000F0EAF815E02DF0B7FE019040
:10DD60004848A178401E0278914207D100210170F5
:10DD70002300320028000091FFF7A7FB01982DF047
:10DD8000A9FE00E000273800FEBDF8B500240126FA
:10DD90003D49394F3603451818206043C119385C96
:10DDA0000A000A3200280BD01088B04208D0091DA2
:10DDB000062228002DF0B5FA002801D10120F8BD77
:10DDC000641C042CE8D30020F8BDFEB504000D004F
:10DDD000407902280DD120000AF026FE002808D044
:10DDE000112040012018418A0122200007F059FE2D
:10DDF000FEBD18216943204802AA0D1868892F002A
:10DE00000D370190781E00900821200005F0FDFEDE
:10DE10000600EDD002980421006F017000214170CE
:10DE20002030042104000DF336E920780421084352
:10DE30002070607801076878090F00010143617064
:10DE4000E078A1780002084301990007000F09015A
:10DE50000843A070000AE0700D49300003F02EFC6A
:10DE60000028C5D03878401C387000980121017016
:10DE7000FEBD0000DCCB00047CCB0004240003C00A
:10DE800074FD02C051B901C029020000C82C000471
:10DE900002100000F8B505002DF018FE434E0700F3
:10DEA00000241820604381190A00305C0C32931E54
:10DEB000002814D01078002811D1188801221203EC
:10DEC00090420CD03A48091D062228182DF029FA54
:10DED000002804D12106090E2800FFF776FF641CF4
:10DEE000042CDED338002DF0F5FDF8BD10B504008C
:10DEF0005F21095D0020C90717D06079022805D18C
:10DF0000200032F0C3FB403080780CE005F0FCFCD0
:10DF10000F21890161180128086902D12030807F12
:10DF200001E02030007FC007C00F10BD7CB50400A9
:10DF30000E00806815004006C00F0FD02EF06EFE58
:10DF4000002807D00F208001201800694030007F92
:10DF5000C00703D100F053FD00280ED0320020008E
:10DF600001A9FFF769FA0198002805D075EF5C3325
:10DF70000100000024DB000000040000C8484E310E
:10DF8000290000F30FFA019805F0BCFE7CBD207952
:10DF900000280ED1E8788006000F0AD1E8796B4698
:10DFA0001870287A58700848009A230000212EF033
:10DFB0008AFA22002900300000F311FA7CBD00002B
:10DFC0007CCB000429020000C82C000410B5FF4CD3
:10DFD000606B002805D135F0EEE9002801D0012062
:10DFE0006063606B10BD10B535F0E8E9F7490020BB
:10DFF000486310BD30B50020F54D0D21040003002D
:10E000008901691814E0E868401CE8601000526B50
:10E010008A62002A00D1CB620279052A0BD12A69D3
:10E02000521C2A618362036003710020002C02D11C
:10E030008A6A002AE7D130BD10B50A68E44B002A8D
:10E0400003D11868401C186010BD8A6A824203D050
:10E050005868401C586010BDDC480024026A002A41
:10E060000FD08A4210D09A68521C9A6004220A711A
:10E07000C26A002A01D0516300E08162C1624C6330
:10E0800010BD012201620A71006A07228462D14830
:10E09000402100682EF03DFE10BD10B50A68002A30
:10E0A00010D0CA4A936B83420CD1106A002809D061
:10E0B000884207D100209063C6480722006880216B
:10E0C0002EF027FE10BDF0B5050085B000F0AEFCC7
:10E0D000002000F0B9FC04007ED0286BBB4F206309
:10E0E000786A401C7862206000F0A8FC01F3A5F972
:10E0F000029000200391019020682E00002120361C
:10E10000002802D1012078622060002327002037F8
:10E110002371787BEF2108407873307A6071A079A1
:10E12000717A800889078000890F0843F321A07164
:10E130000840B17A8907090F0843CF21A071084030
:10E14000F17A8907890E0843A071696928695940E5
:10E1500008430DD02A6902986B690399121A8B4102
:10E160000AD3029A2869039B6969801A994102E0DF
:10E17000A869002800D0019001A80DC800218018CE
:10E180005941E160A060E8692061286A6061686ABD
:10E19000A0612868E06168682062A8686062787B96
:10E1A000317B400889074000C90F0843FD2178737F
:10E1B0000840317B4907C90F49000843FB217873A8
:10E1C0000840317BC906C90F89000843F7217873DD
:10E1D0000840317B890600E01DE0C90FC9000843F3
:10E1E00078730220B873307B000701D50620B8731E
:10E1F000317B0120C90700D102203873BA7B23008C
:10E2000000927548019A28332100F7F7C7FF0028CC
:10E2100006D1206001E000F011FC002005B0F0BD47
:10E220002068FBE7F8B505250E0000F00DFC0400A2
:10E230006648016AA14216D1A06A002803D0FBF209
:10E24000F2FE0020A062002E66610CD000222300A6
:10E2500000926148283332002100F7F79FFF032521
:10E26000002800D104252800F8BD70B5052500F070
:10E27000EBFB04005548016AA14207D1A06A0028BF
:10E2800004D0FBF2D0FE00200325A062280070BD60
:10E29000F8B50F00052600F0D7FB4C4C0500216AAD
:10E2A000814215D1A06B002803D0FBF2BCFE0020F8
:10E2B000A063002F0CD0454B002200924748383312
:10E2C0003A002900F7F76AFF0326002800D1042648
:10E2D0003000F8BD70B5052500F0B6FB3B4C216A57
:10E2E000814207D1A06B002803D0FBF29CFE0020E6
:10E2F000A0630325280070BD38B50120FDF7BAFCE6
:10E30000324C2C20236AC15C5A6A1868DB69984732
:10E31000206A006B04F02DFB00F088FB2DF0E0FB81
:10E32000216A05000020086000F088FBFFF762FE0C
:10E33000206228002DF0D8FB216A002909D02E2068
:10E34000425C0B000092264A23482833F7F726FF49
:10E3500003E0FFF748FE15F0A7FE032038BDF8B52F
:10E3600005002048194F006A002813D0386A046B52
:10E37000200014F0A4FA182D06D10228CF370D0F73
:10E380000100000020DF0000000400009B929D5D62
:10E3900004D0194920310979814204D12A00002191
:10E3A000200005F00DFDF8BD072032F093F94DE097
:10E3B000386A006BB04204D0300020F03FF90028EA
:10E3C00040D12C00162D1FD1300020F01CF9002860
:10E3D00033D07079022830D1386A2030407B0DE08C
:10E3E00078360004383300047C050004DDDB0000CF
:10E3F0003FDC0000A086010020420004400701D558
:10E400002A241AE0282418E0192D03D01A2D01D04F
:10E41000182D12D10F20800130180069817B00294E
:10E4200001D02C2409E0C07B002801D0292404E07D
:10E43000386A006BB04200D018242200002130005E
:10E4400005F0BEFC0721300011F072FE0600AFD1CE
:10E45000F8BDFEB505250F0000F000FB040073D0E9
:10E46000A06A0026002802D0FBF2E7FDA662FC4D60
:10E47000286AA04273D100F0E3FA2DF03BFB019033
:10E480002079022801D0012810D12034607B10218E
:10E490000843607300F0DCFAF2480722006840216C
:10E4A0002EF041FC01982DF029FB53E001982DF04E
:10E4B00025FB207903281ED1267100F0C9FA286AAD
:10E4C0002030072F077308D0082F0BD11A20FFF731
:10E4D00050FF39200EF0B8FA42E01920FFF749FF4B
:10E4E0003820F7E7286A006B1FF0DEFA1820FFF7E4
:10E4F00040FF3720EEE704282ED100F0A9FAE369A7
:10E50000626A20680B219847286A006B04F03BFA86
:10E5100000F096FA2DF0EEFA26600700267100F062
:10E5200097FAFFF771FD286238002DF0E7FA296AA3
:10E5300000290BD02E20425C0B000092CA4ACB4827
:10E540002833F7F735FE05E00BE008E0FFF755FD4F
:10E5500015F0B4FD0320FEBD00F07AFA00E026605D
:10E5600003252800FEBD70B5040004252DF0C2FA75
:10E570000600BB48006AA04219D021792068032513
:10E58000042906D105212171E369626A0B219847AC
:10E590000DE0A06AFBF251FD012808D1E369626A2F
:10E5A00020680B2198470021A16221602171300071
:10E5B0002DF0A4FA280070BD70B50500042400F009
:10E5C0003FFA280000F04AFA002802D0FFF7CBFFFC
:10E5D000040000F03DFA200070BDF8B505000E0003
:10E5E00000F02EFAA24F002438206043C019816940
:10E5F00000290ED0002D03D04521095C890705D4E0
:10E60000002E06D04521095CC90702D01830FFF75B
:10E61000AAFF641C0F2CE7D300F01AFAF8BD012101
:10E620000020DAE710B51FF038F8002801D10120EA
:10E6300010BD002010BD38B51FF0F5F81620FFF70B
:10E6400098FE1520FFF795FE854C206A4179002938
:10E6500006D081790091417900980022FFF7E2FF0E
:10E66000216A03200871206A02002030417BCB061A
:10E6700008D5EF2211404173206A06210068FFF798
:10E68000E8FE1FE09069002808D000F3E0FE256A4C
:10E69000AA68EB68801A9941A9690860216ACB6968
:10E6A0004A6A086803219847216A4869002809D006
:10E6B0008A6A002A06D100920B0002006B482833B8
:10E6C000F7F776FD032038BDF1B582B0694E644D91
:10E6D000306800282BD12C6A27002037787B01076F
:10E6E000CA0F00924007C30F6179206BA21D15F07D
:10E6F000B3FC1FF089F8E369397B626A20689847A8
:10E70000022829D00298002805D01620FFF731FEF4
:10E710000120306005E01720FFF72BFE36200EF0B9
:10E7200093F9296A02200871306800281BD0286AF2
:10E730002030407B400711D5042013F0C6F8002894
:10E740000CD111F03CFD040011F046FD844205D0CF
:10E750004948006A002801D10220FEBD0020306037
:10E7600035200EF071F90320FEBDF7B586B0040028
:10E770001600002513002F0003AA04A905A830F0F5
:10E7800045F9059B002B14D0606900284816AC6B36
:10E79000010000001CE3000000040000B30318E0C7
:10E7A00002D1306801256061039A079901920091B6
:10E7B000220000211E0004980B00B0470700002D26
:10E7C00001D000206061380009B0F0BD70B586B09E
:10E7D0000600002503AA04A905A802AB30F020F921
:10E7E000059C002C09D0039A002101920A00009197
:10E7F000310004980023A0470500280006B070BD32
:10E800001C482030017F491C01771A49096A0029F8
:10E810000AD00A79032A07D1427F521C4277CB697A
:10E820004A6A0868092118477047124810B5006AFB
:10E8300000280BD02030017B032907D1012101736F
:10E840000D480722006840212EF077FA10BD70B500
:10E850000420084C236A002B33D02C21C95C186893
:10E860000325012918D1FFF7C5FB00281FD001207F
:10E8700019E00000783600047C050004A086010041
:10E88000DDDB0000383300040003000420420004F4
:10E89000206A2030057313E0022913D1FFF7AAFB89
:10E8A000002804D00020FFF719FF0328F0D0012032
:10E8B000F7F782FA78480722006840212EF03DFAE7
:10E8C000032070BD03290ED1186B0F218901401858
:10E8D0000069022103F0D6FF206A04212030017371
:10E8E000FFF7B3FEECE7062901D1062006E0072971
:10E8F00007D100210120FFF77AFE0720FFF710FD66
:10E90000DEE7082901D10820F8E75A6ADB69984751
:10E91000D6E762490420096A002907D00A79032A48
:10E9200004D1CB694A6A0868052118477047052851
:10E9300001D2002801D100207047594AC000801838
:10E9400006C906C001207047F3B587B002250798B5
:10E950004278037810021843012836D1079F891E98
:10E96000BF1C30E0F8780E1FB97800023C00084365
:10E97000B0422ADC6078217800020843FF3864380E
:10E980001AD1201D0CF320EC401E0090200008300E
:10E990000CF31AEC7D23DB005843019020000C306F
:10E9A0000CF312EC7D23DB0058430290009801A980
:10E9B0000006000EFFF7BBFFE078A17800020843D5
:10E9C000311A3F1DC7190429CCD2FF2064306B4691
:10E9D00098810C20D881079FBF1C01243048E1009A
:10E9E0000E18601C7D2104903068C9000CF3FAEF0A
:10E9F0007D2105907068C9000CF3F4EF0690102299
:10EA0000380003A90CF39EEA10371035641C052C5E
:10EA1000E4DB2800D8E62148006A002800D0012065
:10EA200070471E48006A002800D0012070471B482C
:10EA3000006A002800D0006B70471A480068002860
:10EA400006D01649096A0968814201D10120704740
:10EA5000002070471148002110B5006BC9432EF00B
:10EA600070F910BD0D4810B5006B2EF071F910BD96
:10EA700030B504000C4D0020010038224A435219E1
:10EA80009369A34201D110001830491C002801D11C
:10EA90000F29F2D330BD00007C0500047836000455
:10EAA00004030004700E00043833000410B5002481
:10EAB00020290FD065290BD108480DF35DF80028F7
:10EAC00005D1064814300DF357F8002800D0012472
:10EAD000200010BD02488260FAE7000068D0000400
:10EAE0002C030004FA48C068012800D000207047B9
:10EAF00010B5040003280CD8112017F0BCFECF215C
:10EB000008402101103901430906090E112017F0B0
:10EB1000C8FE10BD70B504000D001600F6F77CFDB0
:10EB20002000FFF7E5FF3100280017F0BAFE0120B2
:10EB3000FFF7DEFFF6F7B7FD70BD70B504000D00FE
:10EB4000F6F76AFD2000FFF7D3FF280017F093FEC9
:10EB500004000120FFF7CCFFF6F7A5FD200070BDF3
:10EB60000002FF30313070B500041407000C240F90
:10EB7000CA070FD0491E4910081805042D0C29009A
:10EB80000220FFF7DAFF0007000F210101430A0608
:10EB9000120E0BE04908081805042D0C26A2462881
:10EBA0000100000018E7000000040000E0D9CB8C51
:10EBB00029000220FFF7CBFF0009000122000243D9
:10EBC00029000220FFF7B0FF70BD00024018FF309F
:10EBD00011300104090C0220A6E70800110010B54D
:10EBE00017F069FE10BD080010B517F04EFE10BDFD
:10EBF00070B50C001500080017F047FEA84301008F
:10EC0000200017F058FE70BDF8B50120B5498860A6
:10EC1000F6F70CFD00252C022000FF309F30000489
:10EC2000000C072117F080FEFF34A0342004000CF4
:10EC3000042117F079FE2806000E0700102220217B
:10EC4000FFF7D6FF00242606360E002231003800DA
:10EC5000FFF7BBFF002231003800FFF78BFF641C79
:10EC6000142CF0DB6D1C012DD5DBF6F726FD02F030
:10EC700042FEF8BDF8B50025F6F7D8FC30272E0285
:10EC80003000FF30B6300404240C200017F0FDFDE6
:10EC900038430100200017F00EFE3000FF30BA307C
:10ECA0000004000CFF2117F006FE3000FF30BB30DF
:10ECB0000004000C002117F0FEFD3000413000047C
:10ECC000000C042117F025FE0024FF22210028005B
:10ECD0001AF003FC0022210028001AF013FC002285
:10ECE00021002800FFF771FF002221002800FFF714
:10ECF00041FF641C2406240E142CE6D33000FF30A0
:10ED000017300004000C402117F003FE3000FF30E4
:10ED1000A0300404240C8021200017F0FAFDFF36F7
:10ED20009F363004000C022117F0F3FD042120006F
:10ED300017F0EFFD6D1C2D062D0E012D9FD3F6F75C
:10ED4000BCFCF8BD6749002010B58860FFF792FF52
:10ED500002F0DAFD10BDF3B581B000250E002C00E5
:10ED60000127019817F091FD3100814304D138004B
:10ED7000A040284305062D0E641C012CF1DB280061
:10ED8000FEBD70B505000E0000243100280017F00C
:10ED900092FD641C012CF8DB70BD70B50C001500F1
:10EDA000080017F072FD28430100200017F083FDD2
:10EDB00070BD70B505000E0000242006000E320064
:10EDC0002900FFF7EAFF641C012CF6DB70BD70B56B
:10EDD00005000E0000242006000E32002900FFF777
:10EDE00007FF641C012CF6DB70BD012804D13E48EE
:10EDF000405C3E49400002E0491E48003C49085A38
:10EE0000704770B50028374B3A4C596018705A70EB
:10EE1000237802D1DF252B4003E0012802D12025F1
:10EE20002B43237001F01AF8012070BD2D48406873
:10EE300070472C48007870472A4840787047020095
:10EE40000020002900B512D011000120FFF7CDFFEE
:10EE500029490122884209D927490222963188424C
:10EE600004D926490322884200D90422100000BD9B
:10EE700023487D2110B5006849012CF040EB89053D
:10EE8000800A08431F4900E0401E0A68002A01DB8F
:10EE90000028F9DC002803D112490869401C0861E8
:10EEA00010BD002010B517F0F0FC0E4CA070012032
:10EEB00017F0EBFCE07010BD08B5F6F7B7FBFFF7F5
:10EEC000F0FF114817F015FDF6F7F7FB0020694633
:10EED0001CF0D8FA002819D16B4618705870987039
:10EEE0001BE000003C03000478420400C4EE310043
:10EEF000A8EE31002CE90004321400004416000092
:10EF0000E0B801C0002B0080907A01C06B461878F1
:10EF1000012802D1FFF778FE03E000210800FFF787
:10EF200011FFF6F783FBF6F7C8FB1AF065FA08BD88
:10EF300010B5FFF7C1FF01201AF00EFD012010BD32
:10EF4000FF48C0787047FE488078704770470002DD
:10EF5000FF3070B5BC3004040D00240CF6F766FBDE
:10EF60002900200017F0A7FCF6F7A7FB70BD0002F0
:10EF7000FF30BC3010B50404240CF6F757FB20001A
:10EF800017F083FC0400F6F798FB200010BDEC4856
:10EF900010B542680078EB4B002808D151001A00E8
:10EFA0000A32891820391888C98B08180946DF18D1
:10EFB0000100000014EB00000004000014B6BE388D
:10EFC00021E011000120FFF71AFFE44C0221595EF5
:10EFD000A04211D9E14C0421595E9634A0420BD9CC
:10EFE000DF4C0621595EA04206D9DD4C00217D345C
:10EFF000A04201D80821595EDA48805CD64A400018
:10F000002632105A40180004001410BD0002FF30D0
:10F0100070B5E93005040A060C002D0C120E29000B
:10F020000320FFF78BFD2004020E681C0104090C6D
:10F030000320FFF783FD2002020EA81C0104090C27
:10F040000320FFF77BFDED1C2904220E090C032091
:10F05000FFF774FD70BDF1B582B0F6F7F1FA02204A
:10F06000FFF75AFD0025029900246800401801901E
:10F07000200246193000FF3091300004000C17F0D8
:10F080000EFC8707FF3671363004BF0F000C17F0F7
:10F0900006FC8000620001993843641C012C8852F0
:10F0A000E6DB6D1C132DDEDB0120FFF735FDF6F7E7
:10F0B0000EFBFEBD00024018FF3051300104090C68
:10F0C000022010B5FFF74DFD4006400E10BD10B5F3
:10F0D0001AF0DAFA10BD0002FF3041300004000CD3
:10F0E000CA0710B509D0491E491008180104090CB7
:10F0F0000220FFF736FD000910BD49080818010479
:10F10000090C0220FFF72DFD0007000F10BD0002C3
:10F11000FF30801D70B505042D0C0024FF2229004E
:10F120000220FFF70BFD6D1C641C2D0424062D0C22
:10F13000240E022CF2D370BDFF230A3370B5002ACF
:10F1400000D11B1FCA08D2180002801804044D0702
:10F15000240C6D0F21000220FFF703FD0121A940BF
:10F1600001430A06120E21000220FFF7E7FC70BDE2
:10F1700010B54C07640FC9080002002A02D0FF3105
:10F180000A3101E0FF31891D40180104090C0220F9
:10F19000FFF7E7FC01210A00A240024200D0002153
:10F1A000080010BD01000120002900D00020704798
:10F1B00010B501246420F6F7A1F96B487D210068A1
:10F1C00049012CF0A6E98905800A0843674900E057
:10F1D000401E0A68002A01DB0028F9DC5D4900288E
:10F1E00005D14869012200241204801801E0486911
:10F1F000401C4861200010BD0100012010B5FFF740
:10F20000FEFD564A0021AA3A904217D9534A0121DD
:10F21000904213D9514A0221963290420ED9504A57
:10F220000321CD3A904209D94D4A0421904205D993
:10F230004B4A0521C832904200D9891F0804000CAE
:10F240001823444958433431401817F05CFB10BD73
:10F25000F7B58EB00E98002800D0012001900F98CD
:10F26000002501280BD00F984008012801D1012565
:10F2700005E00F9802258008012800D0ED1E0198B6
:10F28000344980001C310D900858691C74D00199D4
:10F290000C23304A5943C4328B18AA000B920C91AC
:10F2A0009C582C4BDC33CB189B580393294BF433DD
:10F2B000C9188958029117F026FB200017F023FB8C
:10F2C0000024F6F7BDF9E8000A90182060432849A9
:10F2D000260240180A990700405801063000FF3006
:10F2E00031300004000C090E099017F0EEFA0A996B
:10F2F0007818406801063000FF3030300004000C00
:10F30000090E089017F0E1FA022D3AD1FFF7FEFB43
:10F31000002836D017482701C05901060998090E60
:10F3200017F0D3FA13483F18786801063000FF3011
:10F3300033300004090E000C17F0C7FAB868010654
:10F340000898090E17F0C1FAF868FF360106090E91
:10F35000323612E03C030004B836000432140000D8
:10F360004416000078420400E0B801C0002B008081
:10F370004C0C00045C540004B1E03004000C17F0A5
:10F38000A4FA641C2406240E012C9ED3F6F79FF9E0
:10F390000320FFF7C1FB019801281DD1022D1BD1CD
:10F3A000A74E0024A00081198978305A17F08DFAF1
:10F3B000641C142CF6DBFF20FF21ED30C0120D98E9
:10F3C0000100000010EF000000040000476C6D54C5
:10F3D00017F085FAFF20FF21EE3017F080FAFF20AA
:10F3E000FF21EF3017F07BFAFF213BE00EA807C8A2
:10F3F00018F0A1FF06000006000E6B46187007907B
:10F400003004000E587006903002000E987005907F
:10F41000300E0024D870012704903800A0403042FC
:10F4200005D00399A00041188978039A04E0029955
:10F43000A00041188978029A105A17F050FA641CFB
:10F44000142CEADBFF200799ED3017F048FAFF2073
:10F450000699EE3017F043FAFF200599EF3017F0C8
:10F460003EFA0499FF20F03017F039FA1BF0E5FC62
:10F4700000283BD078490D98774A08580C99E83213
:10F480008A180B995658754A0C998A180B9957582F
:10F4900017F043FA0320FFF749FB019801280DD12B
:10F4A000022D0BD16E4D0024A00041198978285AF5
:10F4B00017F015FA641C142CF6DB17E00EA807C829
:10F4C00018F039FF050000240120A040284204D094
:10F4D000A00081198978305A03E0A000C119897809
:10F4E000385A17F0FCF9641C142CEDDB0120FFF7EF
:10F4F0001DFB11B0F0BDF7B584B00498002801D011
:10F50000012200E000220026012909D04808012834
:10F5100001D1012604E002268808012800D0F61E49
:10F520004D49900008310858711C01D1002406E0B3
:10F530000C215143494A18328918B2008C5817F0EF
:10F54000ECF9200017F0E9F9F6F784F80024F00050
:10F550000390182060434349250247180398385800
:10F5600001062800FF3031300004000C090E029023
:10F5700017F0B5F903983818406801062800FF30E5
:10F5800030300004000C090E019017F0A8F9022E8B
:10F5900026D1FFF7C5FA002822D033482701C059E9
:10F5A00001060298090E17F09AF92F483F1878685B
:10F5B00001062800FF3033300004090E000C17F05C
:10F5C0008EF9B86801060198090E17F088F9F868F5
:10F5D000FF35010632352804090E000C17F07FF9BB
:10F5E000641C2406240E012CB3D3F6F77AF8049891
:10F5F000012802D10698FFF709FE07B0F0BD0028E8
:10F6000010B505D11948002900D1194817F085F91E
:10F6100010BD10B5F6F73AF916494000085A4004F3
:10F62000000C10BD70B504000D00FFF7F2FF0300E1
:10F6300029002000FFF7EDFB0022190017F093F9D5
:10F6400070BD0D4908680222904308600B490020F4
:10F65000086070471C8701C0600300046004000458
:10F66000348E01C04C0C00045C540004488101C07D
:10F67000588101C0E4340400002B0080EC07000432
:10F6800070B5FE4C60680125ED052843691088437C
:10F6900060600120F5F73CFF60680321890508439D
:10F6A0006060A843606070BD10B50400F448006855
:10F6B000002801D100240CE00021012016F032FBCB
:10F6C000F049A000401800680406240E012016F03E
:10F6D0004BFB200010BD70B5040018D000210120A4
:10F6E00016F020FBE848E74BE849026806E0012AEB
:10F6F00003D18000A578C0180560241D20888842A9
:10F70000F5D1A578FF2DF2D1012016F02DFB70BDAB
:10F71000DF48012210B5052142700170DD48016803
:10F72000130619430160DC480168114301602CF0A5
:10F7300009FA0400D948FFF7CEFFD948FFF7B4FF14
:10F74000D349891FC87020002CF000FA012010BD99
:10F7500070B52CF0F7F905000020FFF7A5FFCC4CA1
:10F76000A41F207128002CF0F1F9207970BD70B52C
:10F770002CF0E8F905000120FFF796FFC44CA41F08
:10F78000607128002CF0E2F9607970BD00207047AC
:10F79000BF49891F487070474042022900D90221A1
:10F7A000BB4A89003E328918BE4A1268012A01D13B
:10F7B0008A5601E000228A5601231018B44A921F8B
:10F7C000D35602228A56C018824203DB775126E8BC
:10F7D000010000000CF3000000040000F8A948E755
:10F7E00003228A56824200DD100000060016704790
:10F7F000B14910B50A68AB494042891C012A01D1C0
:10F800008A5601E000228A56A64C0223CB56A41C3D
:10F81000032161561018834201DA180002E0814288
:10F8200000DD08009F4B03249B1F1C57121B8A42BC
:10F8300000DC0A00000600169A7010BD9949027893
:10F84000891C0A7002794A7082783C310A70827988
:10F850004A7042780A7142794A71C2780A72C07954
:10F86000487270478F4B04219B1CC9431A001970C2
:10F870003C32597011705170117151711172517285
:10F880007047002801DD002004E06421C94388425C
:10F8900000DA08004042000600167047002070475A
:10F8A00070B505007D480C00006800280AD00021D2
:10F8B000012016F041FA7849A800401804600120A0
:10F8C00016F05CFA70BDF7B588B004000020029015
:10F8D0002CF042F9039000252004000C07900998B1
:10F8E000002824D100242806000E069002AA0192C6
:10F8F0000094069B0A9A0799099833F0A0ED002816
:10F900000FD0684829014A300E18A7006B46F05BFB
:10F91000597AFFF7C5FFF0196B464088197AFFF74F
:10F92000BFFF641C2406240E042CDFD344E0099896
:10F93000012841D100242806000E059002AA009457
:10F940000192059B0A9A0799099833F078ED0028EF
:10F950002DD0012C1AD118215248694300265A3063
:10F960000F18A019800004906B46385A597AFFF797
:10F9700097FF04986B4638184088197AFFF790FF74
:10F98000761C3606360E052EEBD310E018214548BE
:10F9900069435A300E18A7006B46F05B597AFFF79F
:10F9A0007FFFF0196B464088197AFFF779FF641CD6
:10F9B0002406240E022CC1D36D1C012D8FDB03986D
:10F9C0002CF0CEF80BB0F0BDF7B584B005002CF0EC
:10F9D000C3F8070000242804000C039002AA009238
:10F9E0002306069A039905981B0E33F02CED002888
:10F9F0000DD02C4EA500B61D6B46597A705BFFF7F3
:10FA00004FFFA8196B46197A4088FFF749FF641C1D
:10FA1000012CE3DB38002CF0A3F807B0F0BDF7B5FC
:10FA200084B005002CF098F8070000242804000C8E
:10FA3000039002AA00922306069A039905981B0ECA
:10FA400033F004ED00280DD0164EA5000A366B46A3
:10FA5000597A705BFFF724FFA8196B46197A408822
:10FA6000FFF71EFF641C012CE3DB38002CF078F854
:10FA7000D3E73EB56B460C0019705870009801A989
:10FA80001BF034FD002819D001A8FFF7D7FE3EBDBA
:10FA90000028008028F900040020009024F90004C8
:10FAA000FFFF00009604000480210080002D0080EC
:10FAB000943E0400CB020000081800042000FFF769
:10FAC000D1FEE4E7002800B511D1022A05D10929A9
:10FAD00001D8481C00BD082000BD032A05D1052916
:10FAE00001D3C81E00BD022000BD481E00BD022A71
:10FAF00001D0032A45D174293DD011DC8807800F3D
:10FB00003DD18B10093B0BF362EC142C2C2E2E3ABA
:10FB10003A30303A3A3A3A3A3A3A3A323234343A75
:10FB20008C292AD00EDC802904D005DC782922D04B
:10FB30007C2924D17E2000BD842901D088291ED1B2
:10FB4000862000BD992904D005DC902915D095297F
:10FB500015D1972000BD9D2901D0A1290FD19F204B
:10FB600000BD262000BD2E2000BD3E2000BD662029
:10FB700000BD6E2000BD762000BD8E2000BD362069
:10FB800000BD900801283BD174291CD011DC8807E6
:10FB9000800F33D18B10093B0BF318EC142A2A2A5F
:10FBA0002A3030303030303030303030302C2C2C67
:10FBB0002C308C2920D00DDC802904D005DC78295C
:10FBC00001D07C291AD17A2000BD842914D088293B
:10FBD00014D111E0992909D004DC9029A209D7B7E2
:10FBE0000100000008F7000000040000AB739B8BCD
:10FBF0000CD095290CD103E09D2901D0A12907D172
:10FC00009B2000BD2A2000BD6A2000BD8A2000BDC7
:10FC10003A2000BD080000BD10B50400FFF75CFFEE
:10FC2000002C00D1401C0006000E10BD4178037866
:10FC30000A021A4301D0012A06D1C17A837A090245
:10FC4000194303D0012901D001207047FF490A70F0
:10FC5000C2788378120612141A434A7042790379E3
:10FC600012021A434A80C279837912021A438A80A7
:10FC7000427A037A12021A43CA80C27A837A120243
:10FC80001A430A72427B037B120612141A434A7209
:10FC9000C27B837B12021A434A81427C037C12029C
:10FCA0001A438A81C27C837C10021843C8810120D8
:10FCB00088770020704770B50500E5480C000068A3
:10FCC00000280ED00021012016F040F8E149A800DC
:10FCD000401801680906090EA1430160012016F0D1
:10FCE00057F870BD70B50500D9480C0000680028B1
:10FCF0000ED00021012016F029F8D649A80040189E
:10FD000001680906090E21430160012016F040F840
:10FD100070BD38B50024CD4D2A69824225D100201E
:10FD20002B0010330129286104D100220092AA6916
:10FD3000002106E0002907D1002200926A6901240F
:10FD40002100C548F6F770FA2BF010FF0500002CD3
:10FD500004D004217020FFF7C5FF03E004217020C8
:10FD6000FFF7A9FF28002BF005FF38BDF8B5040008
:10FD7000B64DA87F002820D02BF0F8FE2969060098
:10FD8000080003D0FAF295F90020286130002BF02A
:10FD9000F1FEEF88002C00D0EF892FF00DFFF9075E
:10FDA000C90F08430AD12BF0E1FE040004217020A2
:10FDB000FFF781FF20002BF0DDFEF8BD2BF0D6FE13
:10FDC0000090287FFF2803D15F20FFF781FC287770
:10FDD000687FFF2803D16020FFF77AFC68772878D6
:10FDE0002900002C00D0087A01268E570500002C2F
:10FDF00001D009268E578888002C00D088897D2361
:10FE0000DB00584388614888002C00D048897D2356
:10FE1000DB0058430C000028486101D1002506E0B2
:10FE2000012D04D104217020FFF75CFF03E00421C1
:10FE30007020FFF740FF207F80190106090E5F2028
:10FE4000FFF738FD607F80190106090E6020FFF77B
:10FE500031FD00982BF08EFE2FF0AEFEFF21491CE5
:10FE60000F403843A9D0002DA7D0A0690028A4D006
:10FE7000764B002200927848626910330121F6F730
:10FE8000D3F9F8BD70B504002BF070FE0500002C0E
:10FE900004D004217020FFF725FF03E00421702027
:10FEA000FFF709FF28002BF065FE70BDF0B50600D6
:10FEB0000C006A481500816A85B0694A1140816268
:10FEC000416A684A114341622BF050FE01901AF0DA
:10FED0004BFB029080210220FFF704FF0120F5F781
:10FEE0002BFB80210220FFF7E6FE0120F5F724FB23
:10FEF0002100300033F0B8EA5B48FFF700FC22062F
:10FF0000120E2900300003921AF094F9002E17D136
:10FF1000022D05D0032D03D00E2C01D1534F06E046
:10FF20001BF013F8012801D1514F00E0514F2BF085
:10FF30001DFE00903800FFF7E2FB00982BF01AFE40
:10FF40001AF0CAF94C48052C01D00D2C03D1012D13
:10FF500001D19A2106E0092C01D00D2C04D1022DEB
:10FF600002D1BA21FFF7A6FC6808012803D1434853
:10FF70008021FFF7A0FE012D07D1424840490160D2
:10FF8000416049008160C16001E01AF097F83000DB
:10FF9000FFF7ECFE02981AF0FDFA2A00310020006B
:10FFA000FFF747FD2A0031002000FFF717FD2A0068
:10FFB00031002000FFF791FC2A0031002000FFF7FC
:10FFC00062FD01982BF0D6FD2448416A254AD243B0
:10FFD00011404162F5F752FB220029003000FFF783
:10FFE0009EFAF5F792FB300016F0F7F8B51936EEE9
:10FFF0000100000004FB0000000400005F1CEE3F55
:020000021000EC
:10000000F5F746FB300015F061FF070001003000F6
:100010001AF07CF939003000FFF70FFB02210720AE
:1000200016F0B4FC33F02EEA002F04D01021072084
:1000300016F0ACFC03E01021072016F09CFC03999D
:100040002A003000FFF7F2FD01003000FFF708FB47
:10005000220029003000FFF723F9FFF7D1F81DE057
:10006000B404000424F90004002000902BF80000E0
:1000700000A80080FCFBFFFFC0000080943E04004D
:1000800080430400784304007C4304005E020000C7
:100090000D0400000101010140B0008033F0F6E9D9
:1000A000BE4D002F1FD0BE480068002817DB072078
:1000B00016F01DFC8009012803D1A869401CA86125
:1000C0000AE0022803D1E869401CE86104E0032843
:1000D00002D1286A401C28626869401C68610221BC
:1000E000072016F048FCF5F71AFBAE48026A032118
:1000F00089028A430262016A002E01D1020D01E0E9
:100100000122920211430162016A0122520211434B
:100110000162A54F002E01D1A44800E0A448386137
:100120002878B04213D030002E7015F08EFF3000CA
:1001300001F00FFC300001F022FC012803D1210066
:10014000300001F038FC2100300001F045FC386936
:10015000082108433861012005B0F0BD8F49FF2018
:1001600008707047F7B580010C00050C8B4A002120
:1001700008325056002800DC41420806000E1F26B7
:100180001F2800D206002BF0FBFC0700202C05D016
:10019000402C05D0802C05D0002404E0102402E07F
:1001A000202400E030242906090ECD20FFF78CFB27
:1001B000290ACE20FFF788FBD220FFF793FA4109E6
:1001C000029849013143002802D14020014301E057
:1001D000BF200140D220FFF777FB210080200143A0
:1001E000CC20FFF771FB38002BF0CEFCFEBDF3B541
:1001F0008FB02BF0C5FC0090D220FFF773FA40219E
:10020000084203D06B480926019003E06948093091
:100210000B2601900F9831000AF396EF00252C0071
:100220000395029528E0CC20FFF75CFA0009000155
:100230004006400E20430106090ECC20FFF744FB88
:10024000D120FFF74FFA0004A70004A9C851D0201D
:10025000FFF748FA04A9C9590002084304A9C85184
:10026000CF20FFF73FFA04A9C959084304A9C85190
:1002700003994018641C0390B442D4DB00982BF01F
:1002800083FC039800281AD0002404AF14E0A000D7
:1002900038580102081A03990BF3E0EB0F99000696
:1002A000000E085541190D0601992D0E09574143BD
:1002B00002980818641C0290B442E8DB09E00F9A27
:1002C000FF21701E0D001154019908560302181ADF
:1002D00002900F980178FF20401B0A180F990A70AE
:1002E000019A00215156414302980818109900299B
:1002F00002D0109900120880300011B0F0BD70B526
:1003000004002BF03DFC05002B48002C03D080217D
:10031000FFF7DBFC02E08021FFF7EEFC28002BF06A
:1003200033FC70BDF7B582B004000E002BF028FC42
:10033000102C019001D900200EE71F4DFF21113D27
:1003400060190700FFF7C1FC3106090E3800FFF7FE
:10035000D3FC102C02D11120002403E0A00812309D
:10036000A1074C0F0321A14009064019090E050001
:10037000FFF7ABFCF005C00FA0400106090E2800F6
:10038000FFF7BAFC0498A0404006010E2800FFF7D2
:10039000B3FC01982BF0F8FB0120DDE6900400048B
:1003A000002B008000280080C0A2008008A8000068
:1003B00008680000A43504009305000070B5F84DEE
:1003C0006969F8484165F84909688165F74800247A
:1003D0008461F4F733F91020F4F708F9E80CF4F726
:1003E00005F92C6070BD10B5EE4C0200616B206BFE
:1003F0000AF3FCEF7D22D2000AF3F8EF1EE8074B68
:100400000100000000FF0000000400000CC63D5386
:10041000E36AA26A0AF3BAEB10BDF8B57D220700C1
:10042000E54CD200616B206B0AF3EAEF05000E0089
:10043000E16AA06A3A000AF3E4EF33002A000AF303
:10044000A6EBF8BD10B5DC4C0200616B206B0AF323
:10045000D8EF7D22D2040AF3D4EFE36AA26A0AF34A
:1004600096EB10BD10B50400F2F7A2FB21002BF0B3
:1004700082E8D44A00230AF38AEB10BD70B5040069
:10048000CD4D01206872D0480168420C11430160D3
:10049000F5F724FACD494000085A64235843A8616F
:1004A0006043F4F78AF870BD10B50124F4F77AF8C8
:1004B000200010BDC0480079704770B5F4F787F888
:1004C0000600F4F793F8BC4C002526636563A16928
:1004D000E5624143BC48A1620168420C914301605E
:1004E0002079002804D10120FFF7ACFFF4F773F85E
:1004F000657270BD70B5B04C2069FFF77EFF6189F1
:100500000BF3B6EAE0610500B148A1690BF3B0EA6C
:100510000100A84201D8E06901E00800E1617D2105
:10052000C9000BF3A6EA206270BD0A2010B5FFF7E0
:10053000A5FFFFF7B9FF040010D0FFF7BEFFFFF7DC
:10054000D9FF9D48016A08000A2907D9FFF796FFDD
:10055000F4F728F8FFF7B1FFFFF7CCFF200010BD3C
:1005600070B50400944D0120687297480168420CF0
:1005700011430160F5F7B2F994494000085A64212B
:100580004143002CA96102D00800604305E0E869FE
:1005900048437D21C9000BF36CEAF4F70EF870BDF7
:1005A00085490A6A824206D84A7A002A03D14979E3
:1005B000002900D1D4E77047F3B583B000277E4906
:1005C0000D006B6B2A6B39000BF30EE802900C00E8
:1005D000E96AA86A049A0AF314EF05000E000622DD
:1005E0000AF30EEF3B0005220AF3D0EA0191AA0FAD
:1005F000B10011430090A8003B0005220AF3C6EAAF
:10060000029A2300121A8B411AD3684607C8801A2F
:10061000A14115D30722310028000AF3F2EE029A15
:1006200080186141644C4A07C0081043636B226B19
:10063000C9080AF3ACEAE162A06204986763206328
:1006400005B0F0BD70B55C4C6079002811D1F3F7AE
:10065000A9FFF3F7BCFF0500F3F7C8FF5A4A0100F2
:100660001068530C98431060A06948432900FFF7B5
:10067000A3FF2079002804D10120FFF7E3FEF3F760
:10068000AAFF0020607270BD70B5FF244A4D5A3435
:100690002B68C31A1B1BFF3BFF3B1B1F002B04DCFB
:1006A0004C49C86A401CC86203E0814201D88242BA
:1006B00001D2002070BD1800FFF7AFFE0600200039
:1006C000FFF7D0FE04002868FFF7A7FE8219230079
:1006D00000213000F4F70AF82879002806D12868AC
:1006E000FFF79BFE0004000CF3F754FF012070BDE0
:1006F000F8B505006846F5F7B4FB3748009900687F
:10070000814201D0F5F792FB34480099006881429C
:1007100001D0F5F78BFB324C324E2078FF280AD1FE
:100720000CF003F9002806D0002D04D03068220018
:100730000D21F5F78DFB00993068814201D0F5F766
:1007400075FB294800990068814201D0F5F76EFBDE
:10075000F8BD214838B50068F5F76EFB1F48006802
:10076000F5F76AFB1F4D2868F5F766FB1E48006821
:10077000F5F762FB1A4C2178FF2905D028686A46F4
:10078000F5F766FBFF20207038BD70B52BF002FA3C
:10079000104C05006068002805D12FF022FB0120D5
:1007A0006060002001E0606B401C606328002BF05B
:1007B000F5F970BD00A50080683700048022008034
:1007C00040A6008040420F0000210080E434040075
:1007D000002D31010C050004A002000410080004E3
:1007E0008CE9000478050004DC06000410B5FF4C19
:1007F0006068002803D02FF008FB0020606010BD67
:1008000010B5FAF72FFA04000CF057FC15EE62BE93
:1008100001000000FC020100000400000E903B7A81
:10082000204310BDF74810B50078C00705D0F4F795
:1008300043FFFEF763FBF4F786FF10BDF8B52BF01E
:10084000B3F904000021012015F09EFAF3F73BFEF6
:10085000ED49086BCA0C90430863012015F0B6FA05
:1008600020002BF0A5F915F0FBFCE54E0025B56046
:10087000E6488168AA2211438160E248E44F00788B
:10088000E44CC00721D02BF08FF9009020690B2198
:10089000884320612069316908432061A561F3F72D
:1008A000E1FEF3F766FFD948C038C760D948C030C9
:1008B0000168022211430160D749086808221043E9
:1008C000086000982BF074F907E0A561F3F7CAFE01
:1008D000F3F74FFFCD48C038C760FEF244FFCF4862
:1008E000CF49406D486120691021884320610CF098
:1008F00021F8002800D002202FF086FF04000DD040
:10090000200010F0A0FD002801D0042100E0052106
:100910000F2080012018006902F004F82BF044F940
:100920000400FFF76DFF20002BF042F9FFF71BFFDB
:10093000F9F23DFCF8BDB74810B501690B229143AF
:1009400001610169AE4AD2681143016100218161F0
:10095000F4F7B2FEFEF7D2FAF4F7F5FEAD48C03078
:100960000168022211430160AB480168082211436B
:10097000016010BDFFB583B004000027A94D0BF046
:10098000D9FF002800D002202FF03EFF060002D041
:10099000B068C004C00FFFF7B5FE2BF005F90022C8
:1009A0000290A148009200680822012101AB2CF0BE
:1009B00008FA019800281BD19C48002200684A21AF
:1009C000F8F283FF002802D00C98002810D0934939
:1009D000974B086E496E3F22184052050023114084
:1009E00059405840084303D1F5F759FE00280AD171
:1009F0008A488F4C026E416E3F2322405B051940AE
:100A00000266416620E0002C2AD0FEF27AFD0090BA
:100A10000498226863680F00101A00218B41009A25
:100A200019003B00121A8B410AD2009A20686168B3
:100A3000801AB941069A0599FFF730FE002806D1C1
:100A40006F48C169491CC161FFF7F8FE11E17348A5
:100A50006268216880304261016100F09EF9070000
:100A60006D4A10680821884310606A4AC0321068D5
:100A700002218843106067480169614A04231940D4
:100A80001161016999430161016903221143016107
:100A900046E05B48816A491C6D1E81623DD10100C0
:100AA000486A401C48620BF04FFF002813D0594899
:100AB0008169816901690B2291430161564A11687C
:100AC00008231943116001694D4A126911430161FC
:100AD000F9F26DFBCDE04F4DA8698006800F01282B
:100AE00003D147484169491C4161FFF724FF0FF0DA
:100AF0005FFA494908680822904308604549C031B7
:100B0000086802229043086028690421884328610C
:100B10002869032108432861424D0120F4F72AFD8A
:100B20003C4880698006800F0328B2D101F051FA59
:100B3000002804D13249086A401C086295E0002C64
:100B400008D000F02AF9069907008842F2D80598E3
:100B50008742EFD332484169304A516502214161F1
:100B60003448F3F76FFCFEF206FE28488168090A54
:100B70000902816027490869102210430861204852
:100B80000078022801D1022500E04025002C02D087
:100B900000F003F90700002F01D001200543002ECB
:100BA00004D00F2080013018006900E000200121EE
:100BB00001F0B8FEF4F782FFE807C00F01D0F3F7A9
:100BC00049FD1D4F422005403AD068060AD5102045
:100BD000F3F71AFD1020F3F729FD0420F3F7D0FDF9
:100BE000F3F7E0FDA8072BD53D003800F3F70CFD27
:100BF0002800F3F721FD0C20F3F7C2FD1EE00000F2
:100C00000C0500042CE90004002100804023008032
:100C1000EFFFFFFF40A6008000A30080170F1C1B02
:100C200001000000F8060100000400005D4AE8161B
:100C30006837000400A500808813000000C001C0D0
:100C40000000000418000400100010000010000054
:100C5000F3F7B2FD0320F3F79DFD5D4E0125B5606E
:100C6000002C16D000F0A3F80699884202D8059906
:100C700088420ED2306A0121090440183062FFF721
:100C8000E7FDFFF7D9FD02982AF09CFF002007B08E
:100C9000F0BD15F0FDFAFFF7C7FD4E4900280D60C5
:100CA00000D001E04C48056002982AF08BFF2AF042
:100CB00085FF04000021012015F070F8F3F717FC00
:100CC0004649086B38430863012015F089F8200075
:100CD0002AF078FFF5F22CFF4149884216D0414CAA
:100CE000606B0221884360633F48EFF787FCE2179F
:100CF0003E48009200680822012101AB2CF06BF8FD
:100D000031200003EFF77AFC394860630120BEE729
:100D100010B50BF023FE002803D02D488068002872
:100D200001D0FFF795FD10BDF8B5334A3148116881
:100D30000826B1431160314B1968022291431960B2
:100D40002E4CC03C2169224D04273940E9602169BD
:100D5000B943216121690B2211432161401E1BD13E
:100D6000FFF7F3FD0FF02EF920693840E8602069A5
:100D7000B843206120490868B04308601F4A1068E2
:100D8000022188431060A0698006800F012802D1EB
:100D9000A869401CA8611748A1698906890F032921
:100DA000D8D1F8BD012070471548407A704710B57A
:100DB000F3F7DDFC0400F3F7A8FC201A05D504497D
:100DC000086B401C0863002010BDFFF72AFB10BD14
:100DD0000C05000460070004640700040021008083
:100DE000E0B90004003400801010030000C001C00E
:100DF000F20101008813000000A3008000A700801A
:100E000068370004F8B50024FF484069FF4E8505A7
:100E1000AD0DB54203D001243000FBF74FF8FC4B79
:100E200000211F00383788001A58126838580260AD
:100E3000491C0929F7D9002C03D03000A843FBF73F
:100E400019F8F44B00201C1FC100CA1812680919B8
:100E50000A60401C0828F7D30020F8BD13000A00E0
:100E6000803010B5C16D806DFEF2C0FE10BD7CB546
:100E700014008030069A009301920A00C16D806DC3
:100E80002300FEF2CAFE7CBD38B51400049A00921D
:100E90002200FEF2D9FE38BDDF4B10B51862596250
:100EA0009862D962186359639863D963DA4B403307
:100EB000186059609860D960186159619861D9616A
:100EC0001A62FEF271F9D34900208C314860CE4994
:100ED000C039486310BD70B50500D0480C0041888A
:100EE000A1421CD0448028002FF058FC10F097FD40
:100EF000002814D1C549002C12D0022D01D11F2683
:100F000000E00F260D00002431002000FEF2BBFAA5
:100F100029002000FEF2C1FA641C032CF4DD70BD30
:100F20000F203F22FFF7B8FF70BD010000200E29FF
:100F300008D2B5484030072901D889000818006B4D
:100F40000004000C70470E2806D2AF4A4032072832
:100F500003D8800080180163704711637047F0B5B3
:100F6000002087B010F015FD002804D1012010F0FA
:100F700010FD002801D0012100E000210220059190
:100F800010F007FD0490032010F003FDA849009124
:100F90004C140599A24AA34BA34EA44F2500002947
:100FA0000393029201D015001C00049901431FD045
:100FB000022032F08EEA002801D035403C40032068
:100FC00032F086EA002803D00298039905400C40CD
:100FD000012032F07EEA002805D0009802990540F1
:100FE00003980D4004400498002801D035403C404F
:100FF0009048C562046307B0F0BD70B50600FFF20B
:10100000D3F98D4C250C002E08D0834900204031A7
:101010000862FFF7A4FFE068284316E011F0CDFA5C
:10102000002810D003210020FEF253FBD8E3A92EA4
:1010300001000000F40A010000040000A9259DA29F
:101040007648C03001680122D206914301600168F0
:101050000E224908490011430160E068A843E0609E
:1010600070BD6E4901235B04C0395A0000288869AD
:1010700004D0184388618869904303E01043886175
:1010800088699843886170476948006B7047684970
:1010900010B50400FC31FFF27DFD6D4A2000110007
:1010A0001031FFF2C4FD10BD614810B5A030FFF251
:1010B000DFFC6749543908000930FFF207FD10BD15
:1010C0005B4810B57830FFF286FC594960483431EE
:1010D0007438FFF2ADFC10BD5E49082010B50870F1
:1010E0005D490A2008705D49012008705C491020A4
:1010F00008705C491E20087019F012F819F00AF8FF
:10110000FFF7DEFFFFF7D0FF4948006B0006000E37
:10111000FFF7BDFF10BD10B5FFF7DEFF002018F090
:10112000CFFF10BDF8B522206B46187032205870E2
:101130003F4CFF2098702161A0690E001500002827
:1011400004D10120A061F4F743FA02E001200EF07F
:1011500023FF3000FFF2D2F800285ED0FFF75CFEDC
:1011600041482E4A406A010080310B7E40321362B2
:101170004B7E53623D4B06789E624088D862C869B8
:101180000104090C002083009B181963401C0728E8
:10119000F9DD0120FEF2F3FEFEF233F86846FEF2BE
:1011A0004CF821493439886A052212069043886236
:1011B0002548C030016889088900016022491E2045
:1011C0008862280001F0ADF8FFF21AF914493F22B5
:1011D0000F20FFF76BFE144925488C310860FFF2A1
:1011E000C9FF00F389FAFFF796FFFEF2C6F8FFF297
:1011F0007FFAFAF7F9F80021012019F052F9606935
:10120000FFF72FFF1B4801680B220904090C520449
:10121000891801601848016830E049E040A2008068
:10122000FF0300002018000434A9008080A0008083
:1012300058B901C0EBEFEBFFE8EEEAFFFAFEFAFF68
:10124000F8ECEAFFFFFFFEFF40A4008000A800804A
:10125000B8BB01C0E0F80004E1F80004E2F80004C3
:10126000E3F80004E4F800047CC7000400A6008052
:101270000100030000AE008000210080420C914379
:101280000160F3F783FAFF4908680122D206104390
:101290000860FD4908690A0D10430861FB4819F010
:1012A0008BF8F9488030016B032211430163012060
:1012B000F8BDF0B504210C05F54ECD058A00921954
:1012C00013681F043F0C2300002800D12B003B4370
:1012D0001360491C0729F1D9F0BDEA490420C0393F
:1012E00010B508600620F4F759F9EA480068C06BA9
:1012F00001F017F810BDF8B5002406008500E64897
:10130000405900287DD0F2F7B2F83106090E3702B5
:101310000028009136D0E14900980026FCF232FB0B
:10132000DF4901281CD14A69D84B0A3A13E0DA4850
:10133000A10028304059401819680006000E3843B3
:10134000014308683A21415E8E19B24202DC002C4A
:1013500057D01EE0641CD0484059A042E7D818E09E
:10136000CD48CA4A28304059126801240006000EB0
:101370003843024310683A22825E48690A38824242
:101380003FDA06E0C4484159C64AD468A14200D2B7
:101390004459C1484159091B4151C348BF494659A5
:1013A0000098FCF2EFFA012820D100201AE0BA4997
:1013B000B64B28314A591B681106090E39431943A7
:1013C00009680423498C121D5B1A9B079B0F59184F
:1013D000B14B091D28335A51D205D20D09030A43D6
:1013E0003260401CA042E2D309E00AE0AA49A20010
:1013F0002831485980184851C005C00D306001207F
:10140000F8BD0020F8BD10B50C00A0301100C37D60
:10141000827D20000C30FEF2F4FC10BD70B5060099
:101420008966086F0C000D000188821D143430009D
:101430002DF09AFD0200296F2000FEF2031818BD5E
:1014400001000000F00E010000040000FAFF4ECE83
:10145000FCFC28882084F9F795FD606880780009F5
:1014600005280CD1E069012149060843E0610A2101
:101470002800217009210C30FEF2BEFC04E022009D
:1014800029003000FFF7C9FFE16901221203A878A3
:101490009143E16105F3E7FB2565E06270BD010062
:1014A000CA007D4900207031511809687A4B7433A5
:1014B000D2181268D206D20E01E0091D401C0B1D85
:1014C000DB06DB0E9342F8D17047F7B582B00125F9
:1014D0000E0017002AF086FB0190C020C45D380082
:1014E00011F06FFA022811D07549097981420DD0A7
:1014F00015235B0172495843203942182C32E00011
:1015000080180300FF33B933181F06E06249E0007A
:1015100074314318624A091F40180C2E1AD1016811
:101520001B680E1DF606DB06F60EDB0E9E4201D191
:10153000002514E0029B12680326B6023243CE0651
:10154000F60E6401264332431360091D8906890E95
:10155000016004E05B48EFF765F8F4F73FFD0198A0
:101560002AF044FB280005B0F0BDF8B5050000895D
:101570006F694419206F00281ED0002F07D12AF070
:1015800031FB5048401CEFF74DF8F4F727FD2600DB
:10159000143621003800FFF74BFF280031F057FDCB
:1015A0006034217F3A003000FFF78FFF002804D11C
:1015B000280031F073FD0020F8BD0120F8BDF8B51A
:1015C0000500012700896E694419280031F03FFDAC
:1015D0007C20015D200032001430FFF776FF0028E8
:1015E00003D1280031F05AFD00273800F8BDF8B5C6
:1015F000050000896E694419002E00D1FEE7206FB6
:1016000027001437002834D021003000FFF710FFE6
:10161000786881780909092902D101227C210A55BB
:101620003179022914D1807800090D2810D1206F5A
:101630002030017803290BD14178002908D1C078E6
:101640008006000F0AF328FF0AF337FF7C210855B4
:10165000280031F0FCFC210030002DF0ABFB00280D
:1016600006D1280031F01AFD0120F4F713FCEFE752
:101670000120F8BDF8B50C0007008966086F0D0061
:10168000143400287ED060606120C05D0A49C00625
:10169000400F4000483117E0C0A80080C0A2008081
:1016A00000A00080C0AE0080F8BF01C0F40003C0FD
:1016B0007CCC0004A847040058B901C058180004A5
:1016C0004042000407000100095A21812988218431
:1016D00020002030417AAB78C9095B06C9015B0E56
:1016E00019434172E261E9886184A888002806D024
:1016F0006088000403D4210028002DF074FD606888
:101700002E0080780C360107890F012910D10009BD
:101710000A2807D1F9F718FC002801D0022104E0BB
:10172000002102E0082803D103213000FEF264FB0F
:10173000606880780107890F02290CD100090C2804
:1017400001D0042807D1F9F7FDF8002803D00221C1
:101750003000FEF251FBF9F7CDFB002815D009F05F
:10176000F2FA002803D1F1F78CFE00280DD02200F8
:1017700029003800FFF751FE21787E2041550021D5
:10178000300000E025E0FEF237FBF9F7B3FB00285C
:1017900007D009F072FA002803D0210028002DF0AC
:1017A00022FD220029003800FFF737FE2200290021
:1017B00038002DF028FC298AA181698AE181F1F79E
:1017C00060FE002803D021003800F1F7FEFE012062
:1017D0002565F8BDF8B504000F0000896669051994
:1017E000002E06D12AF0FEF9FF48EEF71BFFF4F7B2
:1017F000F5FB286F002824D02AF0F4F9009020008F
:1018000031F025FC3A0029003000FFF733FF0EE0ED
:10181000200031F043FC00982AF0E8F90120F4F7A9
:1018200039FB2AF0DFF90090200031F010FC29008C
:1018300030002DF0BFFA0028EAD000982AF0D6F93F
:101840000120F8BD7FB50400150002002B0E5BBA25
:1018500001000000EC12010000040000453A6B7D1D
:10186000E332511EE13001AE07C62200E032200013
:1018700000922A00D830FEF21AFB7FBD38B5040072
:10188000E034E27800920A008030C16DA378806D68
:10189000FEF253FE38BD0200803210B5D36D926D5A
:1018A0000800FEF29AF910BDD54A10B5126904235A
:1018B0001A40D44B5A64D44AFEF2B8FB10BDD0484B
:1018C00001698908890001610169CE4A526C11439E
:1018D00001617047CA4880698006800F032801D1E2
:1018E0000120704700207047002801D10820704770
:1018F00010207047C249203108757047C34A8000E4
:10190000821810B513688806800E01020404214372
:1019100000060143BE4803400B43136010BDBB4AA1
:101920008000801802688906890E0B0409060B43A3
:10193000B8490A401A4302607047B44B10B5403BA7
:1019400019688006800E0202040422430006024346
:10195000AF4801401143196010BDAC4B403B1968C2
:101960008006800E020400060243AA48014011438B
:101970001960704710B50524200017F046FE0100DD
:101980002000FEF2FFF8200017F042FEFF2801D0F1
:10199000FFF7D3FF200017F043FEFF2801D0FFF729
:1019A000DCFF10BDE03010B582780100C0788242C3
:1019B00008D20A784878824204D21BF0DCFF022861
:1019C00001D1052010BD002010BD10B519F075FB28
:1019D00010BD914810B58168090A0902816014F0B0
:1019E00040FC10BD8C4810B58168AA22114381606B
:1019F00014F038FC10BD08B5694619F0B1FD002897
:101A000004D16B4618705870987003E06B461878D4
:101A1000002804D1002031F07EED012002E00128F1
:101A200002D1002026F06BFA6B46187808BD0EB57F
:101A30006B4618705970009801A919F068FD0028CC
:101A400005D001A831F06AED012031F064ED0EBD42
:101A50001CB56B4618705970009801A919F06CFDFF
:101A6000002803D001A831F05EED012031F05EEDD9
:101A70001CBD70B52AF0C0F8684C002125000B0091
:101A80002835260050368A00A350491CAB5009293E
:101A9000B350F8DD2AF0B4F870BDF3B581B007009B
:101AA0002AF0AAF800902CF0ADFF01003800FEF2F9
:101AB0000FFB5B490A688018086052480299403061
:101AC000FEF213FB02988400564800590068534DFB
:101AD00029592E005036002907D152493831095969
:101AE00009682A002832315111513159029A3B00BC
:101AF000FEF21EFE002804D100982AF081F8002092
:101B0000FEBD3059001D30512859401C2851009805
:101B10002AF076F80120FEBD10B52AF06DF83F4A94
:101B200000218B00D358002B03D02AF069F8012044
:101B300010BD491C0929F4DD2AF062F8002010BD0F
:101B400070B501890C18216F2500406914350029F2
:101B500001D1002070BD2100FFF774FC6868807817
:101B60000009092801D1012101E06034217F28000A
:101B7000FFF793FF70BD70B502891418226F25001E
:101B800040691435002A01D1002070BD0A002100EF
:101B9000FFF77AFD6034217F2800FFF77EFF70BDDC
:101BA000F8B500252AF028F80027009000263CE030
:101BB00014481A495830845DA000085800281AD0EB
:101BC00010486C30005D002801D1092C13D1200091
:101BD000FFF7A5FB0500F1F75EFC002801D0002D02
:101BE00009D0092C06D007496C31085D401E085504
:101BF000044804700125761C092E15E00900010037
:101C000040A6008058B901C05150000040B000808B
